:020000040800F2
:10800000000001206103010845F7000849F7000856
:108010004DF7000851F7000855F700080000000070
:1080200000000000000000000000000059F70008F8
:108030005DF700080000000061F7000865F7000820
:10804000A9030108A9030108A9030108A90301085C
:10805000A9030108A9030108A9030108A90301084C
:10806000A9030108A9030108A903010869F7000889
:1080700099F70008A5F70008A9030108A90301085A
:10808000B1F70008BDF70008C9F70008A903010807
:10809000F9F70008A9030108A9030108A9030108C9
:1080A000A9030108A9030108A9030108A9030108FC
:1080B000A903010829F80008A9030108A903010878
:1080C000A9030108A9030108A9030108A9030108DC
:1080D000A903010859F8000865F8000891F800089C
:1080E000A9030108A9030108A90301080000000071
:1080F0000000000000000000000000000000000080
:108100000000000000000000A9030108A903010805
:10811000A9030108BDF80008A9030108A903010883
:10812000A9030108A9030108A9030108A90301087B
:10813000A9030108A9030108A9030108E9F8000837
:10814000A903010819F90008A9030108A9030108F6
:10815000000000000000000000000000000000001F
:10816000000000000000000000000000000000000F
:1081700000000000000000000000000000000000FF
:1081800000000000000000000000000000000000EF
:1081900000000000000000000000000000000000DF
:1081A00000000000000000000000000000000000CF
:1081B00000000000000000000000000000000000BF
:1081C00000000000000000000000000000000000AF
:1081D000000000000000000000000000000000009F
:0881E0005FF8E0F166666666D7
:1081E80010B5054C237833B9044B13B10448AFF3E9
:1081F80000800123237010BD280200200000000029
:108208000890010808B5034B1BB103490348AFF3B5
:10821800008008BD000000002C0200200890010822
:10822800034613F8012B002AFBD1181A01387047AE
:1082380081F0004102E000BF83F0004330B54FEA0F
:1082480041044FEA430594EA050F08BF90EA020F7C
:108258001FBF54EA000C55EA020C7FEA645C7FEA0F
:10826800655C00F0E2804FEA5454D4EB5555B8BF32
:108278006D420CDD2C4480EA020281EA030382EAA3
:10828800000083EA010180EA020281EA0303362D35
:1082980088BF30BD11F0004F4FEA01314FF4801C08
:1082A8004CEA113102D0404261EB410113F0004F1A
:1082B8004FEA03334CEA133302D0524263EB4303D1
:1082C80094EA050F00F0A780A4F10104D5F1200E6F
:1082D8000DDB02FA0EFC22FA05F2801841F10001CA
:1082E80003FA0EF2801843FA05F359410EE0A5F19E
:1082F80020050EF1200E012A03FA0EFC28BF4CF0CF
:10830800020C43FA05F3C01851EBE37101F0004584
:1083180007D54FF0000EDCF1000C7EEB00006EEB91
:108328000101B1F5801F1BD3B1F5001F0CD349081B
:108338005FEA30004FEA3C0C04F101044FEA445272
:1083480012F5800F80F09A80BCF1004F08BF5FEAF9
:10835800500C50F1000041EB045141EA050130BDD9
:108368005FEA4C0C404141EB0101013C28BFB1F5EB
:10837800801FE9D291F0000F04BF01460020B1FA36
:1083880081F308BF2033A3F10B03B3F120020CDA09
:108398000C3208DD02F1140CC2F10C0201FA0CF0E7
:1083A80021FA02F10CE002F11402D8BFC2F1200C4C
:1083B80001FA02F120FA0CFCDCBF41EA0C01904002
:1083C800E41AA2BF01EB0451294330BD6FEA04044B
:1083D8001F3C1CDA0C340EDC04F11404C4F1200236
:1083E80020FA04F001FA02F340EA030021FA04F348
:1083F80045EA030130BDC4F10C04C4F1200220FA9F
:1084080002F001FA04F340EA0300294630BD21FADC
:1084180004F0294630BD94F0000F83F4801306BFA2
:1084280081F480110134013D4EE77FEA645C18BF96
:108438007FEA655C29D094EA050F08BF90EA020F2D
:1084480005D054EA000C04BF1946104630BD91EA25
:10845800030F1EBF0021002030BD5FEA545C05D128
:108468004000494128BF41F0004130BD14F5800467
:108478003CBF01F5801130BD01F0004545F0FE41DB
:1084880041F470014FF0000030BD7FEA645C1ABF10
:10849800194610467FEA655C1CBF0B46024650EA47
:1084A800013406BF52EA033591EA030F41F4002173
:1084B80030BD00BF90F0000F04BF0021704730B5F9
:1084C8004FF4806404F132044FF000054FF00001CE
:1084D80050E700BF90F0000F04BF0021704730B58F
:1084E8004FF4806404F1320410F0004548BF404264
:1084F8004FF000013EE700BF42004FEAE2014FEAB9
:1085080031014FEA02701FBF12F07F4393F07F4F93
:1085180081F06051704732F07F4208BF704793F096
:108528007F4F04BF41F40021704730B54FF46074A9
:1085380001F0004521F000411CE700BF50EA0102AC
:1085480008BF704730B54FF000050AE050EA010255
:1085580008BF704730B511F0004502D5404261EBC5
:1085680041014FF4806404F132045FEA915C3FF406
:10857800D8AE4FF003025FEADC0C18BF03325FEAA3
:10858800DC0C18BF033202EBDC02C2F1200300FA54
:1085980003FC20FA02F001FA03FE40EA0E0021FA79
:1085A80002F11444BDE600BF70B54FF0FF0C4CF467
:1085B800E06C1CEA11541DBF1CEA135594EA0C0F19
:1085C80095EA0C0F00F0DEF82C4481EA030621EA54
:1085D8004C5123EA4C5350EA013518BF52EA03358F
:1085E80041F4801143F4801338D0A0FB02CE4FF041
:1085F8000005E1FB02E506F00042E0FB03E54FF071
:108608000006E1FB03569CF0000F18BF4EF0010E68
:10861800A4F1FF04B6F5007F64F5407404D25FEA64
:108628004E0E6D4146EB060642EAC62141EA555117
:108638004FEAC52040EA5E504FEACE2EB4F1FD0C59
:1086480088BFBCF5E06F1ED8BEF1004F08BF5FEAD7
:10865800500E50F1000041EB045170BD06F0004689
:1086680046EA010140EA020081EA0301B4EB5C0436
:10867800C2BFD4EB0C0541EA045170BD41F480112E
:108688004FF0000E013C00F3AB8014F1360FDEBF53
:10869800002001F0004170BDC4F10004203C35DA2F
:1086A8000C341BDC04F11404C4F1200500FA05F3B2
:1086B80020FA04F001FA05F240EA020001F0004253
:1086C80021F0004110EBD37021FA04F642EB0601C9
:1086D8005EEA430E08BF20EAD37070BDC4F10C04F3
:1086E800C4F1200500FA04F320FA05F001FA04F2B7
:1086F80040EA020001F0004110EBD37041F10001A3
:108708005EEA430E08BF20EAD37070BDC4F12005AD
:1087180000FA05F24EEA020E20FA04F301FA05F215
:1087280043EA020321FA04F001F0004121FA04F2BD
:1087380020EA020000EBD3705EEA430E08BF20EA8D
:10874800D37070BD94F0000F0FD101F000464000C7
:1087580041EB010111F4801F08BF013CF7D041EA49
:10876800060195F0000F18BF704703F0004652004D
:1087780043EB030313F4801F08BF013DF7D043EA1E
:108788000603704794EA0C0F0CEA135518BF95EAD4
:108798000C0F0CD050EA410618BF52EA4306D1D15B
:1087A80081EA030101F000414FF0000070BD50EA7A
:1087B800410606BF1046194652EA430619D094EA04
:1087C8000C0F02D150EA013613D195EA0C0F05D1EE
:1087D80052EA03361CBF104619460AD181EA030142
:1087E80001F0004141F0FE4141F470014FF00000FA
:1087F80070BD41F0FE4141F4780170BD70B54FF095
:10880800FF0C4CF4E06C1CEA11541DBF1CEA135514
:1088180094EA0C0F95EA0C0F00F0A7F8A4EB0504F6
:1088280081EA030E52EA03354FEA013100F08880ED
:108838004FEA03334FF0805545EA131343EA1263B6
:108848004FEA022245EA111545EA10654FEA00266B
:108858000EF000419D4208BF964244F1FD0404F524
:10886800407402D25B084FEA3202B61A65EB030580
:108878005B084FEA32024FF480104FF4002CB6EB3D
:10888800020E75EB030E22BFB61A754640EA0C00BD
:108898005B084FEA3202B6EB020E75EB030E22BFFD
:1088A800B61A754640EA5C005B084FEA3202B6EB3E
:1088B800020E75EB030E22BFB61A754640EA9C00FD
:1088C8005B084FEA3202B6EB020E75EB030E22BFCD
:1088D800B61A754640EADC0055EA060E18D04FEA8B
:1088E800051545EA16754FEA06164FEAC30343EA2B
:1088F80052734FEAC2025FEA1C1CC0D111F4801FF8
:108908000BD141EA00014FF000004FF0004CB6E7F0
:1089180011F4801F04BF01430020B4F1FD0C88BF8F
:10892800BCF5E06F3FF6AFAEB5EB030C04BFB6EB9A
:10893800020C5FEA500C50F1000041EB045170BD8D
:108948000EF0004E4EEA113114EB5C04C2BFD4EBBA
:108958000C0541EA045170BD41F480114FF0000E3E
:10896800013C90E645EA060E8DE60CEA135594EABA
:108978000C0F08BF95EA0C0F3FF43BAF94EA0C0FBD
:108988000AD150EA01347FF434AF95EA0C0F7FF432
:1089980025AF104619462CE795EA0C0F06D152EA86
:1089A80003353FF4FDAE1046194622E750EA41066A
:1089B80018BF52EA43067FF4C5AE50EA41047FF47B
:1089C8000DAF52EA43057FF4EBAE12E74FF0FF3CE0
:1089D80006E000BF4FF0010C02E000BF4FF0010CB1
:1089E8004DF804CD4FEA410C7FEA6C5C4FEA430C2A
:1089F80018BF7FEA6C5C1BD001B050EA410C0CBF79
:108A080052EA430C91EA030F02BF90EA020F0020DA
:108A1800704710F1000F91EA030F58BF994208BF41
:108A280090422CBFD8176FEAE37040F001007047FE
:108A38004FEA410C7FEA6C5C02D150EA013C07D155
:108A48004FEA430C7FEA6C5CD6D152EA033CD3D0A0
:108A58005DF8040B704700BF8446104662468C469A
:108A68001946634600E000BF01B5FFF7B7FF0028CD
:108A780048BF10F1000F01BD4DF808EDFFF7F4FFF6
:108A88000CBF012000205DF808FB00BF4DF808ED81
:108A9800FFF7EAFF34BF012000205DF808FB00BFA4
:108AA8004DF808EDFFF7E0FF94BF012000205DF8C6
:108AB80008FB00BF4DF808EDFFF7CEFF94BF01207B
:108AC80000205DF808FB00BF4DF808EDFFF7C4FF74
:108AD80034BF012000205DF808FB00BF4FEA410CBD
:108AE8007FEA6C5C02D150EA013C0AD14FEA430CA0
:108AF8007FEA6C5C02D152EA033C02D14FF00000DD
:108B080070474FF0010070474FEA410212F500121A
:108B180015D211D56FF47873B3EB625212D94FEABC
:108B2800C12343F0004343EA505311F0004F23FAA6
:108B380002F018BF404270474FF00000704750EAFB
:108B4800013005D111F0004008BF6FF000407047B8
:108B58004FF00000704700BF4FEA4102B2F1E04316
:108B680024BFB3F5001CDCF1FE5C0DD901F0004C0C
:108B78004FEAC0024CEA5070B2F1004F40EB83005C
:108B880008BF20F00100704711F0804F21D113F188
:108B98003872BCBF01F00040704741F480114FEAC1
:108BA8005252C2F11802C2F1200C10FA0CF320FA4A
:108BB80002F018BF40F001004FEAC1234FEAD32367
:108BC80003FA0CFC40EA0C0023FA02F34FEA4303D1
:108BD800CCE77FEA625307D150EA01331EBF4FF05A
:108BE800FE4040F44000704701F0004040F0FE4075
:108BF80040F40000704700BF80F0004002E000BF72
:108C080081F0004142001FBF5FEA410392EA030F6F
:108C18007FEA226C7FEA236C6AD04FEA1262D2EBB9
:108C28001363C1BFD218414048404140B8BF5B42BE
:108C3800192B88BF704710F0004F40F4000020F057
:108C48007F4018BF404211F0004F41F4000121F06D
:108C58007F4118BF494292EA030F3FD0A2F10102B7
:108C680041FA03FC10EB0C00C3F1200301FA03F1F5
:108C780000F0004302D5494260EB4000B0F5000F18
:108C880013D3B0F1807F06D340084FEA310102F1D7
:108C98000102FE2A51D2B1F1004F40EBC25008BF89
:108CA80020F0010040EA03007047490040EB000053
:108CB800013A28BFB0F5000FEDD2B0FA80FCACF154
:108CC800080CB2EB0C0200FA0CF0AABF00EBC25081
:108CD80052421843BCBFD0401843704792F0000F6F
:108CE80081F4000106BF80F400000132013BB5E7C2
:108CF8004FEA41037FEA226C18BF7FEA236C21D038
:108D080092EA030F04D092F0000F08BF084670479C
:108D180090EA010F1CBF0020704712F07F4F04D16A
:108D2800400028BF40F00040704712F100723CBF7D
:108D380000F50000704700F0004343F0FE4040F4A7
:108D4800000070477FEA226216BF08467FEA236365
:108D58000146420206BF5FEA412390EA010F40F450
:108D6800800070474FF0000304E000BF10F000439C
:108D780048BF40425FEA000C08BF704743F0964383
:108D880001464FF000001CE050EA010208BF70479E
:108D98004FF000030AE000BF50EA010208BF704725
:108DA80011F0004302D5404261EB41015FEA010C3A
:108DB80002BF84460146002043F0B64308BFA3F132
:108DC8008053A3F50003BCFA8CF2083AA3EBC25314
:108DD80010DB01FA02FC634400FA02FCC2F1200233
:108DE800BCF1004F20FA02F243EB020008BF20F06A
:108DF8000100704702F1200201FA02FCC2F12002D0
:108E080050EA4C0021FA02F243EB020008BF20EAC4
:108E1800DC7070474FF0FF0C1CEAD0521EBF1CEAF2
:108E2800D15392EA0C0F93EA0C0F6FD01A4480EAE0
:108E3800010C400218BF5FEA41211ED04FF00063C9
:108E480043EA501043EA5111A0FB01310CF00040F5
:108E5800B1F5000F3EBF490041EAD3715B0040EA1B
:108E6800010062F17F02FD2A1DD8B3F1004F40EBEB
:108E7800C25008BF20F00100704790F0000F0CF0BE
:108E8800004C08BF49024CEA502040EA51207F3A82
:108E9800C2BFD2F1FF0340EAC250704740F400005D
:108EA8004FF00003013A5DDC12F1190FDCBF00F04E
:108EB80000407047C2F10002410021FA02F1C2F1FC
:108EC800200200FA02FC5FEA310040F1000053EA98
:108ED8004C0308BF20EADC70704792F0000F00F0E6
:108EE800004C02BF400010F4000F013AF9D040EAEC
:108EF8000C0093F0000F01F0004C02BF490011F480
:108F0800000F013BF9D041EA0C018FE70CEAD1537D
:108F180092EA0C0F18BF93EA0C0F0AD030F0004CFD
:108F280018BF31F0004CD8D180EA010000F00040B1
:108F3800704790F0000F17BF90F0004F084691F06F
:108F4800000F91F0004F14D092EA0C0F01D14202A9
:108F58000FD193EA0C0F03D14B0218BF084608D172
:108F680080EA010000F0004040F0FE4040F40000BC
:108F7800704740F0FE4040F4400070474FF0FF0C4F
:108F88001CEAD0521EBF1CEAD15392EA0C0F93EA96
:108F98000C0F69D0A2EB030280EA010C49024FEAE8
:108FA800402037D04FF0805343EA111143EA1013A1
:108FB8000CF000408B4238BF5B0042F17D024FF459
:108FC800000C8B4224BF5B1A40EA0C00B3EB510F34
:108FD80024BFA3EB510340EA5C00B3EB910F24BF1D
:108FE800A3EB910340EA9C00B3EBD10F24BFA3EBA2
:108FF800D10340EADC001B0118BF5FEA1C1CE0D16A
:10900800FD2A3FF650AF8B4240EBC25008BF20F01C
:10901800010070470CF0004C4CEA50207F32C2BF70
:10902800D2F1FF0340EAC250704740F400004FF00D
:109038000003013A37E792F0000F00F0004C02BF3E
:10904800400010F4000F013AF9D040EA0C0093F008
:10905800000F01F0004C02BF490011F4000F013B62
:10906800F9D041EA0C0195E70CEAD15392EA0C0FCA
:1090780008D142027FF47DAF93EA0C0F7FF470AF02
:10908800084676E793EA0C0F04D14B023FF44CAF45
:1090980008466EE730F0004C18BF31F0004CCAD1DA
:1090A80030F000427FF45CAF31F000437FF43CAF16
:1090B8005FE700BF4FF0FF3C06E000BF4FF0010C38
:1090C80002E000BF4FF0010C4DF804CD4FEA40021A
:1090D8004FEA41037FEA226C18BF7FEA236C11D064
:1090E80001B052EA530C18BF90EA010F58BFB2EB17
:1090F800030088BFC81738BF6FEAE17018BF40F097
:10910800010070477FEA226C02D15FEA402C05D14A
:109118007FEA236CE4D15FEA412CE1D05DF8040BCF
:10912800704700BF844608466146FFE70FB5FFF762
:10913800C9FF002848BF10F1000F0FBD4DF808ED1A
:10914800FFF7F4FF0CBF012000205DF808FB00BF0B
:109158004DF808EDFFF7EAFF34BF012000205DF865
:1091680008FB00BF4DF808EDFFF7E0FF94BF0120B2
:1091780000205DF808FB00BF4DF808EDFFF7D2FFAF
:1091880094BF012000205DF808FB00BF4DF808EDF2
:10919800FFF7C8FF34BF012000205DF808FB00BFBF
:1091A8004FEA4002B2F1FE4F0FD34FF09E03B3EBEC
:1091B80012620DD94FEA002343F0004310F0004F2C
:1091C80023FA02F018BF404270474FF00000704782
:1091D80012F1610F01D1420205D110F0004008BF21
:1091E8006FF0004070474FF00000704753B94AB91C
:1091F800002908BF00281CBF4FF0FF314FF0FF3097
:1092080000F08CB9ADF1080C6DE904CE00F006F859
:10921800DDF804E0DDE9022304B070472DE9F047EA
:10922800089D8E4604468846002B4AD18A42174636
:1092380062D9B2FA82F64EB1C6F1200301FA06F8F5
:1092480020FA03F3B74043EA0808B4404FEA174E40
:10925800B8FBFEF11FFA87FC0EFB118801FB0CF22C
:10926800230C43EA08439A4209D9FB1801F1FF305D
:1092780080F0EB809A4240F2E88002393B449A1A27
:10928800B2FBFEF00EFB102200FB0CFCA3B243EA7B
:1092980002439C4509D9FB1800F1FF3280F0D780C2
:1092A8009C4540F2D4803B44023840EA014000210A
:1092B800A3EB0C031DB10022F340C5E90032BDE861
:1092C800F0878B4205D90DB1C5E900010021084698
:1092D800F5E7B3FA83F1002946D1734502D38242F8
:1092E80000F20881841A6EEB030201209046002DDB
:1092F800E5D0C5E90048E2E7002A00F09180B2FA1B
:1093080082F6002E40F0A5808A1A0121030C4FEA4C
:10931800174E80B2BCB2B2FBFEFC0EFB1C2243EA25
:10932800024304FB0CF29A4207D9FB180CF1FF38F0
:1093380002D29A4200F2E380C4469B1AB3FBFEF2C3
:109348000EFB123302FB04F440EA03439C4207D9A4
:10935800FB1802F1FF3002D29C4200F2CD80024697
:109368001B1B42EA0C40A5E7C1F120068B4022FAFC
:1093780006F71F432EFA06FA4FEA1749BAFBF9F81F
:109388000EFA01FE20FA06F309FB18AA1FFA87FC59
:1093980043EA0E0300FA01FE08FB0CF01C0C44EA39
:1093A8000A44A04202FA01F20AD93C1908F1FF3A2C
:1093B80080F09E80A04240F29B80A8F102083C44C5
:1093C800241A98B2B4FBF9F309FB134403FB0CFC11
:1093D80040EA0444A44509D93C1903F1FF3080F060
:1093E8008580A44540F28280023B3C4443EA084021
:1093F800A4EB0C04A0FB028C64454346E14664D30D
:1094080061D05DB1BEEB030264EB090404FA06F611
:1094180022FA01F31E43CC40C5E9006400214EE75F
:10942800B1FBF2FC010C41EA0E4180B240EA014274
:109438003B46B1FBF7F138463C46B846BE462026C7
:10944800A2EB080241EA0C4165E7014617E710461E
:109458002BE7C6F120012EFA01FCB7400EFA06FEF2
:1094680020FA01F141EA0E014FEA174EBCFBFEF863
:10947800BCB20EFB18CC08FB04F90A0C42EA0C42F9
:10948800B04091454FEA104380B23ED9BA1808F16E
:10949800FF3C01D291451FD8A2EB0902B2FBFEF9AD
:1094A80009FB04F80EFB192A8AB242EA0A4242452D
:1094B80029D2BA1809F1FF31C2D24245C0D2A9F166
:1094C80002013A44BCE7C6459BD2B8EB02036CEBF9
:1094D800070C0138E14694E7A7EB09094A44B2FBB7
:1094E800FEF9A8F1020C09FB04F8DBE703467DE767
:1094F800D04665E70846FAE63B44023A30E7ACF165
:10950800020C3B4419E749469AE7A2EB0902B2FB71
:10951800FEF9C44609FB04F8C4E700BF704700BF62
:1095280080B500AF06220549054807F099F80346BB
:10953800002B01D001F0B4FC00BF80BD4402002024
:10954800600200200E4B02689A4218D14FF0010CBD
:109558000C4A0D4B11880D4889B21980518889B27F
:109568005980918889B29980D18889B2D980118926
:1095780089B21981528992B25A8180F800C0704725
:109588000024014044020020500200205C02002018
:1095980080B584B000AF3B1D00221A605A609A6003
:1095A8003C4B3D4A1A603B4B4FF480729A60394BF2
:1095B80000221A73374B00221A75364B4FF40022DB
:1095C800DA61344B00225A60324B06221A61314864
:1095D80006F06EFF0346002B01D001F061FC032367
:1095E8007B600123BB600423FB603B1D19462948AF
:1095F80007F0EEF90346002B01D001F051FC0423DB
:109608007B600223BB603B1D1946224807F0E0F946
:109618000346002B01D001F043FC08237B600323A1
:10962800BB603B1D19461B4807F0D2F90346002BC7
:1096380001D001F035FC09237B600423BB603B1D8E
:109648001946144807F0C4F90346002B01D001F06D
:1096580027FC10237B600523BB603B1D19460D4882
:1096680007F0B6F90346002B01D001F019FC1123CD
:109678007B600623BB603B1D1946064807F0A8F926
:109688000346002B01D001F00BFC00BF1037BD468C
:1096980080BD00BF600200200024014080B58AB070
:1096A80000AF786007F1180300221A605A609A60C8
:1096B800DA607B681B68384A934268D1374B9B69EC
:1096C800364A43F400739361344B9B6903F4007387
:1096D8007B617B69314B9B69304A43F0040393619A
:1096E8002E4B9B6903F004033B613B692B4B9B6941
:1096F8002A4A43F008039361284B9B6903F0080347
:10970800FB60FB681823BB610323FB6107F11803A7
:109718001946234809F09AF80323BB610323FB6128
:1097280007F1180319461F4809F090F81E4B1F4A05
:109738001A601D4B00225A601B4B00229A601A4B7C
:109748008022DA60184B4FF480721A61164B4FF47E
:1097580080625A61144B20229A61134B4FF4805255
:10976800DA61114808F0E4FB0346002B01D001F050
:1097780097FB7B680C4A1A620B4A7B68536200228B
:109788000721122008F081FB122008F09AFB00BF85
:109798002837BD4680BD00BF0024014000100240AC
:1097A80000080140000C014090020020080002401F
:1097B80080B483B000AF0346FB80FB88002B01D048
:1097C800FB8800E0852318460C37BD4680BC7047EF
:1097D80080B584B000AF104B1B68B3F80F309BB254
:1097E8001846FFF7E5FF03467B817A8913469B00FD
:1097F80013445B00FB6040F232537B60FA687B687D
:109808009A4201D97B68FB60FB689AB2034B1A80C5
:1098180000BF1037BD4680BD0000002004000020B6
:1098280080B400AF024B1B881846BD4680BC704709
:109838000400002080B584B000AF0346FB80FFF72A
:10984800EFFF0346FB81FA88FB89934228BF134642
:109858009BB218461037BD4680BD000080B582B067
:1098680000AF03460A46FB711346BB71FB79072B11
:1098780050D801A252F823F0A1980008B198000826
:10988800C1980008D1980008E1980008F1980008EC
:10989800FF9800080F990008BB791A464FF48071A9
:1098A800214809F06EF936E0BB791A464FF4007189
:1098B8001D4809F066F92EE0BB791A464FF480611D
:1098C800194809F05EF926E0BB791A464FF40061A1
:1098D800154809F056F91EE0BB791A464FF4805135
:1098E800114809F04EF916E0BB791A4608210F48CD
:1098F80009F047F90FE0BB791A464FF400410C48CC
:1099080009F03FF907E0BB791A460821094809F030
:1099180038F900E000BFFB790749BA79CA5400BF9B
:109928000837BD4680BD00BF001801400010014047
:109938000008014000140140D402002080B483B024
:1099480000AF0346FB71FB79034AD35C18460C371A
:10995800BD4680BC704700BFD402002080B582B0ED
:1099680000AF0346FB71FB79062B3BD801A252F8E6
:1099780023F000BF99990008A5990008B19900083B
:10998800BD990008C9990008D5990008E19900080F
:109998000221174809F0DEF8034624E004211448A0
:1099A80009F0D8F803461EE08021124809F0D2F8E1
:1099B800034618E08021104809F0CCF8034612E06D
:1099C80010210E4809F0C6F803460CE008210B48A0
:1099D80009F0C0F8034606E00221064809F0BAF883
:1099E800034600E0002318460837BD4680BD00BF87
:1099F800000801400018014000140140000C01401B
:109A080080B483B000AF02237B600F4B9B690E4A82
:109A180043F0100393610C4B9B6903F010033B6008
:109A28003B680A4B5B6823F470227B681B04074978
:109A380013434B60054B4FF080521A6100BF0C373F
:109A4800BD4680BC704700BF0010024000100140B6
:109A580080B500AFFFF7D4FF00224FF480511848BB
:109A680009F08FF8174807F0ADF9FFF759FD002105
:109A78000020FFF7F3FE00210120FFF7EFFE002191
:109A88000220FFF7EBFE00210320FFF7E7FE00218D
:109A98000420FFF7E3FE00210520FFF7DFFE002189
:109AA8000620FFF7DBFE00210720FFF7D7FE064858
:109AB80005F086FD054805F083FD00BF80BD00BFA9
:109AC8000010014060020020DC0200200403002096
:109AD80090B587B000AF78600C4B7B610C4B3B6155
:109AE80079697868FFF78CF803461C463969786904
:109AF800FFF790F9034619462046FFF73FFA034659
:109B0800FB60FB6818461C37BD4690BD00007A44D0
:109B18003211803B00000000B0B586B000AFF8609D
:109B2800B9607A603B60F868FEF7D4FC1CA3D3E9FF
:109B38000023FEF763FE02460B4614461D46B8682E
:109B4800FEF7DAFC02460B4620462946FEF72CFDB6
:109B580002460B4610461946FEF7FEFF03467B6198
:109B680079687869FFF708FB0346002B01D00E4B94
:109B780010E079697868FFF743F803461946786971
:109B8800FFF7FCF9034619463868FFF743F903461F
:109B98003B613B6918461837BD46B0BDAFF300803E
:109BA8000000000000FEAF40000080BF80B588B014
:109BB80000AF0346FB710023FB61FB79002B03D048
:109BC8001C4BDB889BB202E01A4B9B889BB2FB6163
:109BD800FB79002B01D0012200E0002213469B00F4
:109BE8001344DB00144A1344FA691146184605F079
:109BF8000CFDB861BB69B3F57A6F01D9142315E080
:109C08000E4B7B610E4B3B610E4BFB60FB683A6968
:109C18007969B869FFF780FF03461846FFF758FFD0
:109C2800B860B868FFF7BCFA03461BB2184620377D
:109C3800BD4680BD50020020DC0200203333534073
:109C48000000A04000007A4480B500AF174B184AC6
:109C58001A60164B08225A60144B00229A60134B64
:109C68000022DA60114B4FF460221A610F4B4FF457
:109C780080125A610D4B00221A760C4B01225A763B
:109C88000A4B01229A76094B0122DA76074B002209
:109C98001A77064B01225A77044807F04AF9034617
:109CA800002B01D001F0FCF800BF80BD2C03002080
:109CB8000064004080B500AF174B184A1A60164B75
:109CC80010225A60144B00229A60134B0022DA606B
:109CD800114B4FF460221A610F4B4FF480125A61F6
:109CE8000D4B00221A760C4B01225A760A4B0122A0
:109CF8009A76094B0122DA76074B00221A77064B2F
:109D080001225A77044807F014F90346002B01D0C2
:109D180001F0C6F800BF80BD540300200068004071
:109D280080B58EB000AF786007F1200300221A607A
:109D38005A609A60DA607B681B68614A934253D123
:109D4800604B1B6801335F4A13605E4B1B68012B35
:109D58000BD15D4BDB695C4A43F00073D3615A4B0E
:109D6800DB6903F00073FB61FB69574B9B69564A3B
:109D780043F020039361544B9B6903F02003BB61BC
:109D8800BB6901233B6200237B620023BB6207F1AE
:109D9800200319464D4808F059FD02233B6202236F
:109DA8007B620323FB6207F120031946474808F04A
:109DB8004DFD474B5B683B633B6B23F4C0433B6300
:109DC8003B6B43F0E0633B633B6B43F4C0433B6353
:109DD8003F4A3B6B536000220321142008F055F8DA
:109DE800142008F06EF867E07B681B68394A9342D4
:109DF80062D1354BDB69344A43F08063D361324B1F
:109E0800DB6903F080637B617B692E4B1B68013340
:109E18002C4A13602B4B1B68012B0BD12A4BDB6997
:109E2800294A43F00073D361274BDB6903F00073C1
:109E38003B613B69244B9B69234A43F008039361C8
:109E4800214B9B6903F00803FB60FB6820233B62FE
:109E580000237B620023BB6207F1200319461E48DA
:109E680008F0F4FC40233B6202237B620323FB627D
:109E780007F120031946184808F0E8FC144B5B6802
:109E88007B637B6B43F0E0637B637B6B43F4800312
:109E98007B630F4A7B6B5360002200213F2007F051
:109EA800F4FF3F2008F00DF800220321412007F0BD
:109EB800ECFF412008F005F800BF3837BD4680BDEB
:109EC800006400407C0300200010024000140140A0
:109ED8000000014000680040000C014080B400AF61
:109EE800134B00221A70124B00225A70104B00229A
:109EF80062F06902DA7300221A740D4B0022DA77D5
:109F0800002283F82020002283F82120002283F8F1
:109F18002220074B002283F82320054B00225A6297
:109F2800034B002283F8282000BFBD4680BC704741
:109F38008003002080B500AF344B5A78344B1B782F
:109F48009A4206D0314B5A78314B1A702F4B002267
:109F58001A7000F041FC0346002B03D02B4B0B2258
:109F68005A7716E02B4B1B7B002B03D0274B07227D
:109F78005A770EE0274B5B7B002B03D0234B0A223A
:109F88005A7706E0214B9B7F002B02D11F4B002202
:109F98005A771E4B5B7F0021184600F0A1FD03464F
:109FA800002B06D0194B5B7F1A461B49052000F091
:109FB8009FFB06F04FFA0246184B1B68D31AB3F5FD
:109FC8007A7F20D3154B1B6803F57A73134A136005
:109FD8000E4B5B78082B06D10C4BD3F81F3001339E
:109FE8000A4AC2F81F30094B5B78012B0BD1074B8B
:109FF8000022DA77002283F82020002283F821202B
:10A00800002283F8222000BF80BD00BF800300200B
:10A01800AA0300207C09002020900108AC0300203E
:10A0280080B485B000AF78603960124BD3F81F3028
:10A03800FB607B68002B07D0FB680F4AA2FB032359
:10A048005B099AB27B681A803B68002B0CD0F968D0
:10A05800094BA3FB01235A0913461B019B1A9B00BA
:10A06800CA1AD2B23B681A7000BF1437BD4680BC0A
:10A07800704700BF800300208988888880B582B037
:10A0880000AF0346FB71414B1B78FA799A4203D122
:10A098003F4AFB79537075E03C4AFB7913703B4BA0
:10A0A8001B78002B03D13B49072000F021FB374BDD
:10A0B8001B78012B03D13849072000F019FB334BDB
:10A0C8001B78022B03D13549072000F011FB2F4BD9
:10A0D8001B78032B03D13249072000F009FB2B4BD7
:10A0E8001B78042B03D12F49072000F001FB274BD5
:10A0F8001B78052B03D12C49072000F0F9FA234BD4
:10A108001B78062B03D12949072000F0F1FA1F4BD1
:10A118001B78072B03D12649072000F0E9FA1B4BCF
:10A128001B78082B03D12349072000F0E1FA174BCD
:10A138001B78092B03D12049072000F0D9FA134BCB
:10A148001B780A2B03D11D49072000F0D1FA0F4BC9
:10A158001B780B2B03D11A49072000F0C9FA0B4BC7
:10A168001B780C2B03D11749072000F0C1FA074BC5
:10A178001B780D2B03D11449072000F0B9FA044AC3
:10A18800FB7953700837BD4680BD00BFA903002086
:10A19800800300203490010848900108609001086D
:10A1A8007890010890900108AC900108CC900108C3
:10A1B800EC9001080C910108249101083C910108D8
:10A1C80054910108709101088891010880B487B002
:10A1D80000AF134B5B889BB27B61114B5B899BB2D1
:10A1E8003B6140F2BA43FB60FB687A6903FB02F209
:10A1F8003B69B2FBF3F3BB60BB68A3F2BB6341F6F8
:10A20800186202FB03F3074A82FB03129211DB1761
:10A21800D31A7B607B6818461C37BD4680BC7047E4
:10A2280050020020D34D621080B500AF0E4B1B6862
:10A238009F229A620C4B1B6840F2C112DA620A4BE9
:10A248001B684FF4E1729A63074B1B6840F2C71210
:10A258005A630421044809F0CBFF0021024809F0A1
:10A26800C5FE00BF80BD00BF9C12002080B485B031
:10A2780000AF0346FB71FB794FF4E17202FB03F375
:10A288000B4A82FB03125211DB17D31AFB60094AEF
:10A29800FB791370084B1B68FA689A63064B1B68B6
:10A2A80001225A6300BF1437BD4680BC704700BF07
:10A2B8001F85EB51B40300209C12002080B400AF2E
:10A2C800024B1B781846BD4680BC7047B40300207B
:10A2D80080B500AFFFF77AFF0346034A1360024BCD
:10A2E8001B68184680BD00BFB003002080B582B04F
:10A2F80000AFFFF7EDFF7860214B1B78062B02D0EB
:10A308001F4B1B7838E07B6842F6F722934201DD49
:10A31800002331E07B68B3F5FA5F06DB7B6842F225
:10A328001072934201DC012326E07B6841F28732F8
:10A33800934206DD7B6841F65832934201DC0223E2
:10A348001AE07B68B3F5FA6F05DB7B68B3F57A6FC3
:10A3580001DC032310E07B6813F57A7F05DB7B685B
:10A36800B3F5FA6F01DC042306E07B68054A9342E3
:10A3780001DA052300E0062318460837BD4680BDEC
:10A388000600002009D5FFFF80B400AF024B1B7800
:10A398001846BD4680BC70470700002080B582B0D3
:10A3A80000AFFFF7A3FF0346FB71FB79062B06D12D
:10A3B800134B06221A70134B00221A701DE0104B23
:10A3C8001B78FA799A4206D00D4AFB7913700D4B27
:10A3D80001221A7011E00B4B1B78632B05D8094B2F
:10A3E8001B780133DAB2074B1A70064B1B78632BC4
:10A3F80003D9034B1A78044B1A700837BD4680BD41
:10A4080008000020B50300200700002080B582B0B6
:10A4180000AF06F01FF80246224B1B68D31A002B28
:10A428003CDD06F017F803461E4A1360FFF7B6FF37
:10A43800FFF7AAFF0346FB711B4B1B78BB711B4B35
:10A448001B78002B09D11A4AFB791370194ABB797A
:10A458001370164B01221A7021E0154B1B78FA79FC
:10A468009A420AD0124B1B781A46FB7912490720E8
:10A4780000F03EF90E4AFB7913700E4B1B78BA793F
:10A488009A420CD00B4B1B781A46BB790B49072014
:10A4980000F02EF9074ABB79137000E000BF0837B7
:10A4A800BD4680BDB8030020B4030020BC030020D3
:10A4B80009000020BD030020A0910108BC910108FB
:10A4C80080B500AF064B074A1A60054807F013FD30
:10A4D8000346002B01D000F0E3FC00BF80BD00BFA5
:10A4E800C00300200030024080B485B000AF78601F
:10A4F8007B681B68094A93420BD1094B5B69084A80
:10A5080043F040035361064B5B6903F04003FB6073
:10A51800FB6800BF1437BD4680BC7047003002405E
:10A528000010024080B584B000AFF860B9607A606E
:10A538007B689BB21946B86800F006F87B68184635
:10A548001037BD4680BD000080B485B000AF78608C
:10A558000B467B8072B600BF0023FB8145E0284B89
:10A56800B3F804349BB2B3F5806F18D3244BB3F817
:10A5780002349BB201335A42C3F30903C2F30902FE
:10A5880058BF53429AB21E4BA3F802241C4BB3F88F
:10A5980004349BB2013B9AB2194BA3F80424FB89FB
:10A5A8007A681344164AB2F8002492B21978144B08
:10A5B8009954134BB3F800349BB201335A42C3F396
:10A5C8000903C2F3090258BF53429AB20C4BA3F8CD
:10A5D80000240B4BB3F804349BB201339AB2084BF6
:10A5E800A3F80424FB890133FB81FA897B889A420A
:10A5F800B5D362B600BF00BF1437BD4680BC7047F4
:10A60800C803002080B483B000AF72B600BF064B09
:10A61800B3F80434FB8062B600BFFB8818460C37D9
:10A62800BD4680BC704700BFC803002080B582B01B
:10A6380000AF72B600BF2D4BB3F804349BB2002BA9
:10A6480002D162B600BF4EE0284BB3F80434FB8059
:10A65800FB88802B01D98023FB80244BB3F802347C
:10A668009BB2C3F58063BB80FA88BB889A4201D944
:10A67800BB88FB801D4BB3F804349BB2FA889A421E
:10A688000CD11A4BB3F802349BB21A46174B134439
:10A69800F9885022184604F0C5FB0BE0134BB3F8B9
:10A6A80002349BB21A46114B1344F98851221846BA
:10A6B80004F0B8FB0D4BB3F802349AB2FB8813448C
:10A6C8009BB2C3F309039AB2084BA3F80224074BC1
:10A6D800B3F804349AB2FB88D31A9AB2034BA3F89E
:10A6E800042462B600BF0837BD4680BDC8030020F9
:10A6F8000EB480B585B000AF0346FB71154AFB79EF
:10A70800137007F12003BB60BB68FA69FE21124889
:10A718000CF090FBF860FB68002B01DAFB6812E094
:10A72800FB68FD2B01DDFE23FB60FB680133094A52
:10A738000021D154FB689BB202339BB219460548ED
:10A74800FFF702FFFB6818461437BD46BDE8804096
:10A7580003B07047D0070020D107002080B582B031
:10A7680000AF1C4B5B691B4A43F001035361194B53
:10A778005B6903F001037B607B68002201210B20E9
:10A7880007F083FB0B2007F09CFB002204210C2020
:10A7980007F07BFB0C2007F094FB002201210D2021
:10A7A80007F073FB0D2007F08CFB0022012110201D
:10A7B80007F06BFB102007F084FB00220421112016
:10A7C80007F063FB112007F07CFB00BF0837BD468C
:10A7D80080BD00BF0010024080B400AF024B1B7860
:10A7E8001846BD4680BC7047D008002080B500AF31
:10A7F800064B1B78002B07D1044B01221A70044921
:10A808000420FFF775FF00E000BF80BDD0080020DE
:10A81800D891010880B58AB000AF07F1140300226F
:10A828001A605A609A60DA60944B9B69934A43F0C5
:10A8380010039361914B9B6903F010033B613B69E3
:10A848008E4B9B698D4A43F0040393618B4B9B6944
:10A8580003F00403FB60FB68884B9B69874A43F05D
:10A8680008039361854B9B6903F00803BB60BB68D1
:10A87800824B9B69814A43F0400393617F4B9B69FC
:10A8880003F040037B607B687C4B9B697B4A43F009
:10A8980020039361794B9B6903F020033B603B687D
:10A8A80000224FF40F71764808F06BF9002248F245
:10A8B8006001744808F065F900224FF4F8517248B5
:10A8C80008F05FF900224FF44861704808F059F920
:10A8D800002218216E4808F054F94FF401737B6187
:10A8E8000123BB610023FB6103233B6207F11403CF
:10A8F8001946634807F0AAFF38237B610123BB612F
:10A908000023FB6102233B6207F1140319465C48EC
:10A9180007F09CFF02237B610023BB610023FB61DE
:10A9280007F114031946574807F090FF04237B6189
:10A938000023BB610223FB6107F114031946514848
:10A9480007F084FF60237B610123BB610023FB6167
:10A9580003233B6207F1140319464A4807F076FFC0
:10A9680044F282037B610023BB610023FB6107F192
:10A9780014031946444807F069FF4FF4F8537B6104
:10A988000123BB610023FB6102233B6207F114032F
:10A9980019463D4807F05AFF4FF440637B61012395
:10A9A800BB610023FB6103233B6207F114031946D3
:10A9B800364807F04BFF4FF400437B610123BB612E
:10A9C8000023FB6102233B6207F1140319462D485B
:10A9D80007F03CFF18237B610123BB610023FB6167
:10A9E80002233B6207F114031946294807F02EFF9A
:10A9F80080237B610023BB610023FB6107F1140303
:10AA08001946234807F022FF18237B610023BB6106
:10AA18000023FB6107F1140319461C4807F016FFD1
:10AA280080237B610123BB610023FB6102233B621E
:10AA380007F114031946154807F008FF4FF440734F
:10AA48007B611223BB6103233B6207F114031946A0
:10AA58000E4807F0FBFE0F4B5B687B627B6A43F096
:10AA6800E0637B627B6A43F002037B62094A7B6A8C
:10AA7800536000BF2837BD4680BD00BF00100240AC
:10AA8800001001400008014000180140000C01407E
:10AA9800001401400000014080B400AFBFF34F8FA5
:10AAA80000BF064BDB6803F4E0620449044B134320
:10AAB800CB60BFF34F8F00BF00BFFDE700ED00E0A4
:10AAC8000400FA0580B400AF034B044A9A6000BF43
:10AAD800BD4680BC704700BF00ED00E00080000864
:10AAE80080B485B000AF03460A46FB711346BB71BC
:10AAF800BB791F2B01D900230EE00023FB73BB7920
:10AB0800084AD35CFA799A4201D00123FB73BB79D6
:10AB18000449FA79CA54FB7B18461437BD4680BCF1
:10AB2800704700BFD408002080B584B000AF7860BB
:10AB380005F090FCB8607B68FB60FB68B3F1FF3FF1
:10AB480010D00F4B1B781A46FB681344FB6009E0D2
:10AB580003F090F900F016F8FFF758FC02F03EFFFA
:10AB680004F006F805F076FC0246BB68D31AFA68CA
:10AB78009A42EDD800BF00BF1037BD4680BD00BF68
:10AB88005800002080B582B000AF05F063FC786003
:10AB98002A4B1B687A68D31A092B49D9274A7B683C
:10ABA80013600320FEF7DAFE0346002B0CBF0123D7
:10ABB8000023DBB2FB70FB78002B02D1204B002274
:10ABC8001A701F4B1B78002B34D1FB78002B2BD02D
:10ABD8001C4B1B68002B02D11B4B01221A70194B0E
:10ABE8001B680A33174A1360164B1B6841F28832F8
:10ABF800934202D1144B03221A70124B1B6849F678
:10AC08004042934217D912220021002004F00AF989
:10AC180000BF0E4B93F84130DBB2212BF9D00A204C
:10AC280005F022FCFFF738FF064B00221A6002E00D
:10AC380000BF00E000BF0837BD4680BDF408002013
:10AC48000A000020F808002080030020BC13002020
:10AC580080B500AF0B4806F08BFBFEF7F5FF0948FF
:10AC680006F042FB0346002B01D000F019F902213F
:10AC7800044806F0EAFD0346002B01D000F010F965
:10AC880000BF80BD2C03002090B583B002AFFFF752
:10AC980019FF05F087FB07F099FF00F091F8FFF71F
:10ACA800B9FDFFF75BFDFEF773FCFEF7CDFFFFF77D
:10ACB80001F802F045FF04F07DFF05F0FBF8FFF70F
:10ACC800FFFB05F0A3F805F0CBF805F01DF904F03B
:10ACD800E3FEFEF7BDFE02F05DFE4FF4967005F050
:10ACE800C3FB03F08FFB03F019FF2E490720FFF782
:10ACF800FFFC03F0EFFE03F0BFFB2B4B1B889BB25E
:10AD08001A462A490720FFF7F3FC274B9B781A4677
:10AD180027490720FFF7ECFCFEF782FD03461A4699
:10AD2800244BA3FB0223DB089BB21C46FEF778FDED
:10AD380003461A461F4BA3FB0213D9080B469B0078
:10AD48000B445B00D31A9BB222461B490720FFF72E
:10AD5800CFFC154B9B889BB21A46134BDB889BB2E2
:10AD68001946114B1B899BB200930B4613490720C8
:10AD7800FFF7BEFCFFF76CFF01F0CCFAFFF7AEF867
:10AD880001F0E2FB01F08CFC0A20FFF7CDFE00F099
:10AD98008DF8FFF7CFF802F065FA0A20FFF7C4FE36
:10ADA80000BFEDE754920108841200206892010860
:10ADB8007C920108CDCCCCCC90920108B4920108C9
:10ADC80080B59CB000AF07F138033822002118463F
:10ADD8000CF03EF807F1240300221A605A609A60CA
:10ADE800DA601A613B1D2022002118460CF030F869
:10ADF8000523BB634FF480333B6404237B64012346
:10AE0800BB640123FB644FF48033FB630223BB65FF
:10AE18004FF48033FB654FF4E0133B6602237B66F7
:10AE28004FF4C063BB664023FB6607F1380318463E
:10AE380007F09CFF0346002B01D000F031F80F23E8
:10AE48007B620223BB620023FB624FF480633B6397
:10AE580000237B6307F124030221184608F09CFABB
:10AE68000346002B01D000F01BF803237B604FF44E
:10AE78008073BB604FF40043FB603B1D184608F02D
:10AE880081FC0346002B01D000F00AF8034B012295
:10AE98001A6000BF7037BD4680BD00BF70004242D7
:10AEA80080B400AF72B600BF00BFFDE72DE9B04F18
:10AEB80086B000AF434B00221A70434B5B78082BD7
:10AEC80003D1404B01221A7602E03E4B00221A764B
:10AED80005F0C0FA78613B4B5B687A69D31A3B612D
:10AEE800384A7B695360384BD3F8033000229A46BE
:10AEF80093463B6900229846914608FB0BF20AFBF1
:10AF080009F31344AAFB08452B441D464FF47A72F3
:10AF18004FF0000320462946FEF768F902460B4623
:10AF2800C7E90223274BD3E90201D7E90223841892
:10AF38003C6041EB03037B60224BD7E90012C3E975
:10AF48000212204BD3E902014FF461624FF0000373
:10AF5800FEF74CF902460B461A4B1A61194B1B7E39
:10AF6800002B1CD0174B1A69164B5B699A4208D301
:10AF7800144B1A69134B5B69D31A134AC2F807308A
:10AF88001AE0114B0022DA7100221A7200225A725A
:10AF980000229A720B4B1B690A4A53610CE00A4B58
:10AFA8000022DA7100221A7200225A7200229A7262
:10AFB800044B1B69034A536100BF1837BD46BDE8FF
:10AFC800B08F00BF000900208003002080B483B048
:10AFD80000AF0346FB71FB79002B0BD0FB79012BEB
:10AFE80008D0FB790A2B05D0FB790C2B02D0FB7912
:10AFF8000B2B01D1012300E00023DBB218460C37EC
:10B00800BD4680BC7047000080B400AF114B96224B
:10B018001A80104B00225A800F4A0E4B1B6813608F
:10B028000E4A0C4B1B6813600D4B00221A700D4B17
:10B0380000221A700C4B00221A700C4B00221A7056
:10B048000B4B00221A600B4B00221A6000BFBD4652
:10B0580080BC70472009002024090020280900200E
:10B068002C0900202D0900202E0900202F0900207E
:10B07800300900203409002080B582B000AF0346B3
:10B088000A46FB801346BB80BB881846FEF7D2FBF6
:10B098000346BB80064AFB881380054ABB88538059
:10B0A800044B01221A7000BF0837BD4680BD00BF9F
:10B0B800240900202C09002080B582B000AF05F0DB
:10B0C800C9F97860254BDB7D002B0BD0234B9B7F88
:10B0D800002B07D0224B1B781846FFF777FF034653
:10B0E800002B0CD01F4B00221A701F4B00221A7025
:10B0F8001E4B00221A601E4B00221A602BE0174BD1
:10B10800B3F81B309BB2142B02D9164B01221A70CC
:10B11800134B1B78082B02D1124B01221A700F4BCC
:10B12800B3F815309BB21D2B12D9114B1B68002B9D
:10B1380003D10F4A7B6813600DE00D4B1B687A68DA
:10B14800D31AB3F5FA7F06D3064B01221A7002E030
:10B15800074B00221A600837BD4680BD80030020D7
:10B16800E40D00202E0900202F09002030090020BE
:10B178003409002080B400AF024B1B781846BD4646
:10B1880080BC70472C09002080B400AF084B1B78A6
:10B19800002B01D1002307E0064BDB79063B042B8B
:10B1A80001D8012300E000231846BD4680BC704743
:10B1B8002D0900207C090020B0B588B000AF786068
:10B1C8001C4BDB7A3B731B4B9B7A7B731A4BB3F894
:10B1D80013309BB2FB81184BB3F815309BB23B82FE
:10B1E800164B1B78BB74144BDB7DFB74114BDB795E
:10B1F800052B01D1012300E000233B750D4B1B7B80
:10B208007B750C4B5B7BBB750D4B1B78FB750D4B36
:10B218001B68BB6105F01EF90346FB617B681D4690
:10B2280007F10C040FCC0FC523682B607868203712
:10B23800BD46B0BD7C090020800300202E090020F7
:10B248002F09002030090020B0B58EB002AF2B4B7B
:10B258001B78002B03D02A4B1B78002B01D000232E
:10B2680048E03B461846FFF7A7FF07F118043D469C
:10B278000FCD0FC42B68236007F118031A46214924
:10B28800214800F0ADF8034687F82F3097F82F30A3
:10B29800012B19D11D4A1B4B1B681360184B012247
:10B2A8001A70164B00221A70174B1B881A46174B38
:10B2B8001B881946154B5B8800930B4614490720D9
:10B2C800FFF716FA022315E0124B5B7A002B01D127
:10B2D80000230FE00B4B1B880A4A528819460020AE
:10B2E80001F076F8084A074B1B681360034B0022ED
:10B2F8001A70012318463037BD46B0BD2C0900200E
:10B308002D090020240900202009002028090020F8
:10B31800F09101087C09002080B483B000AF786008
:10B328007B68002B03D07B68034A1068186000BF55
:10B338000C37BD4680BC70472809002080B500AF97
:10B348000E4A0F4B1B6813600E4B00221A700E4BEF
:10B358001B780133DAB20C4B1A7005F07BF8034600
:10B368000A4A13600A4BB3F813309BB21A460949CC
:10B378000720FFF7BDF900BF80BD00BF20090020EE
:10B38800280900202D0900202F090020300900205D
:10B39800800300201492010880B500AF0A4B0022F8
:10B3A8001A700A4A0A4B1B6813600A4B01221A706A
:10B3B800094BB3F813309BB21A4608490520FFF72A
:10B3C80097F900BF80BD00BF2D0900202409002087
:10B3D800280900202C09002080030020349201084D
:10B3E80080B487B000AFF860B9607A60FB68002B62
:10B3F80005D0BB68002B02D07B68002B01D100234D
:10B4080069E0BB681A88FB681B889A4201D300234D
:10B4180061E0FB681A88BB681B88D31AFB82FB8A29
:10B42800312B01D8002356E0FB685B88142B03D826
:10B43800BB685B88142B01D900234CE07B689B8890
:10B448001D2B01D9002346E07B685A88BB681B88FE
:10B458000F339BB29A4201D800233CE07B689B796A
:10B46800002B01D0002336E07B68DB79002B01D16B
:10B47800002330E07B681B7A002B01D100232AE0EF
:10B488007B681B78002B01D1002324E07B685B7864
:10B49800002B01D100231EE07B685B7A002B03D1CF
:10B4A8007B689B7A002B01D0002314E07B68DB7A51
:10B4B800032B01D900230EE07B68DB68002B09D041
:10B4C8007B681A697B68DB68D31AB3F5FA6F01D217
:10B4D800002300E0012318461C37BD4680BC704796
:10B4E80080B483B000AF0346FB71FB790E2B3FD8C5
:10B4F80001A252F823F000BF3DB5000841B500088D
:10B5080045B5000849B500084DB5000851B5000813
:10B5180055B5000859B500085DB5000861B50008C3
:10B5280065B5000869B5000871B500086DB5000873
:10B5380075B50008114B1CE0114B1AE0114B18E0CF
:10B54800114B16E0114B14E0114B12E0114B10E0B7
:10B55800114B0EE0114B0CE0114B0AE0114B08E0C7
:10B56800114B06E0114B04E0114B02E0114B00E0D7
:10B57800114B18460C37BD4680BC7047CC92010869
:10B58800D4920108DC920108E4920108EC920108C7
:10B59800F492010800930108089301081093010828
:10B5A80018930108209301082C9301083893010887
:10B5B80044930108509301085C930108F0B5ADB0BD
:10B5C80018AF04F047FFF8647F4B5B78082B40F016
:10B5D800F4807E4B1B68FA6CD31AB3F5FA6FC0F08F
:10B5E800EE807A4AFB6C1360FFF7C4FD0346002B1C
:10B5F80004D1FFF7C9FD0346002B01D0012300E069
:10B60800002387F84B30724BDB791846FFF768FF49
:10B6180084466D4BB3F80F309BB29E466A4BB3F825
:10B6280011309BB26B4AA2FB0323DB089BB27B64FD
:10B63800654BB3F811309AB2664BA3FB0213D908D5
:10B648000B469B000B445B00D31A9BB23B645E4BDA
:10B65800B3F80F309BB2FB635B4BB3F81B309BB264
:10B668005C4AA2FB0323DB089BB2BB63564BB3F8CF
:10B678001B309AB2574BA3FB0213D9080B469B0009
:10B688000B445B00D31A9BB27B63534B1B883B6311
:10B69800524B1B884F4AA2FB0323DB089BB2FB6279
:10B6A8004E4B1A884B4BA3FB0213D9080B469B0041
:10B6B8000B445B00D31A9BB2BB62434BB3F8133005
:10B6C8009BB27B62404BB3F815309BB2414AA2FB58
:10B6D8000323DB089BB23B623B4BB3F815309BB2AC
:10B6E80019463F4B83FB01239A10CB17D21A1346F6
:10B6F8009B0013445B00CA1AFA61334BDB7DBB61C4
:10B70800314B1B7E7B61324B5B7A3B61304B9B7AC2
:10B71800FB602F4BDB7ABB602D4B1B787B602A4B81
:10B7280093F823303B6097F84B00274B5B7F1E460E
:10B73800274B1B7F1D46264B5B7F1C46244B9B7F5C
:10B748001946284B1B68002B04D0264B1A68FB6C43
:10B758009B1A01E042F20F731793169115941495F2
:10B76800139612903B6811937B681093BB680F93F4
:10B77800FB680E933B690D937B690C93BB690B9334
:10B78800FB690A933B6A09937B6A0893BB6A079330
:10B79800FB6A06933B6B05937B6B0493BB6B03932C
:10B7A800FB6B02933B6C01937B6C00937346624680
:10B7B8000D490720FEF79CFF02E000BF00E000BF34
:10B7C8005437BD46F0BD00BF80030020A809002003
:10B7D8007C090020CDCCCCCCA0090020A2090020F7
:10B7E800676666669C09002060930108F0B5ADB0F5
:10B7F80016AF034687F84730894B1B7F87F85430CC
:10B80800874B5B7F87F85030854B9B7F87F84C30A0
:10B8180097F8543003F00103DBB2002B02D0814BC0
:10B828003B6401E0804B3B6497F8543003F002031B
:10B83800DBB2002B02D07D4BFB6301E07A4BFB634C
:10B8480097F8543003F00403DBB2002B02D0784B96
:10B85800BB6301E0744BBB6397F8543003F00803F3
:10B86800DBB2002B02D0734B7B6301E06E4B7B6332
:10B8780097F8543003F01003DBB2002B02D06E4B64
:10B888003B6301E0684B3B6397F8543003F02003B7
:10B89800DBB2002B02D0694BFB6201E0624BFB621A
:10B8A80097F8543003F04003DBB2002B02D0644B0E
:10B8B800BB6201E05C4BBB6297F8503003F00103B8
:10B8C800DBB2002B02D05F4B7B6201E0564B7B6200
:10B8D80097F8503003F00203DBB2002B02D05A4B2A
:10B8E8003B6201E0504B3B6297F8503003F0040391
:10B8F800DBB2002B02D0554BFB6101E04A4BFB61E8
:10B9080097F8503003F00803DBB2002B02D0504BFD
:10B91800BB6101E0444BBB6197F8503003F0100362
:10B92800DBB2002B02D04B4B7B6101E03E4B7B61CD
:10B9380097F8503003F02003DBB2002B02D0464BBF
:10B948003B6101E0384B3B6197F8503003F040030E
:10B95800DBB2002B02D0414BFB6001E0324BFB60B5
:10B9680097F8503023F07F03DBB2002B02D03C4B1A
:10B97800BB6001E02C4BBB6097F84C3003F001032F
:10B98800DBB2002B02D0374B7B6001E0264B7B609B
:10B9980097F84C3003F00203DBB2002B02D0324B95
:10B9A8003B6001E0204B3B6097F84C3003F0040308
:10B9B800DBB2002B01D02D4E00E01B4E97F84C3027
:10B9C80003F00803DBB2002B01D0294D00E0164D2F
:10B9D80097F84C3003F01003DBB2002B01D0254C54
:10B9E80000E0114C97F84C3003F02003DBB2002B39
:10B9F80001D0214900E00C4997F84C3003F040038E
:10BA0800DBB2002B01D01D4A00E0074A97F84C3002
:10BA180023F07F03DBB2002B34D0194B33E000BF97
:10BA28007C09002020940108289D0108249401081D
:10BA38002C9401083894010840940108489401089E
:10BA4800509401085894010860940108689401080A
:10BA580070940108789401087C9401088494010882
:10BA68008C94010898940108A0940108AC940108EA
:10BA7800B8940108C4940108CC940108D094010832
:10BA8800D4940108174B97F8470014931392129116
:10BA9800119410950F963B680E937B680D93BB68C5
:10BAA8000C93FB680B933B690A937B690993BB6909
:10BAB8000893FB6907933B6A06937B6A0593BB6A05
:10BAC8000493FB6A03933B6B02937B6B0193BB6B01
:10BAD8000093FB6B3A6C0449FEF70AFE00BF5C3723
:10BAE800BD46F0BD289D0108E0940108F0B589B075
:10BAF80006AF04F0AFFC7860854B5B78082B0CBF71
:10BB080001230023DBB2FB70814BB3F81B309BB2DF
:10BB1800002B05D07E4BB3F80F309BB2002B01D120
:10BB2800012300E00023BB70FB78002B15D0784B75
:10BB3800DB7D002B11D0774B1B7A002B0DD0754B7A
:10BB4800DB79052B07D0734BDB79032B03D0714BC3
:10BB5800DB79042B01D1012300E000237B70FB7803
:10BB6800002B0CD06A4BDB7D002B08D0694BDB79AE
:10BB7800052B04D1BB78002B01D1012300E0002361
:10BB88003B70654B1B78002B13D1624B1A7F634BBC
:10BB98001A70604B5A7F624B1A705E4B9A7F614BEA
:10BBA8001A705C4B9A7A604B1A705B4B01221A70C0
:10BBB80029E17B78002B2FD0564B1A7F574B1B78E7
:10BBC8009A420BD1534B5A7F554B1B789A4205D159
:10BBD800504B9A7F534B1B789A421DD04F4B1B7882
:10BBE8001C464C4B1B7F1D464D4B1B781A46494B38
:10BBF8005B7F19464B4B1B781846464B9B7F03933C
:10BC08000290019100922B46224648490520FEF7F2
:10BC18006FFD0520FFF7EAFD3E4B1A7F3F4B1A7078
:10BC28003C4B5A7F3E4B1A703A4B9A7F3D4B1A70E9
:10BC38003B78002B2DD13E4B00221A60344BDB7D24
:10BC4800002B1ED0BB78002B1BD1314B5B78082B07
:10BC580017D1304BDB79022B13D02E4BDB79002B1D
:10BC68000FD02C4BDB790E2B0BD02A4BDB790C2B0E
:10BC780007D0284BDB790D2B03D0264BDB790B2B18
:10BC880002D12C4B00221A70224B9A7A264B1A703A
:10BC9800B9E0204B9B7A002B09D0254B00221A6073
:10BCA800244B00221A70204B01221A70ABE0214B62
:10BCB8001B78002B03D01C4B00221A70A3E01A4BF0
:10BCC8001B78002B03D11A4B00221A609BE0114B02
:10BCD8001B7A002B52D10F4B5B881E460D4BB3F9D4
:10BCE80004309C460B4BDB7A1946134B1B781846DD
:10BCF800124B1B781C46124B1B781D46114B1B68B8
:10BD0800002B21D00F4B1B687A68D31A1EE000BFA6
:10BD1800800300207C090020AC090020AD09002028
:10BD2800AE090020AF090020B00900201C950108C9
:10BD3800B4090020B8090020A4090020A5090020A2
:10BD4800A60900209C09002042F20F730493039572
:10BD5800029401900091634632462C490420FEF774
:10BD6800C7FC0420FFF742FD294B01221A70294B1A
:10BD780000221A60284B00221A7044E0254B1B68E9
:10BD8800002B03D1234A7B6813603CE0214B1B68DE
:10BD98007A68D31AC72B35D9204B5B881E461F4BB0
:10BDA800B3F904309C461D4BDB7A19461B4B1B7FAD
:10BDB80018461A4B5B7F1C46184B9B7F1D46184B39
:10BDC8001B68002B04D0164B1B687A68D31A01E055
:10BDD80042F20F7304930395029401900091634615
:10BDE800324610490420FEF783FC0420FFF7FEFCCE
:10BDF800074B01221A70074B00221A60064B0022DB
:10BE08001A7000E000BF0C37BD46F0BD6895010808
:10BE1800B8090020B4090020B00900207C090020DE
:10BE28009C090020DC95010880B582B002AF8E4BDA
:10BE3800DB7D002B23D18C4B93F82330002B04D1CE
:10BE4800894B93F82830002B03D088490720FEF748
:10BE58004FFC854B002283F82320834B002283F874
:10BE68002420002283F82520002283F8262000229F
:10BE780083F827207C4B002283F82820F2E07C4BB3
:10BE88001B7A002B23D1784B93F82330002B04D155
:10BE9800754B93F82830002B03D076490720FEF71E
:10BEA80027FC714B002283F823206F4B002283F874
:10BEB8002420002283F82520002283F8262000224F
:10BEC80083F82720684B002283F82820CAE0664BB5
:10BED80093F82330002B6ED1634B93F82830022B54
:10BEE8005BD8614BB3F813309BB2B3F5F07F54D2F3
:10BEF8005D4BB3F815309BB2B3F5967F4DD95A4BCD
:10BF08005B6A002B05D104F0A5FA0346564A536232
:10BF1800A5E004F09FFA0246534B5B6AD31AB3F5C7
:10BF28007A7FC0F09C80504B012283F823204E4B2F
:10BF380093F828300133DAB24B4B83F828204A4B68
:10BF4800002283F82420002283F82520002283F889
:10BF58002620002283F82720434BB3F813309BB2E6
:10BF68001A46414BB3F815309BB219463E4B93F82D
:10BF7800283000930B4640490520FEF7B9FB3A4BA1
:10BF880093F82830022B6AD9374B93F828301A4691
:10BF98003A490520FEF7ACFB61E0334B002283F8F9
:10BFA8002420002283F82520002283F8262000225E
:10BFB80083F8272056E02C4BB3F813309BB2B3F527
:10BFC800F87F06D2284BB3F815309BB2B3F5967FAD
:10BFD80037D8254B5B6A002B05D104F03BFA0346A2
:10BFE800214A53623DE004F035FA02461E4B5B6A73
:10BFF800D31AB3F57A7F34D31B4B002283F823205E
:10C00800194B002283F82420002283F825200022DF
:10C0180083F82620002283F82720134BB3F8133027
:10C028009BB21A46104BB3F815309BB219460E4B0B
:10C0380093F8283000930B4611490720FEF758FB68
:10C048000FE0094B002283F82420002283F82520E2
:10C05800002283F82620002283F8272002E000BF70
:10C0680000E000BFBD4680BD800300205496010853
:10C078007C0900207096010888960108A896010896
:10C08800C0960108F0B589B006AF0346FB711A4B9C
:10C09800DB79FA799A4222D0174BDB791846FFF7F9
:10C0A8001FFA0446FB791846FFF71AFA0346134AA3
:10C0B800D27D1146104A527A10460F4A927A154696
:10C0C8000D4AD27A16460D4A527F0492039602957B
:10C0D8000190009122460A490720FEF709FB064A0B
:10C0E800FB79D37104F0B6F90346034A136100BF24
:10C0F8000C37BD46F0BD00BF7C090020800300203E
:10C10800E096010880B500AF04F0A4F90246024B9E
:10C118001B69D31A184680BD7C09002080B582B0FF
:10C1280000AF3B1D1846FFF7F7F8BB88FA88194699
:10C13800002000F04DF90121002000F019F900BF9E
:10C148000837BD4680BD00BF80B500AFFFF724F9B2
:10C15800054B9B7A002B01D1FFF7E0FF0520FFF785
:10C1680091FF00BF80BD00BF7C09002038B5444C5A
:10C17800444D23462A46012105F046FA10B96D6858
:10C18800EBB203B138BD04F065F9C5F305453E4B84
:10C19800022D186016D0042D1AD194E803003B4BE9
:10C1A8003B4A83E803001C7AD87999791B79394D81
:10C1B80093611477384B50779177384A2C70107008
:10C1C800197038BD364B94E8030083E8030038BD86
:10C1D800062D11D194E80300324B83E80300188838
:10C1E80059889A8840BA49BA52BA80B289B292B28A
:10C1F800C3E902011A6138BD082D3AD0092DC1D111
:10C2080094E80300214B284D214C93F804C0274A99
:10C2180085E8030000BA84F806C0A2FB00C209BA88
:10C22800C5E90201C2F38F1013284FF0010E94BF25
:10C23800002501251E4B84F808E0A3FB01C3E17922
:10C248005B0971456080A3804FEA9212A57299D963
:10C2580099B292B201FB02F2164C1749A4FB0242B2
:10C26800A1F815300D76D308A1F81300C1F80330F2
:10C2780038BD124B94E8030083E8030038BD00BFC3
:10C28800D8090020BC0900209C090020440900208E
:10C298007C090020A4090020A6090020A509002087
:10C2A80038090020500900206C090020D34D621085
:10C2B8001F85EB51CDCCCCCC800300206409002035
:10C2C80080B58AB000AF0E237B610023BB610123D8
:10C2D800FB6100233B6000237B600023BB600023DD
:10C2E800FB6000233B6101233B6201233B610E237A
:10C2F8007B623B461946064804F016FF0346002BAE
:10C3080001D0FEF7CDFD00BF2837BD4680BD00BF78
:10C318005403002080B500AF134805F029F8FDF755
:10C32800C9FCFFF7CDFF104804F0DEFF10210E48CE
:10C3380005F08BFA202200210C480AF089FD0B4BEE
:10C348000022DA7104F086F80346084A1361074BA5
:10C3580049F640425A610021002000F009F8FEF732
:10C3680053FE00BF80BD00BF540300207C0900209D
:10C3780080B584B000AF03460A46FB711346BB7113
:10C3880007F108030822002118460AF061FDFB792D
:10C39800002B15D10D4B1B7A002B13D0BB79002B2A
:10C3A8000CBF01230023DBB23B7207F10803F979C4
:10C3B8001A22F02000F072F81420FEF7B5FB02E014
:10C3C80000BF00E000BF1037BD4680BD7C090020DB
:10C3D80080B586B000AF0346FB710B46BB801346A1
:10C3E8007B8007F108030822002118460AF030FD77
:10C3F800FB79002B47D1BB88952B01D89623BB80AE
:10C40800234B93F82330002B06D0BB88B3F5FA7F73
:10C4180002D340F2F313BB807B88642202FB03F350
:10C428007B61BB884FF47A7202FB03F33B617B6943
:10C438001B0EDBB23B737B691B0CDBB27B737B6926
:10C448001B0ADBB2BB737B69DBB2FB733B691B0E58
:10C45800DBB23B723B691B0CDBB27B723B691B0A8C
:10C46800DBB2BB723B69DBB2FB720A4ABB88138042
:10C47800094A7B88138007F10803F9791C22F02008
:10C4880000F00CF800E000BF1837BD4680BD00BFC3
:10C4980080030020A0090020A209002080B58CB0EC
:10C4A80000AF3B600346FB710B46BB7113467B71C3
:10C4B800FB7987F82830BB7987F829307B7903F036
:10C4C8003F03DAB297F82A3062F3050387F82A3077
:10C4D8007B8D0A2262F389137B850A2387F82F3024
:10C4E800BB6A7B610023FB610423BB6108233B62B9
:10C4F8001EE0144805F054F80346002B0ED007F14F
:10C508000C0307F110013A680E4804F07AFF03465D
:10C5180087F82E3097F82E30002B0ED00120FEF72A
:10C5280003FB97F92F30DBB2013BDBB287F82F30E2
:10C5380097F92F30002BDCDC00E000BF3037BD4618
:10C5480080BD00BF5403002080B584B000AF3B1D00
:10C5580000221A605A603B1D04220021F020FFF7D8
:10C568009DFF1420FEF7E0FA3B1D06220021F02073
:10C57800FFF794FF1420FEF7D7FA3B1D092200218C
:10C58800F020FFF78BFF1420FEF7CEFA404BB3F8EC
:10C598001B309BB23F4AA2FB0323DB089BB21A461F
:10C5A8003B4BB3F813309BB202FB03F31A463A4BEA
:10C5B8005B699A4211D9384B5A6913469B00134458
:10C5C8005B001A46324BB3F813309BB2B2FBF3F35D
:10C5D8009AB22F4BA3F8112006E02D4BB3F81B306D
:10C5E8009AB22B4BA3F81120294BB3F811309BB208
:10C5F80040F23252934208D9254B002242F03202CF
:10C608005A74002242F005029A74214BB3F8113093
:10C618009BB21A461E4BB3F80F309BB202FB03F3D2
:10C628001E4A82FB03129210DB17D31A1A46184BC4
:10C63800C3F80B20FEF79EFD0346002B04D1FEF73E
:10C64800A3FD0346002B01D0012300E00023FB7368
:10C65800114B5B7A002B11D0FB7B002B0ED10C4BBE
:10C66800B3F80F309BB20A4AB2F8112092B21946B9
:10C678000020FFF7ADFE1420FEF756FA064B5B7A52
:10C68800002B01D0FFF7D0FB00BF1037BD4680BD9F
:10C6980080030020CDCCCCCC7C0900206766666680
:10C6A800B0B586B002AFFEF707FDFEF763FD03469F
:10C6B800002B09D0FEF7C8FD0346FB73FB7B022B5A
:10C6C80002D10620FFF7DEFC03F0C4FE0246AD4BA4
:10C6D8001B68D31AB3F5FA7F2FD9AB4B1B7A002B03
:10C6E8000AD003F0B7FE0246A64B1B68D31A1A46B7
:10C6F800A6490520FDF7FCFFA34B00221A72A24BA6
:10C7080000229A72A24B00221A71A14B00221A72BF
:10C718009F4B0022DA719E4B00229A719D4B00229A
:10C728009A609C4B0022DA609A4B00221A619A4B5D
:10C738000022DA60984B00229A60934B1B7A002BF8
:10C7480003D0914B1B78002B0CD1944B0022DA7448
:10C7580000221A75914B00225A7500229A758F4B48
:10C7680000221A768D4B9B7F002B0CD001210420D0
:10C77800FDF774F803F06EFE0346894A1360824B96
:10C7880001221A7010E003F065FE0246844B1B6814
:10C79800D31A4EF66022934206D900210420FDF7F1
:10C7A8005DF8794B00221A700520FDF7D7F803468B
:10C7B8001A46754BDA72744B1B7A002B07D0724BF2
:10C7C8001B7B002B03D1704B1B78002B02D16E4BC7
:10C7D80000225A72FFF78AF96B4BDB790E2B00F2B5
:10C7E800C08201A252F823F02DC8000861C80008D1
:10C7F8007DC80008D9C800081DC9000875C9000807
:10C808000BCA00084FCA0008D9CA000829CB00087B
:10C8180077CB000831CC00081DCD0008A1CC00085A
:10C8280057CD0008584B00225A7000210320FDF70D
:10C8380015F8554B1B7A002B00F09782524B1B784A
:10C84800002B00F09282504B1B7B002B40F08D8216
:10C858000120FFF717FC88E2FFF754FC0346B3F505
:10C868007A6F40F28482484B01225A720220FFF705
:10C8780009FC7CE2494B002283F82320474B002225
:10C8880083F82420002283F82520002283F826201C
:10C89800002283F82720414B002283F8282000211A
:10C8A8000320FCF7DBFF384B5B7A002B03D1002019
:10C8B800FFF7E8FB70E2394BDB7D002B00F0598273
:10C8C80001210020FFF754FD0320FFF7DBFB50E2B6
:10C8D8002D4B9B7A002B07D02B4B5B7A002B03D078
:10C8E8000420FFF7CFFB46E2FFF70CFC034642F2B9
:10C8F8001072934240F23F82234B01225A73274B16
:10C908000A225A770020FFF7BDFB26490420FDF7CD
:10C91800EFFE30E201210320FCF7A0FF1A4BDB7A7F
:10C92800002B0ED0184BDB7A1C46FFF7EBFB0346B7
:10C9380022461D490720FDF7DBFE0520FFF7A2FB75
:10C948001BE2FFF7DFFB0346B3F57A7F40F215825F
:10C958000D4B01221A73114B07225A770B20FFF750
:10C9680091FB12490420FDF7C3FE06E20B4BDB7D69
:10C97800002B03D0044B5B7A002B19D10B20FFF757
:10C9880081FB09E29C0900207C090020149701081A
:10C9980044090020500900206C0900208003002071
:10C9A800E00900203C9701084C9701088897010886
:10C9B8000520FCF7D3FF03461C460320FCF7BEFF07
:10C9C80003469C4217D003F045FD0246A84B1B685E
:10C9D800D31AB3F57A7F40F2D281A64B07225A7751
:10C9E800A54B01221A730B20FFF74CFBA349042027
:10C9F800FDF77EFEC3E103F02DFD03469C4A13605C
:10CA0800BDE19C4BDB7D002B0BD09B4B5B7A002B55
:10CA180007D0994B1B7B002B03D1974B5B7B002BDB
:10CA280009D097490520FDF763FEFEF7B5FC0B20FA
:10CA3800FFF728FBB0E100210020FFF799FC072051
:10CA4800FFF720FBA8E18B4BDB7D002B0BD08A4B3B
:10CA58005B7A002B07D0884B1B7B002B03D1864BBE
:10CA68005B7B002B09D086490520FDF741FEFEF7C8
:10CA780093FC0B20FFF706FB8EE17F4B9B7A002B84
:10CA880012D107F108031846FEF746FC794BB3F8B4
:10CA980013309BB21A463B897A490720FDF728FED6
:10CAA8000820FFF7EFFA6CE1FFF72CFB034642F290
:10CAB8001072934240F265816E4BB3F813309BB20B
:10CAC8001A4671490520FDF713FEFFF73DFB58E1B3
:10CAD800684BDB7D002B0BD0674B5B7A002B07D0B4
:10CAE800654B1B7B002B03D1634B5B7B002B09D071
:10CAF80063490520FDF7FCFDFEF74EFC0B20FFF710
:10CB0800C1FA49E13B1D1846FEF706FCBB88FA88C6
:10CB180019460020FFF75CFC0920FFF7B3FA3BE158
:10CB2800544BDB7D002B0BD0534B5B7A002B07D08B
:10CB3800514B1B7B002B03D14F4B5B7B002B09D048
:10CB48004F490520FDF7D4FDFEF726FC0B20FFF723
:10CB580099FA21E101210020FFF70AFC03F07AFC91
:10CB680003464A4A13600A20FFF78CFA14E1414B46
:10CB7800DB7D002B0BD0404B5B7A002B07D03E4B64
:10CB88001B7B002B03D13C4B5B7B002B09D03C4922
:10CB98000520FDF7ADFDFEF7FFFB0B20FFF772FA4E
:10CBA800FAE03B461846FEF7B7FB3B88282B03D92B
:10CBB8003B88283B9BB200E00023BB812E4B9B7A2D
:10CBC800002B0CD02B4BB3F813309BB2BA899A4286
:10CBD80005D8FEF7B3FB0520FFF754FAD3E003F0BE
:10CBE80039FC0246294B1B68D31AB3F5FA7F06D3E2
:10CBF800FFF794FA03F02EFC0346244A1360FFF76C
:10CC080081FA034642F21072934240F2BC80194BFB
:10CC1800B3F813309BB21A463B881D490520FDF72F
:10CC280067FDFFF791FAAEE0124B00225A7400221A
:10CC38009A74104BB3F815309BB21D2B07D9FFF728
:10CC480061FA034641F28832934240F29E80094BD2
:10CC5800B3F815309BB21C46FFF754FA0346224638
:10CC68000C490720FDF744FD0D20FFF70BFA8CE077
:10CC7800E4090020800300207C090020889701082F
:10CC8800A8970108C8970108F0970108E80900204B
:10CC9800149801084498010800210320FCF7DEFDE0
:10CCA800404BDB7A002B0FD1FFF72CFA03461A46CC
:10CCB8003D490720FDF71CFD00210020FFF758FB28
:10CCC8000C20FFF7DFF962E0FFF71CFA0346B3F523
:10CCD8007A7F5CD9334B01221A73344B07225A7777
:10CCE80000210020FFF744FB0C20FFF7CBF90320BD
:10CCF800FCF724FE03461C462A4BDB7A1D46FFF749
:10CD080001FA034600932B46224629490420FDF7E1
:10CD1800EFFC3CE0234B9B7A002B03D10E20FFF75E
:10CD2800B1F936E0FFF7EEF9034642F2107293428A
:10CD38002FD91C4B01225A731C4B0A225A77002008
:10CD4800FFF7A0F91B490420FDF7D2FC21E0FFF70B
:10CD5800D9F90346B3F57A6F1DD90220FFF792F986
:10CD680019E00020FFF78EF916E000BF14E000BFBD
:10CD780012E000BF10E000BF0EE000BF0CE000BFF3
:10CD88000AE000BF08E000BF06E000BF04E000BF03
:10CD980002E000BF00E000BFFEF710FC00BF103744
:10CDA800BD46B0BD7C09002084980108800300209E
:10CDB800AC980108E498010880B485B000AF3B60E6
:10CDC8000346FB710B46BB7113467B71BB79002B85
:10CDD8000BD13B687A799A703B689A783B685A70AD
:10CDE8003B685A783B681A7086E0FB79444AA2FB94
:10CDF8000323DB08FB73FB7B1A4652001A441146D7
:10CE0800C9008A1A52001344DBB2FA79D31ADBB28A
:10CE18001A46520013445B00BB737B79BA79C2F19E
:10CE2800FF0202FB03F31B0A7B737B79BA79B97B98
:10CE380001FB02F21212C2F1FF0202FB03F31B0A0A
:10CE48003B737B79BA79B97BC1F1FF0101FB02F22F
:10CE5800120AC2F1FF0202FB03F31B0AFB72FB7BFF
:10CE6800042B3FD801A252F823F000BF89CE000856
:10CE78009DCE0008B1CE0008C5CE0008D9CE000866
:10CE88003B687A791A703B68FA7A5A703B687A7B01
:10CE98009A7031E03B683A7B1A703B687A795A702D
:10CEA8003B687A7B9A7027E03B687A7B1A703B680C
:10CEB8007A795A703B68FA7A9A701DE03B687A7BF7
:10CEC8001A703B683A7B5A703B687A799A7013E01B
:10CED8003B68FA7A1A703B687A7B5A703B687A79B1
:10CEE8009A7009E03B687A791A703B687A7B5A70C5
:10CEF8003B683A7B9A7000BF1437BD4680BC7047C8
:10CF080083BEA02F80B582B000AF5523FB71F523F7
:10CF1800BB711B4B1B78F92B02D91A4B00221A70D4
:10CF2800174B1B781E2B02D8164B01221A70154B73
:10CF38001B78002B0CD0124B1B78F62B04D8104B07
:10CF48001B780433DBB200E0FA230D4A13700BE0C0
:10CF58000B4B1B78212B04D9094B1B78043BDBB204
:10CF680000E01E23064A1370054B1978BA79F87940
:10CF7800054BFFF721FF00BF0837BD4680BD00BF46
:10CF880033000020310A0020F409002080B487B063
:10CF980000AF786039603B689B795E2B8CBF0123BA
:10CFA8000023DBB2FB7507F10C0300221A605A60FC
:10CFB8001A813B681B781A463B68DB7802FB03F34F
:10CFC8004A4A82FB03125211DB17D31ADBB23B73B6
:10CFD8003B685B781A463B68DB7802FB03F3434AFD
:10CFE80082FB03125211DB17D31ADBB27B733B6847
:10CFF8009B781A463B68DB7802FB03F33B4A82FBCB
:10D0080003125211DB17D31ADBB2BB733B685B798F
:10D01800C3F16403042B05DD3B685B79C3F164034A
:10D02800DBB200E00523FB730A233B743B685B79A2
:10D03800C3F16403042B05DD3B685B79C3F164032A
:10D04800DBB200E005237B74FB7D002B01D00A23B3
:10D0580000E00023BB743B681B79002B08D107F163
:10D06800130307F10C021188927819809A702FE047
:10D078003B7B1A463B689B79C3F1640302FB03F3CD
:10D088001A4A82FB03125211DB17D31ADBB2FB7464
:10D098007B7B1A463B689B79C3F1640302FB03F36D
:10D0A800124A82FB03125211DB17D31ADBB23B750B
:10D0B800BB7B1A463B689B79C3F1640302FB03F30D
:10D0C8000A4A82FB03125211DB17D31ADBB27B75B3
:10D0D8007B681A4607F10C0303CB106051601B886C
:10D0E800138178681C37BD4680BC70471F85EB519B
:10D0F80080B485B000AF78607B68002B21D07B6856
:10D108001B78012B1DD87B685B7803F0FE03002B8E
:10D1180017D17B68DB78002B13D17B685B7803F031
:10D128000103002B03D07B689B78002B09D07B6818
:10D138005B7803F00103002B05D17B689B78002BFB
:10D1480001D0002323E00023FB731CE0FA7B134685
:10D15800DB009B1A7A6813440433BB60BB68DB7836
:10D16800642B0BD8BB681B79012B07D8BB685B798C
:10D17800642B03D8BB689B79642B01D9002306E094
:10D18800FB7B0133FB73FB7B042BDFD901231846A0
:10D198001437BD4680BC7047F0B583B000AF7860E7
:10D1A8007868FFF7A5FF0346002B01D100234CE068
:10D1B8007B685B7803F00103002B29D0254A7B6844
:10D1C8001C46164604F1200C354623461868596853
:10D1D8009A68DB680FC5103410366445F4D13346BD
:10D1E8002246106818609188927999809A711A4B32
:10D1F80001221A7003F02EF902467B689B781946C3
:10D208004FF47A7301FB03F31344144A13601BE0D1
:10D21800134A7B681C46164604F1200C3546234603
:10D22800186859689A68DB680FC510341036644569
:10D23800F4D1334622461068186091889279998013
:10D248009A71054B00221A70012318460C37BD4607
:10D25800F0BD00BF040A0020300A00202C0A00207C
:10D268000C00002080B58CB000AF694BFB62694BA5
:10D2780000221A70684B1B78012B03D1674800F015
:10D2880077FBC1E0644B5B7F002B03D1624B5B787B
:10D29800022B15D1FB6A03F120023B4611461846C2
:10D2A800FFF774FE07F120033A461068516803C37C
:10D2B80012891A8007F12003184600F059FBA3E0F1
:10D2C800574B1B78002B0AD003F0C4F80246554B85
:10D2D8001B68D31A002B02DB514B00221A70504BEB
:10D2E8001B78002B01D0504BFB62FB6A1B78012B8B
:10D2F8000BD107F1140300221A605A601A8107F152
:10D308001403184600F034FB7EE0434B1B78032BD4
:10D3180003D1464800F02CFB76E03F4B5B78002BAE
:10D3280003D13C4B01221A706EE03B4B5B78013B0A
:10D338000C2B60D801A252F823F000BF79D3000863
:10D34800FFD3000899D3000899D30008BBD300087D
:10D35800BBD30008BBD30008BBD30008DDD300084B
:10D36800DDD30008DDD30008DDD3000899D3000819
:10D37800FB6A1A1D3B4611461846FFF707FE07F1E0
:10D3880020033A461068516803C312891A8036E0B0
:10D39800FB6A03F10B023B4611461846FFF7F6FD00
:10D3A80007F120033A461068516803C312891A80AE
:10D3B80025E0FB6A03F112023B4611461846FFF7C7
:10D3C800E5FD07F120033A461068516803C3128946
:10D3D8001A8014E0FB6A03F119023B46114618460D
:10D3E800FFF7D4FD07F120033A461068516803C3DC
:10D3F80012891A8003E0074B01221A7004E007F132
:10D408002003184600F0B4FA3037BD4680BD00BF8F
:10D418000C000020020A002080030020E0A0010880
:10D42800300A00202C0A0020040A0020ECA0010881
:10D4380080B487B000AFF860B96011461A460B4651
:10D44800FB801346BB80FA88BB889A4201D9BB8807
:10D45800FB80BB88002B01D10123BB80FA881346CF
:10D468001B029A1ABB8892FBF3F3FB82FB681B78BA
:10D478001A46FB8AC3F1FF0303FB02F2BB681B7861
:10D488001946FB8A01FB03F31344204A82FB03126B
:10D498001A44D211DB17D31ADAB23B6A1A70FB6846
:10D4A8005B781A46FB8AC3F1FF0303FB02F2BB68F1
:10D4B8005B781946FB8A01FB03F31344134A82FB8A
:10D4C80003121A44D211DB17D31ADAB23B6A5A7024
:10D4D800FB689B781A46FB8AC3F1FF0303FB02F241
:10D4E800BB689B781946FB8A01FB03F31344074A80
:10D4F80082FB03121A44D211DB17D31ADAB23B6A41
:10D508009A7000BF1C37BD4680BC70478180808000
:10D5180042EA002242EA014230B44FF0180C4FF4BC
:10D528000075D343564C52E000BF00BF00BF00BF98
:10D5380000BF00BF00BF00BF00BF00BF00BF00BFEB
:10D5480000BF00BF00BF00BF00BF00BF00BF00BFDB
:10D5580000BF00BF00BF00BF00BF656100BF00BFC4
:10D5680000BF00BF00BF00BF00BF00BF00BF00BFBB
:10D5780000BF00BF00BF00BF00BF00BF00BF00BFAB
:10D5880000BF00BF00BF00BF00BF00BF00BF00BF9B
:10D5980000BF00BF00BF00BF00BF00BF00BF00BF8B
:10D5A80000BF00BF00BF00BF00BF00BF00BF00BF7B
:10D5B80000BF00BF00BF00BF00BF00BF00BF00BF6B
:10D5C80000BF00BFBCF1010C4FEA430355D01A025B
:10D5D8002561A9D400BF00BF00BF00BF00BF00BFC6
:10D5E80000BF00BF00BF00BF00BF00BF00BF00BF3B
:10D5F80000BF00BF00BF00BF00BF00BF00BF00BF2B
:10D6080000BF00BF00BF00BF00BF00BF00BF00BF1A
:10D6180000BF00BF00BF00BF00BF00BF00BF00BF0A
:10D6280000BF00BF00BF00BF00BF00BF00BF00BFFA
:10D6380000BF00BF00BF00BF00BF00BF656100BFE3
:10D6480000BF00BF00BF00BF00BF00BF00BF00BFDA
:10D6580000BF00BF00BF00BF00BF00BF00BF00BFCA
:10D6680000BF00BF00BF00BF00BF00BF00BF00BFBA
:10D67800BCF1010C4FEA4303A9D130BC704700BF8D
:10D688000010014038B50C46EFF3108572B6827869
:10D6980041780078FFF73CFFA27861782078FFF79F
:10D6A80037FF85F3108838BD80B485B000AF786047
:10D6B8007B681B781A4613461B019B1A9B00214A5C
:10D6C80082FB03121A44D211DB17D31ADBB23B7266
:10D6D8007B685B781A4613461B019B1A9B00194A04
:10D6E80082FB03121A44D211DB17D31ADBB27B7206
:10D6F8007B689B781A4613461B019B1A9B00114AAC
:10D7080082FB03121A44D211DB17D31ADBB2BB72A5
:10D7180007F10C0307F10802126811461980023359
:10D72800120C1A7000233A7B62F307037A7B62F3C8
:10D738000F23BA7B62F3174318461437BD4680BCE3
:10D74800704700BF8180808080B582B000AF4C4BAD
:10D758005B7FBB7102F07EFE3860BB79002B18D16D
:10D76800484B00221A70484B00221A70474B00227F
:10D778001A70474B00221A60464B00221A70464B1B
:10D7880000221A70444B00225A70434B00229A70B0
:10D7980072E0404B1B78BA799A420ED0394B00227E
:10D7A8001A70394B00221A70384B00221A70384B05
:10D7B80000221A60374ABB791370354B1B683A68E8
:10D7C8009A4209D2344BFF221A70334B00225A7006
:10D7D800314B00229A704FE02F4B00221A702E4BCB
:10D7E80000225A702C4B00229A702C4B1B683A6806
:10D7F800D31A632B3FD9294A3B6813600023FB7176
:10D80800224B1B78002B06D0204B1B78013BDAB249
:10D818001E4B1A701EE01B4B1B78BA799A4213D91B
:10D82800194B1B78002B03D1174B01221A7011E0FA
:10D838000123FB71144B00221A70124B1B78013321
:10D84800DAB2104B1A7005E00E4B00221A700F4B1B
:10D858001E221A70FB79002B0ED03B6864330C4AE9
:10D8680013600D4BFF221A700B4B00225A700A4BA3
:10D8780000229A7000E000BF0837BD4680BD00BF97
:10D8880080030020320A0020330A0020340A0020D6
:10D89800380A00203C0A0020EC090020400A002039
:10D8A80080B483B000AF78607B681B781A46642325
:10D8B80002FB03F3174A82FB03121A44D211DB1747
:10D8C800D21A154B1B689A637B685B781A466423E7
:10D8D80002FB03F30F4A82FB03121A44D211DB172F
:10D8E800D21A0D4B1B68DA637B689B781A4664234F
:10D8F80002FB03F3074A82FB03121A44D211DB1717
:10D90800D21A054B1B681A6400BF0C37BD4680BC91
:10D91800704700BF81808080E412002080B584B009
:10D9280000AF78607868FFF7BFFE03461A463A737F
:10D93800C3F307227A73C3F30743BB730B48FFF79C
:10D94800B3FE03461A463A72C3F307227A72C3F348
:10D958000743BB7207F1080207F10C03114618468A
:10D96800FFF790FE00BF1037BD4680BDEC090020D0
:10D9780080B483B000AF7860054B7A68106851684E
:10D9880003C312891A8000BF0C37BD4680BC70479C
:10D99800F809002080B582B000AF00233B71002356
:10D9A8007B710023BB7104210B4806F021FC082180
:10D9B800094806F01DFC0C21074806F019FC3B1D20
:10D9C8001846FFF76DFF3B1D1846FFF7A7FF00BF7E
:10D9D8000837BD4680BD00BFE412002080B582B084
:10D9E80002AF02F037FD02464F4B1B68D31A142BC7
:10D9F80040F2988002F02EFD03464B4A1360FFF771
:10DA0800A3FE4A4B1B78002B08D0FFF77BFA484847
:10DA1800FFF746FF4648FFF781FF83E0454B5B88E9
:10DA280001339AB2434B5A80424B1B78032B68D878
:10DA380001A252F823F000BF51DA000883DA000887
:10DA4800AFDA0008E1DA00083A4B5A883A4BDB783B
:10DA58001946374B00930B4637493848FFF7E8FC1F
:10DA6800344B5B88344AD27893424ED9314B0122E9
:10DA78001A70304B00225A8047E02E4B2E4A04334E
:10DA88001268114619800233120C1A70294B5B88F0
:10DA9800294A127993423AD9264B02221A70254B09
:10DAA80000225A8033E0234B5A88234B5B7919466E
:10DAB8001F4B00930B4621491F48FFF7B9FC1D4B2C
:10DAC8005B881D4A5279934223D91A4B03221A7054
:10DAD800184B00225A801CE0164B174A04330732B1
:10DAE8001188927819809A70124B5B88124A927941
:10DAF800934210D90F4B00221A700E4B00225A8005
:10DB080009E00C4B00221A7006E000BF04E000BFD9
:10DB180002E000BF00E000BF0548FFF7C1FE04486F
:10DB2800FFF7FCFEBD4680BD440A0020020A002023
:10DB3800F4090020F0090020F8090020FF0900205E
:10DB480080B500AF0A4B0B4A1A60094B4FF0FF3201
:10DB58005A60074B4FF480729A60054806F096F8B1
:10DB68000346002B01D0FDF79BF900BF80BD00BF25
:10DB7800480A00200028004080B584B000AF7860D3
:10DB88007B681B680B4A934210D105F013F80A4BC7
:10DB9800DB69094A43F00063D361074BDB6903F093
:10DBA8000063FB60FB68054B01221A6000BF103759
:10DBB800BD4680BD00280040001002403C0442429F
:10DBC800024659B370B50C46CB0758BF1549154DD9
:10DBD80048BF144986B054BF0B46134B14F0020FCC
:10DBE8000491124908BF294614F0040F104808BFD1
:10DBF800284614F0080F01900E480F4E08BF2E4615
:10DC080014F0100F18BF05460091CDE902650B49C5
:10DC180005940420FCF76CFD06B070BD042008498B
:10DC2800FCF766BD289D0108F8980108FC980108D2
:10DC3800009901080C990108049901083499010810
:10DC48001499010830B54FF48072054683B0114924
:10DC5800114807F0C8FA08B903B030BD04460E48A9
:10DC680007F0D3FE0246234614460C492A460420F0
:10DC78000094FCF73DFD03202146FFF7A1FF08486B
:10DC880000F002FF002CE7D0034803B0BDE83040A5
:10DC980007F06ABB800A0020041400206899010874
:10DCA800A499010838B51A4B0C46834213D129B3FD
:10DCB800B1F5807F16D802F0CDFB0346154D164A04
:10DCC800214616482B60136000F036FEBDE8384048
:10DCD8001348FFF7B7BF0A46BDE838400520114989
:10DCE800FCF706BD4FF480730A4604200E49FCF782
:10DCF800FFFCBDE838400A48FFF7A4BF05200B49E0
:10DD0800FCF7F6FCBDE838400548FFF79BBF00BFAD
:10DD180004140020900D0020940D0020800A00209B
:10DD2800309A0108C0990108409A0108FC99010835
:10DD3800F8B5044607F069FE294B05469C4232D0E7
:10DD4800284EB44217D0284B9C4245D003460022A7
:10DD580026490420FCF7CCFC29460020FFF730FFB9
:10DD6800204607F001FB204607F096FA2046BDE85A
:10DD7800F84001F045B9034603221C490420FCF78A
:10DD8800B7FC29460320FFF71BFF204607F0ECFAF3
:10DD9800204607F081FA0022154B16481A70BDE894
:10DDA800F840FFF74FBF022217460E4E2B460F4989
:10DDB8000420FCF79DFC29463846FFF701FF204662
:10DDC80007F0D2FA204607F067FAB442E3D02046BB
:10DDD800BDE8F84001F014B905221746E6E700BF90
:10DDE800BC130020041400202C130020809A010882
:10DDF800820D0020CC9A010880B582B000AF78600F
:10DE08007B68164A934224D1154B00221A70154B91
:10DE18001B88002B1ED0134B1B881A461249134827
:10DE280009F0A3F80E4B01221A700E4B1B881A46F4
:10DE38000E490A4807F00AF90346002B05D0084B9B
:10DE480000221A700A4800F01FFE064B00221A80B2
:10DE580000E000BF0837BD4680BD00BF04140020A5
:10DE6800820D0020800D0020800C0020800B0020F7
:10DE7800DC9A0108B0B586B004AF02F0EBFA0246AE
:10DE8800A54B1B68D31A002B40F3988202F0E2FAE4
:10DE98000346A14A136000F0BDFDA04B1B78002B80
:10DEA80003D09E4B1A789E4B1A709C4B1B78032B01
:10DEB8001BD19C4B1B68002B05D102F0CBFA034603
:10DEC800984A136014E002F0C5FA0246954B1B68A5
:10DED800D31A1A4642F20F739A4209DD8F4B002279
:10DEE8001A70904B00221A6002E08E4B00221A60D2
:10DEF8008A4B1B78012B19D18B4B1B68002B05D142
:10DF080002F0A8FA0346884A136012E002F0A2FA67
:10DF18000246854B1B68D31AB3F57A7F09DB7F4B22
:10DF280000221A70804B00221A6002E07E4B002209
:10DF38001A6002F08FFA02467C4B1B68D31A0A2B30
:10DF48005EDD02F087FA0246794B1B68D31AC72BAD
:10DF580006DD00F0D9FB02F07DFA0346744A13602F
:10DF6800744B1B78002B08D073490420FCF7C0FBC6
:10DF780000F06AFB6F4B00221A70684B1B78012B6C
:10DF880007D0664B1B78032B03D0644B5B7F002BB9
:10DF98001AD002F05FFA0246684B1B68D31AB3F531
:10DFA8007A7F11DD02F056FA0346644A1360644929
:10DFB8000520FCF79DFB594B1B78032B02D16420ED
:10DFC800FCF754F900F040FB5E4B1B780C2B03D098
:10DFD8005C4B1B780B2B13D102F03CFA0246574BD3
:10DFE8001B68D31AB3F57A7F0ADD02F033FA0346C9
:10DFF800524A136054490520FCF77AFB00F024FBD1
:10E00800524B1B68002B0CD002F024FA02464F4BEF
:10E018001B68D31A1A4641F288339A4201DD01235C
:10E0280000E00023BB71494B1B68002B0CD002F0A9
:10E0380011FA0246454B1B68D31A1A4642F210736E
:10E048009A4201DD012300E000237B717B793B715B
:10E05800BB79002B0AD03E4B1B78002B06D13D49DB
:10E068000420FCF745FB3A4B01221A707B79002B00
:10E078000AD0394B1B78002B06D138490420FCF70D
:10E0880037FB354B01221A70BB79002B05D1304B79
:10E0980000221A70304B00221A70314A7B791370B3
:10E0A800304B1B78052B00F2138101A252F823F0A4
:10E0B800D1E00008F9E0000875E10008B9E10008BE
:10E0C800F5E100084DE2000800210520FBF7C6FB3A
:10E0D8000020FBF7D3FF244B1B78002B00F0ED80CA
:10E0E8003B79002B40F0E9801E4B02221A70E4E0D5
:10E0F80000210520FBF7B2FB0220FBF7BFFF074B0F
:10E108005B7F002B40F0DB803B79002B40F0D78011
:10E11800144B02221A70D2E0E80D00208003002080
:10E128007C0A0020EC0D0020F00D0020740A00206D
:10E13800F40D0020830D0020F89A0108780A0020C9
:10E148000C9B0108E40D0020249B0108880D002089
:10E158008D0D0020409B01088E0D0020549B010866
:10E168008C0D0020E50D00209412002001210520CF
:10E17800FBF774FB0120FBF781FF924B1B78012B07
:10E1880003D0904B1B78022B02D18F4B03221A70BD
:10E198008E4B5B7F002B00F094808C4B5B7F1A4684
:10E1A8008B490420FCF7A4FA874B01221A7088E0F7
:10E1B80001210520FBF752FB0420FBF75FFF834B8F
:10E1C8001B78022B06D183490720FCF791FA7E4B76
:10E1D80004221A707B4B1B78002B74D17E490720D0
:10E1E800FCF786FA784B02221A706CE001210520B0
:10E1F800FBF734FB794B1B78022B03D9774B1B7841
:10E20800042B03D10320FBF739FF04E0734B1B7881
:10E218001846FBF733FF6B4B1B78002B06D16E4972
:10E228000720FCF765FA684B02221A706C4B1B78C2
:10E23800002B4AD06B490720FCF75AFA624B05229B
:10E248001A7042E000210520FBF708FB0D20FBF7C0
:10E2580015FF02F0FFF80246634B1B68D31AB3F5AB
:10E268007A7F1ADD02F0F6F803465F4A13605C4BCA
:10E278001B78002B0AD05A4B1B78FF2B0DD0584B1C
:10E288001B78013BDAB2564B1A7006E05749072053
:10E29800FCF72EFA4C4B02221A70514B1B78002BBC
:10E2A80015D1484B1B78012B11D151490720FCF798
:10E2B8001FFA454B03221A7009E000BF08E000BFAF
:10E2C80006E000BF04E000BF02E000BF00E000BFBE
:10E2D8007B79002B16D03D4B0022DA753F4B00228C
:10E2E8001A706420FBF7C2FF374B1B78012B06D04E
:10E2F800354B1B78002B02D0334B01221A700023B8
:10E30800FB711FE03B4B1B78012B03D12F4B0022E5
:10E31800DA7514E0384B1B78002B14BF0123002357
:10E32800DBB21A46294BDA75284BDB7D002B06D168
:10E33800264B5B78032B02D1244B0022DA75234B42
:10E34800DB7DFB712D4B1B78FF2B20D02B4B1B78D3
:10E35800FA799A421BD0294B1B781D46FA79264B2D
:10E368001B781846234B1B78012B0CBF0123002375
:10E37800DBB21C467B791549497F039102930194CE
:10E38800009013462A461E490720FCF7B1F91B4A9C
:10E39800FB7913700B4B1B78012B07D0094B1B78AB
:10E3A800022B03D0074B1B78032B03D1074B012209
:10E3B8009A7704E0054B00229A7700E000BF0837FF
:10E3C800BD46B0BD07000020E50D002080030020F9
:10E3D8007C9B0108A49B0108C89B0108E40D002050
:10E3E800840D0020D89B0108F80D0020E89B010847
:10E3F800109C01087C0A00207D0A002035000020BE
:10E408004C9C010880B500AFFBF70EFF6420FBF7BA
:10E418002DFF144B4FF47A721A80124B96225A80B1
:10E42800FBF7FEF903461A460E4B9A800D4B0A225B
:10E43800DA800C4B49F640429A6002F00BF803462A
:10E44800094A1360084B1B68084A13600848FFF71D
:10E45800F9FB00F0EFF807490720FCF749F900BF7E
:10E4680080BD00BF5C0A0020900D0020940D0020A4
:10E47800849C01088C9C010880B500AFFBF7D0F99B
:10E4880003461A46014B9A8000BF80BD5C0A0020F3
:10E49800E9B3844600B58E464FF6FF701D49E64441
:10E4A8001CF8012B424042F300030B4083EA52035D
:10E4B80043F300020A40C3F34E035A4042F30003F9
:10E4C8000B40C2F34E02534043F300020A40C3F329
:10E4D8004E035A4042F300030B40C2F34E0253402E
:10E4E80043F300020A40C3F34E035A4042F30003C9
:10E4F8000B40C2F34E02534043F300000840C3F3FD
:10E508004E035840E64580B2CAD15DF804FB4FF689
:10E51800FF70704701A0FFFF80B586B000AFB960FB
:10E528007B600346FB731346BB81BB890333FB82C5
:10E53800FA8A3B8C9A4201D9002329E07B68FA7B4E
:10E548001A70BB89002B09D0BB68002B06D07B68EA
:10E558000133BA89B968184608F007FDBB89013349
:10E568009BB219467868FFF793FF0346BB82BB89C5
:10E5780001337A681344BA8AD2B21A70BB8A1B0A6A
:10E5880099B2BB8902337A681344CAB21A70FB8AFB
:10E5980018461837BD4680BD80B586B002AF034621
:10E5A8003960FB711346BB80BA88F8794FF48073E1
:10E5B8000093194B3968FFF7AFFF0346FB81FB89CE
:10E5C800002B1FD0154B1B78002B09D0FB891A464E
:10E5D8001149134808F0C9FC124AFB89138011E05D
:10E5E8000E4B01221A70FB891A460B490E4806F099
:10E5F8002DFD0346002B05D0084B00221A700B484E
:10E6080000F042FA01F026FF0346094A136000BFF2
:10E618001037BD4680BD00BF800B0020820D002052
:10E62800800C0020800D002004140020989C010814
:10E63800740A002080B500AF002200215220FFF7A5
:10E64800ABFF00BF80BD00BF80B500AF0022002136
:10E658005320FFF7A1FF00BF80BD00BF80B582B087
:10E6680000AF01F0F7FE78601E4B1B687A68D31A7A
:10E678003B601C4A7B6813601B4BB3F813309BB29A
:10E688001A46194BB3F815309BB202FB03F3174A2D
:10E6980082FB03129210DB17D31A1A46144B1A6026
:10E6A800134B1B683A6802FB03F3124AA2FB0323CD
:10E6B8009A09114B1B6813440F4A13600F4B1B78C0
:10E6C800012B02D10C4B00221A600B4B1B680C4A21
:10E6D800A2FB0323DB0A0B4A136000BF0837BD46C1
:10E6E80080BD00BFFC0D00208003002067666666C1
:10E6F800680A0020D34D62106C0A0020E40D002047
:10E70800C5B3A291700A002080B500AFFFF7A6FF3D
:10E71800FBF7D4FD03461A462A4B1A702A4BDA7ABD
:10E72800284B5A70294BB3F813309AB2254B5A80AC
:10E73800264BB3F815309AB2224B9A80244B1B68AB
:10E74800204AC2F80630234B1B681E4AC2F80A301A
:10E75800214B1B78042B04D1204B1A78194BDA74FF
:10E7680002E0184B0022DA741D4B1A88154B9A8266
:10E778001B4B5A88134BDA82194B9A88114B1A8310
:10E78800174BDA880F4B5A83154B9B680D4AD36198
:10E79800144B1A780B4B9A740A4A002343F07F43B0
:10E7A80043F47F0343F43B4343F0A003D3810023A6
:10E7B80043F00D031382202202495020FFF7ECFE9C
:10E7C80000BF80BD980D00207C0900208003002038
:10E7D800680A0020700A0020E50D002007000020CC
:10E7E8005C0A0020860D00204038C0B209289ABF74
:10E7F800024B33F810004FF6FF707047F8A001087D
:10E80800F8B504460D4601F025FE00233C4A3D4E6E
:10E8180013703D4A306013703C4A1370A4F14003F2
:10E82800092B65D8DFE803F009145B4E551B2A2E27
:10E838004A0501F00FFE3060F8BD2878344B642893
:10E8480028BF64201B78334A032B107043D1F8BDCE
:10E858002B78314A003B18BF01231370F8BD688834
:10E86800FAF7E8FF01462A88294B90B2A3F80F204F
:10E87800A3F81B10BDE8F840FCF7FEBB2A78274B2D
:10E888001A70F8BD264F2C463E4605F1200C354639
:10E8980020686168A268E368103464450FC506F112
:10E8A8001006F4D16168A268206807C61D4A7B88F3
:10E8B8001749A2FB0323DB088B70F8BD2A781A4B93
:10E8C8001A70F8BD2B78194A003B18BF0123137042
:10E8D800F8BD104B1878BDE8F840FBF7C7BC2B789B
:10E8E800002BA9D0BDE8F84005201149FBF700BF6F
:10E8F8002246BDE8F84005200E49FBF7F9BE00BFE7
:10E908008C0D0020880D00208D0D00208E0D00201C
:10E9180080030020340000207D0A0020860D00209E
:10E92800B80D0020CDCCCCCCE40D0020850D002006
:10E93800B49C0108CC9C01082DE9F04102290C4641
:10E94800054684B030D9431813F8012C13F8027C1B
:10E95800CE1E023989B247EA022790F80080FFF7F5
:10E9680097FD8742B6B212D14046FFF73DFF4FF6FA
:10E97800FF7290423AD086422AD13246FEB93146D9
:10E988004046FFF73DFF012004B0BDE8F08102904A
:10E99800234642460420CDE900671849FBF7A8FE44
:10E9A800002004B0BDE8F081D9B1012902784FF008
:10E9B800050009D06B781249FBF79AFEF0E740464C
:10E9C800691CFFF71DFFDEE70E49FBF791FEE7E73D
:10E9D80003464246CDE900640B490420FBF788FE54
:10E9E800DEE70A490520FBF783FED9E723464246BE
:10E9F800074900960520FBF77BFED1E7BC9D01087F
:10EA0800889D01085C9D0108649E01082C9D0108F1
:10EA1800209E010880B582B000AF01F01BFD0246C0
:10EA2800144B1B68D31A7B6001F014FD0246124B8D
:10EA38001B68D31A3B607B6840F2DB52934215DDBA
:10EA48003B6840F2DB52934210DD0C4B93F84230A6
:10EA5800DBB2202B0AD10A48FFF7F4F8094800F086
:10EA680013F801F0F7FC0346034A136000BF0837A8
:10EA7800BD4680BD900D0020940D00200414002098
:10EA8800BC9E0108C89E010880B586B004AF7860B6
:10EA98000D4806F0BAFF03460B4A92F84120D2B25D
:10EAA8001146094A92F84220D2B21046074A127813
:10EAB8000292019000917A6805490420FBF718FE3C
:10EAC80000BF0837BD4680BD04140020820D002019
:10EAD800E09E010880B500AF0E4B1B681B689AB218
:10EAE8000D4B1A800B4B1B685A790B4B9A70094BCC
:10EAF8001B681A79084BDA70074B01229A80064B7B
:10EB08000022DA80044B24221A81FAF761FE00BF42
:10EB180080BD00BF000000208412002080B500AF37
:10EB28004FF4047200210D4808F092F94FF4047272
:10EB380000210B4808F08CF90A4B00221A7001F0EA
:10EB480089FC0346084A1360074B1B68074A136091
:10EB580000F014FA00F036FA00BF80BD000E002065
:10EB6800101000202112002024120020281200205A
:10EB780080B500AF01F06EFC0246214B1B68D31A2A
:10EB8800002B3BDD01F066FC03461D4A136000F0D4
:10EB9800ADF900F0F3F900F015FA1A4B93F841308B
:10EBA800DBB2212B14D1184BD3F80C32002B0FD029
:10EBB80001F050FC0246144BD3F80C32D31A642BE4
:10EBC80006DD104806F068FB0F4B0022C3F80C2244
:10EBD8000D4B93F80832DBB2002B10D0094B93F899
:10EBE8004130DBB2212B0AD0084800F087FA064BE7
:10EBF800002283F8082200F0C1F900E000BF80BDC0
:10EC080090120020BC130020000E002000100020ED
:10EC18002E4B70B51A6803680C46934219D02C4ADB
:10EC28001268934204D02B4A126893424AD070BDAE
:10EC380099B329492246A1F5807000F049F910BB23
:10EC4800224605202549FBF753FDBDE8704000F03A
:10EC5800B9B991B301F0FEFB0022214B21491A708A
:10EC68000346214D214E2246A1F580702B6033606A
:10EC780000F02EF90546A8B100221D4B1A70BDE818
:10EC8800704000F07BB90122194B1A481A7000F045
:10EC980035FABDE8704000F095B917490520FBF733
:10ECA80027FDC6E7224615490520FBF721FD14225A
:10ECB8002946284600F0B6F8DEE711490520FBF79B
:10ECC80017FDC7E7BDE87040FEF7ECBFBC13002096
:10ECD8002C1300200414002010110020749F010838
:10ECE80021120020000F00202812002024120020EA
:10ECF8002012002010120020509F0108309F0108A8
:10ED08000C9F0108084B1A680368934204D0074A0D
:10ED18001268934205D070470022054BC3F80C22B5
:10ED28007047FFF769B800BFBC1300200414002027
:10ED3800000E0020C9B34FF0FF3300B51C4A014450
:10ED480010F801EB8EEA030E4EF300034EF3400C6D
:10ED5800134083EA5E030CEA020C8CEA530C43F37B
:10ED680040034CF3400E134083EA5C030EEA020EA4
:10ED78008EEA530E43F340034EF3400C134083EAEC
:10ED88005E030CEA020C8CEA530C43F34003134075
:10ED98004CF3400E83EA5C0381420EEA020C8CEAD3
:10EDA8005303CDD1D8435DF804FB0846704700BF34
:10EDB8002083B8ED70B51546137060B359B3944607
:10EDC800022302784C1EA4B21C440CF8012F05E063
:10EDD80010F8011FFB2B0CF8011F20D0A34203F1F0
:10EDE8000103F5D1A1B24E1CB6B22846FFF7A2FF27
:10EDF8000346711CB21C2B55C3F3072CC3F30744FD
:10EE080089B292B2C3F3076305F806C0F01C6C54CC
:10EE1800AB5480B270BD012402262146E5E70020EC
:10EE280070BD00BF38B51346114AFFF7C3FF80B164
:10EE38000446104890F84130202B0BD10C4D224647
:10EE480029460C4806F002F958B901F003FBC5F849
:10EE58000C0238BD06F020FA07490520FBF748FCEC
:10EE6800ECE704490548BDE8384000F005B900BFA3
:10EE7800000E0020BC130020949F0108C49F0108C5
:10EE88002DE978414B1FFB2B13D804398CB2031999
:10EE98009D7890465A782D0445EA0225025DDB7874
:10EEA8001543214645EA03650646FFF743FF8542B9
:10EEB80002D00020BDE87881731CC8F8043033788C
:10EEC800013C88F8003088F801400120BDE87881CD
:10EED80010B504460846114604F50072FFF7D0FF46
:10EEE80018B10123184684F8083210BD80B582B0E5
:10EEF80000AF01F0AFFA78601A4B1B687A68D31A32
:10EF08003B603B6841F28732934212DD164B1B7817
:10EF1800DBB2002B09D1154B002283F8082241F2FD
:10EF2800883213490520FBF7E3FB0F4B01221A70C7
:10EF380002E00D4B00221A700E4B93F84230DBB200
:10EF4800202B0AD10C4B1B687A68D31AC72B04DD17
:10EF580000F014F8084A7B68136000BF0837BD4604
:10EF680080BD00BF2412002021120020000E0020C6
:10EF7800E09F0108BC1300202812002080B500AFD4
:10EF88000C4B93F84230DBB2202B11D10A4B93F88B
:10EF98000832DBB2002B0BD1FF220849054806F0E6
:10EFA80022F90346002B03D00249054800F064F813
:10EFB80000BF80BDBC130020000E0020000F002001
:10EFC80004A0010880B500AF0A4B93F84230DBB2C9
:10EFD800202B0DD1FF220849064806F0A7F8034662
:10EFE800002B04D00349054800F046F800E000BFB4
:10EFF80080BD00BF2C130020101100201CA00108A8
:10F0080080B582B000AF78607B68154A934215D10D
:10F018001349144800F030F8114806F0A5F91048D3
:10F0280006F03AF9104B0022C3F80C22FFF7A6FFAE
:10F0380001F010FA03460D4A13600CE07B680C4A95
:10F04800934208D10A490B4800F016F8084806F020
:10F058008BF9FFF7B7FF00BF0837BD4680BD00BF7B
:10F06800BC13002034A00108000E00202812002044
:10F078002C13002048A0010890B587B004AF786031
:10F0880039607B68002B1CD03B68002B19D03B688B
:10F098001B681C46386806F0B8FC02463B6893F8C3
:10F0A8004130DBB219463B6893F84230DBB2029339
:10F0B8000191009223467A6804490420FBF718FB63
:10F0C80000E000BF0C37BD4690BD00BF5CA0010842
:10F0D80080B400AFBFF34F8F00BF064BDB6803F46B
:10F0E800E0620449044B1343CB60BFF34F8F00BF6A
:10F0F80000BFFDE700ED00E00400FA0580B584B02C
:10F1080000AF78601323FB737B681B78C22B00F376
:10F11800FF80B02B0FDA602B42D0602B00F3F88011
:10F12800502B43D0502B00F3F380012B00F0D980F3
:10F13800402B2DD0ECE0B03B122B00F2E98001A26D
:10F1480052F823F0BBF10008F9F100081DF200089D
:10F1580019F3000819F30008C9F2000819F30008A8
:10F16800BFF2000819F3000819F3000819F30008A2
:10F1780019F3000819F3000819F3000819F3000837
:10F1880019F3000855F20008B9F200088DF20008DA
:10F1980000F0E6F8402258216448FFF743FEC2E039
:10F1A80060220A216248FFF73DFEBCE0FBF73EFA09
:10F1B800B9E07B685B780B2B17D17B685A685D4B8D
:10F1C8001068516803C31189927A19809A705A4B52
:10F1D80001221A70574BD3F80330564A5749072073
:10F1E800FBF786FA1223FB7395E01323FB7392E077
:10F1F8007B685B78272B0AD17B685B681846FDF72C
:10F20800CBFF0346002B02D01223FB7383E01323AA
:10F21800FB7380E07B685B78012B14D17B685B68AB
:10F228001B78BB73BB7B012B0DD8BB7B1946022017
:10F23800FAF714FBBB7B1A4641490720FBF758FA3B
:10F248001223FB7367E01323FB7364E07B685B782E
:10F25800012B14D17B685B681B781A464FF47A73CC
:10F2680002FB03F31A46374B5A61364B5B691A4661
:10F2780035490720FBF73CFA1223FB734BE01323B5
:10F28800FB7348E07B685B78012B0ED17B685B6879
:10F298001A782E4B1A702D4B1B781A462C490720CA
:10F2A800FBF726FA1223FB7335E01323FB7332E0D6
:10F2B8001323FB732FE0FBF799FA1223FB732AE061
:10F2C800122200210020FFF7ADFD00BF214B93F86B
:10F2D8004130DBB2212BF9D00A2001F0C5F8FFF745
:10F2E800F7FE7B685B78092B0FD17B685A681A4B4D
:10F2F8001068516803C3127A1A70184B1B78DBB276
:10F30800012B0FD01223FB7305E01323FB7302E0DC
:10F318001323FB7300BFFB7B1A4600210020FFF775
:10F3280081FD00E000BF1037BD4680BD2C120020D3
:10F338008412002044000020941200208CA00108B0
:10F34800A0A001087C090020B8A0010880030020C3
:10F35800CCA00108BC130020380000202012002097
:10F3680080B500AF8D4B9A788D4B9A708B4BD3F844
:10F3780007308B4AC2F80330884BB3F80F309AB283
:10F38800874BA3F80720854BB3F81B309AB2844B00
:10F39800A3F80920814BB3F813309AB2804BA3F835
:10F3A8000B207E4BB3F815309AB27D4BA3F80D2095
:10F3B8007A4B1A7E7A4BDA73784B5A7F784B5A70AD
:10F3C800764B5A78764B1A7076497748FAF728FEC2
:10F3D800734B0022DA7400221A750420FAF7AEFA89
:10F3E800034603F00103D9B26D4A537D61F300036C
:10F3F80053750320FAF7A2FA034603F00103D9B2C2
:10F40800674A537D61F3410353750020FAF796FA72
:10F41800034603F00103D9B2614A537D61F38203C5
:10F4280053755F4A537D23F0080353750320FAF799
:10F4380095FA0346002B0CBF01230023D9B2584A82
:10F44800537D61F304135375FBF7DCF80346002B77
:10F4580014BF01230023D9B2514A537D61F34513E8
:10F4680053754F4A537D23F0400353754F4B1B7A16
:10F4780003F00103D9B24A4A537D61F3C7135375A8
:10F488000020FAF793FB03465AB2454B5A760120FF
:10F49800FAF78CFB03465AB2414B9A76434B9B6969
:10F4A8005AB23F4BDA763E4B00221A773C4B002289
:10F4B8005A773B4B00229A770022DA77384B0022A2
:10F4C80083F820203A4B9B689AB2354BA3F8212049
:10F4D800374BDB689AB2324BA3F82320344B1B69B5
:10F4E8009AB22F4BA3F8252011220021314807F0AA
:10F4F800AFFC2B4B002283F83820294B002283F8DD
:10F508003920002283F83A20254B002283F83B203B
:10F51800002283F83C2004220021274807F098FCA9
:10F528001F4B002283F84120002283F8422000224A
:10F5380083F84320002283F84420194B002283F8E3
:10F548004720174B002283F84620154B002283F8EA
:10F558004520134B002283F84820002283F84920D5
:10F568000F4B002283F84A2008220021134807F095
:10F578006FFC0B4B002283F85320094B002283F8C1
:10F588005420002283F85520054B002283F856208A
:10F59800002283F8572000BF80BD00BF80030020F1
:10F5A8002C1200203E1200203C1200207C09002072
:10F5B8005009002053120020691200207712002001
:10F5C80080B485B000AF78607B68002B18D07B686A
:10F5D80000221A607B6800229A807B680022DA8009
:10F5E8000023FB8108E0FA897B680232002143F896
:10F5F8002210FB890133FB81FB89072BF3D900E03B
:10F6080000BF1437BD4680BC704780B485B000AFDA
:10F61800786039607B68002B01D13B6856E07B68D5
:10F62800DB88072B27D87B689B881A467B680232C1
:10F63800396843F822107B681A683B681A447B686B
:10F648001A607B689B8801339AB27B689A807B68D2
:10F658009B88072B02D97B6800229A807B68DB880D
:10F6680001339AB27B68DA807B681B687A68D28833
:10F6780093FBF2F32AE07B689B881A467B68023288
:10F6880053F82230FB607B689B881A467B680232FD
:10F69800396843F822107B681A683968FB68CB1A06
:10F6A8001A447B681A607B689B8801339AB27B682E
:10F6B8009A807B689B88072B02D97B6800229A80F6
:10F6C8007B681B68002B00DA0733DB1018461437F9
:10F6D800BD4680BC7047000080B485B000AF154BB4
:10F6E8009B69144A43F001039361124B9B6903F031
:10F6F8000103BB60BB680F4BDB690E4A43F08053C4
:10F70800D3610C4BDB6903F080537B607B680A4B49
:10F718005B68FB60FB6823F0E063FB60FB6843F019
:10F728000073FB60044AFB68536000BF1437BD4692
:10F7380080BC70470010024000000140FEE700BF97
:10F74800FEE700BFFEE700BFFEE700BFFEE700BF21
:10F75800704700BF704700BF704700BF00F068BE29
:10F7680010B5094C01224FF40061204603F009FA54
:10F77800064802F0F7FD2046BDE8104000224FF48D
:10F78800006103F0FEB900BF000C014090020020A8
:10F79800014802F0E7BD00BF18150020014802F03B
:10F7A800E1BD00BFD4140020014802F0DBBD00BF5A
:10F7B8004C140020014802F0D5BD00BF9014002071
:10F7C80010B5094C01224FF40061204603F0D9F925
:10F7D800064801F023F82046BDE8104000224FF407
:10F7E800006103F0CEB900BF000C014060020020A8
:10F7F80010B5094C01224FF48061204603F0C1F98D
:10F80800064802F047F82046BDE8104000224FF4B1
:10F81800806103F0B6B900BF000C01402C03002042
:10F8280010B5094C01224FF40061204603F0A9F9F4
:10F83800064804F087FD2046BDE8104000224FF43A
:10F84800006103F09EB900BF000C01409C1200202B
:10F85800014805F02DBE00BF7413002010B5084CF8
:10F8680001222021204603F08CF9064805F020FEED
:10F878002046BDE810400022202103F082B900BFD5
:10F8880000080140BC13002010B5084C012240219B
:10F89800204603F076F9064805F00AFE2046BDE842
:10F8A80010400022402103F06CB900BF000801405D
:10F8B8000414002010B5084C01220421204603F04E
:10F8C80060F9064805F0F4FD2046BDE81040002226
:10F8D800042103F056B900BF001001402C1300208A
:10F8E80010B5094C01224FF48061204603F049F914
:10F8F800064801F0CFFF2046BDE8104000224FF433
:10F90800806103F03EB900BF000C014054030020A1
:10F9180010B5094C01224FF48061204603F031F9FB
:10F92800064801F0B7FF2046BDE8104000224FF41A
:10F93800806103F026B900BF000C01405403002089
:10F9480080B400AF01231846BD4680BC704780B51F
:10F9580082B000AF7860396007F0CCFA034616220F
:10F968001A604FF0FF3318460837BD4680BD80B592
:10F9780082B000AF78604FF0FF317868FFF7E7FF9B
:10F9880000BFFDE780B586B000AFF860B9607A6067
:10F9980000237B610AE0AFF300800146BB685A1C74
:10F9A800BA60CAB21A707B6901337B617A697B6875
:10F9B8009A42F0DB7B6818461837BD4680BD80B494
:10F9C80083B000AF78604FF0FF3318460C37BD4660
:10F9D80080BC704780B483B000AF786039603B6802
:10F9E8004FF400525A60002318460C37BD4680BCBD
:10F9F800704780B483B000AF7860012318460C3795
:10FA0800BD4680BC704780B485B000AFF860B9606F
:10FA18007A60002318461437BD4680BC7047000042
:10FA280080B586B000AF7860144A154BD31A7B6155
:10FA38007B693B61134B1B68002B02D1114B124AA7
:10FA48001A60104B1A687B6813443A699A4207D2C5
:10FA580007F050FA03460C221A604FF0FF3309E012
:10FA6800084B1B68FB60074B1A687B681344054A00
:10FA78001360FB6818461837BD4680BD000001209A
:10FA88000004000098120020B016002080B400AFD7
:10FA980000BFBD4680BC704780B58EB000AF07F18F
:10FAA800280300221A605A609A60DA6007F120037E
:10FAB80000221A605A603B1D00221A605A609A6040
:10FAC800DA601A615A619A61384B394A1A60374BC1
:10FAD80000225A60354B00229A60344B4FF6FF7271
:10FAE800DA60324B00221A61304B00229A612F48AB
:10FAF80004F0D5F90346002B01D0FBF7D1F94FF4F8
:10FB08008053BB6207F128031946284804F028FEF1
:10FB18000346002B01D0FBF7C3F9244804F00EFA82
:10FB28000346002B01D0FBF7BBF9204804F008FB83
:10FB38000346002B01D0FBF7B3F930233B620023C7
:10FB48007B6207F120031946184805F0B7F9034608
:10FB5800002B01D0FBF7A4F900237B600123BB60D5
:10FB68000023FB6000237B613B1D002219460F48E0
:10FB780004F0D8FC0346002B01D0FBF791F9602371
:10FB88007B600023BB603B1D04221946074804F034
:10FB980025FD0346002B01D0FBF782F9034800F04E
:10FBA800CFF800BF3837BD4680BD00BF9C1200208B
:10FBB8000004004080B58EB000AF07F12803002292
:10FBC8001A605A609A60DA6007F1200300221A600E
:10FBD8005A603B1D00221A605A609A60DA601A6106
:10FBE8005A619A61374B384A1A60364B4FF434726F
:10FBF8005A60344B00229A60324B6422DA60314BEF
:10FC080000221A612F4B00229A612E4804F047F90E
:10FC18000346002B01D0FBF743F94FF48053BB6236
:10FC280007F128031946274804F09AFD0346002BDC
:10FC380001D0FBF735F9234804F082FA0346002B7C
:10FC480001D0FBF72DF900233B6200237B6207F10B
:10FC5800200319461B4805F031F90346002B01D053
:10FC6800FBF71EF960237B600023BB600023FB6069
:10FC780000237B613B1D04221946124804F0AEFCA8
:10FC88000346002B01D0FBF70BF93B1D0822194650
:10FC98000C4804F0A3FC0346002B01D0FBF700F945
:10FCA8003B1D0C221946074804F098FC0346002B1C
:10FCB80001D0FBF7F5F8034800F042F800BF3837E9
:10FCC800BD4680BDE41200200008004080B584B025
:10FCD80000AF78607B681B68164A934214D1164BB4
:10FCE800DB69154A43F00203D361134BDB6903F068
:10FCF8000203FB60FB68002206211D2002F0C5F804
:10FD08001D2002F0DEF810E07B681B680B4A934266
:10FD18000BD1094BDB69084A43F00403D361064B56
:10FD2800DB6903F00403BB60BB6800BF1037BD4646
:10FD380080BD00BF000400400010024000080040E1
:10FD480080B58AB000AF786007F1140300221A600A
:10FD58005A609A60DA607B681B68264A934218D119
:10FD6800254B9B69244A43F004039361224B9B690A
:10FD780003F004033B613B6980237B610223BB6181
:10FD880002233B6207F1140319461C4802F05EFD8A
:10FD98002BE07B681B681A4A934226D1164B9B6955
:10FDA800154A43F020039361134B9B6903F020032A
:10FDB800FB60FB684FF460437B610223BB61022355
:10FDC8003B6207F1140319460E4802F03FFD0E4B43
:10FDD8005B687B627B6A43F0E0637B627B6A43F427
:10FDE80080537B62084A7B6A536000BF2837BD4650
:10FDF80080BD00BF00040040001002400008014020
:10FE080000080040001401400000014080B500AF28
:10FE1800114B124A1A60104B4FF416525A600E4B8F
:10FE280000229A600C4B0022DA600B4B00221A6108
:10FE3800094B0C225A61084B00229A61064B00229A
:10FE4800DA61054805F0B2F80346002B01D0FBF74C
:10FE580027F800BF80BD00BF2C13002000500040D1
:10FE680080B500AF114B124A1A60104B4FF4E132C3
:10FE78005A600E4B00229A600C4B0022DA600B4B42
:10FE880000221A61094B0C225A61084B00229A6120
:10FE9800064B0022DA61054805F088F80346002B76
:10FEA80001D0FAF7FDFF00BF80BD00BF741300202A
:10FEB8000038014080B500AF114B124A1A60104B50
:10FEC8004FF4E1325A600E4B00229A600C4B00222C
:10FED800DA600B4B00221A61094B0C225A61084B5D
:10FEE80000229A61064B0022DA61054805F05EF8A7
:10FEF8000346002B01D0FAF7D3FF00BF80BD00BF37
:10FF0800BC1300200044004080B500AF114B124ADA
:10FF18001A60104B4FF4E1325A600E4B00229A607F
:10FF28000C4B0022DA600B4B00221A61094B0C22A1
:10FF38005A61084B00229A61064B0022DA61054893
:10FF480005F034F80346002B01D0FAF7A9FF00BFEB
:10FF580080BD00BF041400200048004080B592B066
:10FF680000AF786007F1300300221A605A609A6087
:10FF7800DA607B681B68924A934245D1914BDB69F2
:10FF8800904A43F48013D3618E4BDB6903F48013EA
:10FF9800FB62FB6A8B4B9B698A4A43F010039361AF
:10FFA800884B9B6903F01003BB62BB6A854B9B6956
:10FFB800844A43F020039361824B9B6903F020033A
:10FFC8007B627B6A4FF480533B6302237B6303238A
:10FFD800FB6307F1300319467B4802F037FC042322
:10FFE8003B6300237B630023BB6307F1300319469F
:08FFF800764802F02BFC002208
:020000040801F1
:100000000521352001F045FF352001F05EFF93E129
:100010007B681B68704A93423AD16C4B9B696B4A70
:1000200043F480439361694B9B6903F480433B62D3
:100030003B6A664B9B69654A43F004039361634BDB
:100040009B6903F00403FB61FB694FF400733B639E
:1000500002237B630323FB6307F1300319465F48E8
:1000600002F0F8FB4FF480633B6300237B630023C3
:10007000BB6307F130031946584802F0EBFB00223E
:100080000521252001F005FF252001F01EFF53E189
:100090007B681B68524A934240F0AE804B4BDB6951
:1000A0004A4A43F40033D361484BDB6903F400331D
:1000B000BB61BB69454B9B69444A43F02003936194
:1000C000424B9B6903F020037B617B6920233B63E8
:1000D00002237B630323FB6307F1300319463D488A
:1000E00002F0B8FB40233B6300237B630023BB6328
:1000F00007F130031946374802F0ACFB394B5B6817
:100100003B643B6C43F0E0633B643B6C43F00803AF
:100110003B64344A3B6C5360334B344A1A60324B75
:1001200000225A60304B00229A602F4B8022DA6006
:100130002D4B00221A612C4B00225A612A4B0022BF
:100140009A61294B4FF44052DA61274801F0F4FEDE
:100150000346002B01D0FAF7A7FE7B68224ADA6338
:10016000214A7B685362224B224A1A60204B10229C
:100170005A601F4B00229A601D4B8022DA601C4B94
:1001800000221A611A4B00225A61194B00229A610F
:10019000174B4FF40052DA61154801F0CDFE0346CB
:1001A000002B01D0FAF780FE7B68114A9A63104A4F
:1001B0007B68536200220221262001F06AFE26207D
:1001C00001F083FEB8E000BF005000400010024084
:1001D00000100140001401400038014000080140B7
:1001E00000440040000001404C1400206C0002401C
:1001F00090140020800002407B681B68504A9342A4
:1002000040F09A804F4BDB694E4A43F48023D36120
:100210004C4BDB6903F480233B613B69494B9B6991
:10022000484A43F010039361464B9B6903F0100367
:10023000FB60FB684FF480633B6302237B63032313
:10024000FB6307F1300319463F4802F003FB4FF40C
:1002500000633B6300237B630023BB6307F1300330
:100260001946394802F0F6FA384B5B687B647B6CC0
:1002700023F030037B647B6C43F0E0637B647B6C36
:1002800043F010037B64314A7B6C5360304B314A3E
:100290001A602F4B00225A602D4B00229A602C4B83
:1002A0008022DA602A4B00221A61294B00225A610F
:1002B000274B00229A61264B4FF44052DA612448C2
:1002C00001F03AFE0346002B01D0FAF7EDFD7B6802
:1002D0001F4ADA631E4A7B6853621F4B1F4A1A602B
:1002E0001D4B10225A601C4B00229A601A4B802230
:1002F000DA60194B00221A61174B00225A61164B23
:1003000000229A61144B4FF40052DA61124801F056
:1003100013FE0346002B01D0FAF7C6FD7B680E4A98
:100320009A630D4A7B68536200220221272001F064
:10033000B0FD272001F0C9FD00BF4837BD4680BD94
:100340000048004000100240001001400000014041
:10035000D414002030000240181500201C00024078
:10036000FFF798FB0B480C490C4A002302E0D458D5
:10037000C4500433C4188C42F9D3094A094C0023F1
:1003800001E013600432A242FBD306F0BDFDFAF790
:100390007FFC70470000002024020020ECA401082C
:1003A00028020020AC160020FEE7000080B500AF58
:1003B000084B1B68074A43F010031360032001F049
:1003C0005DFD0F2000F008F8FFF78AF900231846BA
:1003D00080BD00BF0020024080B582B000AF7860D1
:1003E000124B1A68124B1B7819464FF47A73B3FB01
:1003F000F1F3B2FBF3F3184601F075FD0346002B51
:1004000001D001230EE07B680F2B0AD80022796807
:100410004FF0FF3001F03DFD064A7B68136000237A
:1004200000E0012318460837BD4680BD500000207B
:10043000580000205400002080B400AF054B1B780A
:100440001A46054B1B681344034A136000BFBD46A0
:1004500080BC7047580000205C15002080B400AFBD
:10046000024B1B681846BD4680BC70475C150020D7
:1004700080B584B000AF7860FFF7F0FFB8607B68AC
:10048000FB60FB68B3F1FF3F05D00A4B1B781A46AF
:10049000FB681344FB6000BFFFF7E0FF0246BB6848
:1004A000D31AFA689A42F7D800BF00BF1037BD468A
:1004B00080BD00BF5800002080B586B000AF7860D6
:1004C0000023FB7500233B610023BB600023FB601E
:1004D0007B68002B01D10123BEE07B689B68002B69
:1004E0007B689B6A002B09D17B680022DA627B68FB
:1004F000002283F824207868F9F7D4F8786800F0AF
:10050000BDFB0346FB757B689B6A03F01003002B61
:1005100040F09980FB7D002B40F095807B689B6AC2
:1005200023F4885323F0020343F002027B689A62AB
:100530007B685A687B68DB691A437B681B7B5B00BE
:100540001343BA681343BB607B689B68B3F5807F35
:1005500003D07B689B68012B02D14FF4807300E0CD
:1005600000233A6913433B617B681B7D012B19D142
:100570007B681B7B002B09D17B689B69013B5A037D
:100580003B69134343F400633B610BE07B689B6A68
:1005900043F020027B689A627B68DB6A43F00102C9
:1005A0007B68DA627B681B685B6823F469417B685F
:1005B0001B683A690A435A607B681B689A68284B33
:1005C00013407A681268B9680B4393607B689B6834
:1005D000B3F5807F03D07B689B68012B04D17B68D7
:1005E0001B69013B1B05FB607B681B68DB6A23F40E
:1005F00070017B681B68FA680A43DA627B681B68D3
:100600009A68184B1340BA689A420BD17B68002253
:10061000DA627B689B6A23F0030343F001027B6884
:100620009A6218E07B689B6A23F0120343F0100281
:100630007B689A627B68DB6A43F001027B68DA625E
:100640000123FB7507E07B689B6A43F010027B681F
:100650009A620123FB75FB7D18461837BD4680BDA5
:10066000FDF7E1FFFE0E1FFF80B586B000AFF8601A
:10067000B9607A600023FB75FB681B68644A93428B
:1006800004D0FB681B68634A934206D1604B5B68E9
:1006900003F47023002B40F0B380FB6893F8243000
:1006A000012B01D10223AEE0FB68012283F8242054
:1006B000F86800F089FA0346FB75FB7D002B40F0DB
:1006C0009A80FB689B6A23F4706323F0010343F470
:1006D0008072FB689A62FB681B684E4A934205D1A0
:1006E0004B4B5B6803F47023002B15D1FB689B6AAE
:1006F00023F48012FB689A62FB681B685B6803F452
:100700008063002B26D0FB689B6A23F4405343F49C
:100710008052FB689A621DE0FB689B6A43F480127A
:10072000FB689A62FB681B68394A934204D0FB68F5
:100730001B68384A93420DD1354B5B6803F48063E4
:10074000002B07D0FB689B6A23F4405343F480528C
:10075000FB689A62FB689B6A03F48053002B06D007
:10076000FB68DB6A23F00602FB68DA6202E0FB68E2
:100770000022DA62FB68002283F82420FB681B6AEF
:10078000254A9A62FB681B6A244ADA62FB681B6A84
:10079000234A1A63FB681B686FF002021A60FB6849
:1007A0001B689A68FB681B6842F480729A60FB6859
:1007B000186AFB681B684C331946BA687B6801F0FD
:1007C00031FCFB681B689B6803F46023B3F5602F62
:1007D00008D1FB681B689A68FB681B6842F4A0029A
:1007E0009A600FE0FB681B689A68FB681B6842F41C
:1007F00080129A6006E0FB68002283F8242001E062
:100800000123FB75FB7D18461837BD4680BD00BF30
:100810000024014000280140FF0C01087B0D010865
:10082000970D010880B584B000AF78607B681B68C5
:100830001B68FB607B681B685B68BB60BB6803F080
:100840002003002B3ED0FB6803F00203002B39D0BD
:100850007B689B6A03F01003002B05D17B689B6AC1
:1008600043F400727B689A627B681B689B6803F4A0
:100870006023B3F5602F1DD17B681B7B002B19D142
:100880007B681B685A687B681B6822F020025A60EC
:100890007B689B6A23F480727B689A627B689B6AA0
:1008A00003F48053002B05D17B689B6A43F001025F
:1008B0007B689A627868F8F749FE7B681B686FF07E
:1008C00012021A60BB6803F08003002B4DD0FB6856
:1008D00003F00403002B48D07B689B6A03F01003ED
:1008E000002B05D17B689B6A43F400527B689A62B7
:1008F0007B681B689B6803F4E043B3F5E04F12D0BC
:100900007B681B685B6803F48063002B25D17B68E0
:100910001B689B6803F46023B3F5602F1DD17B68CF
:100920001B7B002B19D17B681B685A687B681B688E
:1009300022F080025A607B689B6A23F480527B68B5
:100940009A627B689B6A03F48073002B05D17B68F5
:100950009B6A43F001027B689A62786800F0E4FACF
:100960007B681B686FF00C021A60BB6803F04003E1
:10097000002B12D0FB6803F00103002B0DD07B6825
:100980009B6A43F480327B689A62786800F012F8C0
:100990007B681B686FF001021A6000BF1037BD460C
:1009A00080BD80B483B000AF786000BF0C37BD4617
:1009B00080BC704780B483B000AF786000BF0C3754
:1009C000BD4680BC704780B483B000AF786000BF84
:1009D0000C37BD4680BC704780B485B000AF7860EE
:1009E00039600023FB730023BB607B6893F82430DD
:1009F000012B01D10223DCE07B68012283F8242053
:100A00003B685B68062B1CD87B681B68596B3B688E
:100A10005A6813469B001344053B1F2202FA03F356
:100A2000DB4319403B6818683B685A6813469B00D3
:100A30001344053B00FA03F27B681B680A435A63C0
:100A40003CE03B685B680C2B1CD87B681B68196B0F
:100A50003B685A6813469B001344233B1F2202FA4B
:100A600003F3DB4319403B6818683B685A68134638
:100A70009B001344233B00FA03F27B681B680A4384
:100A80001A631BE07B681B68D96A3B685A68134687
:100A90009B001344413B1F2202FA03F3DB4319403E
:100AA0003B6818683B685A6813469B001344413BF7
:100AB00000FA03F27B681B680A43DA623B681B6832
:100AC000092B1CD97B681B68D9683B681A681346D8
:100AD0005B0013441E3B072202FA03F3DB43194079
:100AE0003B6898683B681A6813465B0013441E3BDA
:100AF00000FA03F27B681B680A43DA6019E07B683E
:100B00001B6819693B681A6813465B001344072287
:100B100002FA03F3DB4319403B6898683B681A68A4
:100B200013465B00134400FA03F27B681B680A4318
:100B30001A613B681B68102B03D03B681B68112BA4
:100B400032D17B681B681D4A934225D17B681B68A4
:100B50009B6803F40003002B26D17B681B689A680E
:100B60007B681B6842F400029A603B681B68102B8C
:100B70001AD1134B1B68134AA2FB03239A0C13468A
:100B80009B0013445B00BB6002E0BB68013BBB60A1
:100B9000BB68002BF9D107E07B689B6A43F0200219
:100BA0007B689A620123FB737B68002283F8242010
:100BB000FB7B18461437BD4680BC704700240140BB
:100BC0005000002083DE1B4380B584B000AF786006
:100BD0000023FB600023BB607B681B689B6803F0FD
:100BE0000103012B40D07B681B689A687B681B68F7
:100BF00042F001029A601F4B1B681F4AA2FB0323AD
:100C00009B0CBB6002E0BB68013BBB60BB68002B78
:100C1000F9D1FFF723FCF8601FE0FFF71FFC024645
:100C2000FB68D31A022B18D97B681B689B6803F0FA
:100C30000103012B11D07B689B6A43F010027B6893
:100C40009A627B68DB6A43F001027B68DA627B6848
:100C5000002283F82420012307E07B681B689B683F
:100C600003F00103012BD8D1002318461037BD46ED
:100C700080BD00BF5000002083DE1B4380B584B0E0
:100C800000AF78600023FB607B681B689B6803F003
:100C90000103012B2ED17B681B689A687B681B6857
:100CA00022F001029A60FFF7D9FBF8601BE0FFF722
:100CB000D5FB0246FB68D31A022B14D97B681B684C
:100CC0009B6803F00103012B0DD17B689B6A43F005
:100CD00010027B689A627B68DB6A43F001027B68E2
:100CE000DA62012307E07B681B689B6803F001035D
:100CF000012BDCD0002318461037BD4680BD80B5DF
:100D000084B000AF78607B685B6AFB60FB689B6ABD
:100D100003F05003002B27D1FB689B6A43F4007259
:100D2000FB689A62FB681B689B6803F46023B3F559
:100D3000602F15D1FB681B7B002B11D1FB689B6AD0
:100D400023F48072FB689A62FB689B6A03F4805309
:100D5000002B05D1FB689B6A43F00102FB689A6295
:100D6000F868F8F7F3FB04E0FB681B6A1B6B786814
:100D7000984700BF1037BD4680BD80B584B000AF36
:100D800078607B685B6AFB60F868FFF70AFE00BF6B
:100D90001037BD4680BD80B584B000AF78607B68F9
:100DA0005B6AFB60FB689B6A43F04002FB689A62E7
:100DB000FB68DB6A43F00402FB68DA62F868FFF75D
:100DC00002FE00BF1037BD4680BD000090B587B061
:100DD00000AF78600023FB750023FB607B6893F80D
:100DE0002430012B01D1022397E07B68012283F894
:100DF00024207868FFF742FF0346FB757868FFF709
:100E0000E3FE0346FB75FB7D002B40F081807B6891
:100E10009B6A23F4885323F0020343F002027B68A9
:100E20009A62404B1C68022002F0E2FD0346B4FBCC
:100E3000F3F35B00FB6002E0FB68013BFB60FB68D7
:100E4000002BF9D17B681B689A687B681B6842F0AD
:100E500008029A60FFF702FB38611BE0FFF7FEFA19
:100E600002463B69D31A0A2B14D97B681B689B681E
:100E700003F00803002B0DD07B689B6A23F012035C
:100E800043F010027B689A627B68002283F824207A
:100E9000012342E07B681B689B6803F00803002B7A
:100EA000DCD17B681B689A687B681B6842F004028F
:100EB0009A60FFF7D3FA38611BE0FFF7CFFA0246DA
:100EC0003B69D31A0A2B14D97B681B689B6803F013
:100ED0000403002B0DD07B689B6A23F0120343F0C0
:100EE00010027B689A627B68002283F82420012329
:100EF00013E07B681B689B6803F00403002BDCD1C4
:100F00007B689B6A23F0030343F001027B689A62CB
:100F10007B68002283F82420FB7D18461C37BD46E1
:100F200090BD00BF5000002080B483B000AF786057
:100F300000BF0C37BD4680BC704780B584B000AFA1
:100F400078607B68002B01D10123EDE07B6893F88A
:100F50002030DBB2002B02D17868F8F7E5FE7B6821
:100F60001B681A687B681B6842F001021A60FFF771
:100F700075FAF86012E0FFF771FA0246FB68D31ABF
:100F80000A2B0BD97B685B6A43F400327B685A6298
:100F90007B68052283F820200123C5E07B681B685D
:100FA0005B6803F00103002BE5D07B681B681A68BF
:100FB0007B681B6822F002021A60FFF74FFAF860A4
:100FC00012E0FFF74BFA0246FB68D31A0A2B0BD943
:100FD0007B685B6A43F400327B685A627B68052257
:100FE00083F8202001239FE07B681B685B6803F087
:100FF0000203002BE5D17B681B7E012B08D17B68A7
:101000001B681A687B681B6842F080021A6007E060
:101010007B681B681A687B681B6822F080021A6074
:101020007B685B7E012B08D17B681B681A687B6834
:101030001B6842F040021A6007E07B681B681A6870
:101040007B681B6822F040021A607B689B7E012B44
:1010500008D17B681B681A687B681B6842F0200215
:101060001A6007E07B681B681A687B681B6822F0BF
:1010700020021A607B68DB7E012B08D17B681B682D
:101080001A687B681B6822F010021A6007E07B6810
:101090001B681A687B681B6842F010021A607B6844
:1010A0001B7F012B08D17B681B681A687B681B6853
:1010B00042F008021A6007E07B681B681A687B68C8
:1010C0001B6822F008021A607B685B7F012B08D145
:1010D0007B681B681A687B681B6842F004021A6010
:1010E00007E07B681B681A687B681B6822F00402B3
:1010F0001A607B689A687B68DB681A437B681B69A7
:101100001A437B685B6942EA03017B685B685A1E8D
:101110007B681B680A43DA617B6800225A627B683D
:10112000012283F82020002318461037BD4680BDD9
:1011300080B487B000AF786039607B681B687B61E2
:101140007B6893F82030FB74FB7C012B03D0FB7C85
:10115000022B40F0BE80654B7B617B69D3F8003287
:1011600043F001027B69C3F800227B69D3F80032A7
:1011700023F47C527B69C3F800227B69D3F80022F8
:101180003B685B6A1B021A437B69C3F800223B6819
:101190005B6903F01F03012202FA03F3FB607B6922
:1011A000D3F81C22FB68DB431A407B69C3F81C227E
:1011B0003B68DB69002B23D17B69D3F80C22FB68E9
:1011C000DB431A407B69C3F80C223B68DB681904D7
:1011D0003B685B689BB23A68526919437B69483245
:1011E00043F832103B689B6819043B681B689AB24D
:1011F0003B685B690A4379694833DB000B445A60FA
:101200003B68DB69012B22D17B69D3F80C22FB6898
:101210001A437B69C3F80C223B681B6819043B68BE
:101220005B689BB23A68526919437B69483243F85C
:1012300032103B689B6819043B68DB689AB23B68D4
:101240005B690A4379694833DB000B445A603B68A9
:101250009B69002B09D17B69D3F80422FB68DB432F
:101260001A407B69C3F8042207E07B69D3F80422A3
:10127000FB681A437B69C3F804223B681B69002B97
:1012800009D17B69D3F81422FB68DB431A407B69E0
:10129000C3F8142207E07B69D3F81422FB681A43D1
:1012A0007B69C3F814223B681B6A012B07D17B6959
:1012B000D3F81C22FB681A437B69C3F81C227B69A4
:1012C000D3F8003223F001027B69C3F80022002327
:1012D00006E07B685B6A43F480227B685A620123E4
:1012E00018461C37BD4680BC704700BF00640040F4
:1012F00080B584B000AF78607B6893F82030DBB2B3
:10130000012B2ED17B68022283F820207B681B688A
:101310001A687B681B6822F001021A60FFF79EF8CA
:10132000F86012E0FFF79AF80246FB68D31A0A2B1E
:101330000BD97B685B6A43F400327B685A627B6836
:10134000052283F82020012312E07B681B685B687C
:1013500003F00103002BE5D17B6800225A620023D1
:1013600006E07B685B6A43F400227B685A620123D3
:1013700018461037BD4680BD80B584B000AF786098
:101380007B6893F82030DBB2022B33D17B681B687B
:101390001A687B681B6842F001021A60FFF75EF86A
:1013A000F86012E0FFF75AF80246FB68D31A0A2BDE
:1013B0000BD97B685B6A43F400327B685A627B68B6
:1013C000052283F8202001231BE07B681B685B68F3
:1013D00003F00103002BE5D07B681B681A687B686B
:1013E0001B6822F002021A607B68012283F8202029
:1013F000002306E07B685B6A43F480127B685A62D4
:10140000012318461037BD4680BD80B489B000AFB7
:10141000F860B9607A603B60FB6893F82030FB7736
:10142000FB681B689B68BB61FB7F012B03D0FB7FC4
:10143000022B40F0AD80BB6903F08063002B0AD122
:10144000BB6903F00063002B05D1BB6903F0805337
:10145000002B00F09580BB691B0E03F003037B613A
:1014600001227B699A403B681A60BB689B68002B2D
:101470000DD1BB681B685A05BB68DB68F968096851
:101480001A437B6918331B010B441A600FE0BB68D9
:101490005B68DA00BB689B681A43BB68DB68F96865
:1014A00009681A437B6918331B010B441A60FB68F7
:1014B0001968BB681A697B6918331B010B44043334
:1014C0001A60BB681B7D012B11D1FB681A687B6910
:1014D00018331B01134404331B68FA68116843F482
:1014E00080727B6918331B010B4404331A607B68DC
:1014F00007331B781A067B6806331B781B041A43D4
:101500007B6805331B781B0213437A680432127818
:101510001046FA68116843EA00027B691B010B441C
:1015200003F5C6731A607B6803331B781A067B6861
:1015300002331B781B041A437B6801331B781B02A0
:1015400013437A6812781046FA68116843EA000279
:101550007B691B010B4403F5C4731A60FB681A68AE
:101560007B6918331B0113441B68FA68116843F048
:1015700001027B6918331B010B441A6000230EE043
:10158000FB685B6A43F40012FB685A62012306E0C1
:10159000FB685B6A43F48022FB685A6201231846A9
:1015A0002437BD4680BC704780B485B000AF7860FA
:1015B0000023FB607B6893F82030FB72FB7A012BE1
:1015C00002D0FB7A022B1DD17B681B689B6803F05D
:1015D0008063002B02D0FB680133FB607B681B68D3
:1015E0009B6803F00063002B02D0FB680133FB60B3
:1015F0007B681B689B6803F08053002B02D0FB685C
:101600000133FB60FB6818461437BD4680BC704749
:1016100080B487B000AFF860B9607A603B60FB6867
:1016200093F82030FB75FB7D012B03D0FB7D022B53
:1016300040F00381BB68002B0ED1FB681B68DB68A0
:1016400003F00303002B16D1FB685B6A43F400121E
:10165000FB685A620123F7E0FB681B681B6903F013
:101660000303002B07D1FB685B6A43F40012FB689D
:101670005A620123E8E0FB681A68BB681B331B0150
:1016800013441B6803F004027B689A607B689B68C4
:10169000002B0CD1FB681A68BB681B331B01134479
:1016A0001B685B0DC3F30A027B681A600BE0FB68E2
:1016B0001A68BB681B331B0113441B68DB0823F04B
:1016C00060427B685A60FB681A68BB681B331B0169
:1016D00013441B6803F002027B68DA60FB681A6837
:1016E000BB681B331B01134404331B6803F008035E
:1016F000002B03D07B6808221A610BE0FB681A6894
:10170000BB681B331B01134404331B6803F00F0237
:101710007B681A61FB681A68BB681B331B011344A2
:1017200004331B681B0ADAB27B689A61FB681A688B
:10173000BB681B331B01134404331B681B0C9AB298
:101740007B685A61FB681A68BB681B01134403F588
:10175000DC731B68DAB23B681A70FB681A68BB68F6
:101760001B01134403F5DC731B681A0A3B68013341
:10177000D2B21A70FB681A68BB681B01134403F5E8
:10178000DC731B681A0C3B680233D2B21A70FB6818
:101790001A68BB681B01134403F5DC731B681A0E3F
:1017A0003B680333D2B21A70FB681A68BB681B012E
:1017B000134403F5DE731A683B680433D2B21A701F
:1017C000FB681A68BB681B01134403F5DE731B68D2
:1017D0001A0A3B680533D2B21A70FB681A68BB68F4
:1017E0001B01134403F5DE731B681A0C3B680633B8
:1017F000D2B21A70FB681A68BB681B01134403F568
:10180000DE731B681A0E3B680733D2B21A70BB68CE
:10181000002B08D1FB681B68DA68FB681B6842F084
:101820002002DA6007E0FB681B681A69FB681B6826
:1018300042F020021A61002306E0FB685B6A43F471
:101840008022FB685A62012318461C37BD4680BCC3
:10185000704780B485B000AF786039607B6893F8DA
:101860002030FB73FB7B012B02D0FB7B022B09D1C9
:101870007B681B6859697B681B683A680A435A6130
:10188000002306E07B685B6A43F480227B685A622F
:10189000012318461437BD4680BC704780B58AB016
:1018A00000AF786000237B627B681B685B693B62EA
:1018B0007B681B685B68FB617B681B689B68BB611E
:1018C0007B681B68DB687B617B681B681B693B610D
:1018D0007B681B689B69FB603B6A03F00103002B7C
:1018E0007CD0BB6903F00103002B23D07B681B680D
:1018F00001229A60BB6903F00203002B03D07868D1
:1019000000F083F916E0BB6903F00403002B04D058
:101910007B6A43F400637B620CE0BB6903F008035D
:10192000002B04D07B6A43F480537B6202E078682A
:1019300000F086F9BB6903F48073002B24D07B6828
:101940001B684FF480729A60BB6903F40073002B2C
:1019500003D0786800F062F916E0BB6903F4806395
:10196000002B04D07B6A43F400537B620CE0BB691C
:1019700003F40063002B04D07B6A43F480437B6252
:1019800002E0786800F065F9BB6903F48033002B4E
:1019900024D07B681B684FF480329A60BB6903F4E3
:1019A0000033002B03D0786800F041F916E0BB69E2
:1019B00003F48023002B04D07B6A43F400437B6252
:1019C0000CE0BB6903F40023002B04D07B6A43F4D2
:1019D00080337B6202E0786800F044F93B6A03F0F0
:1019E0000803002B0CD07B6903F01003002B07D0F9
:1019F0007B6A43F400737B627B681B681022DA60A9
:101A00003B6A03F00403002B0BD07B6903F008034F
:101A1000002B06D07B681B680822DA60786800F02B
:101A200033F93B6A03F00203002B09D07B681B6883
:101A3000DB6803F00303002B02D0786800F01BF989
:101A40003B6A03F04003002B0CD03B6903F010030A
:101A5000002B07D07B6A43F480637B627B681B6842
:101A600010221A613B6A03F02003002B0BD03B6964
:101A700003F00803002B06D07B681B6808221A615C
:101A8000786800F00AF93B6A03F01003002B09D0D4
:101A90007B681B681B6903F00303002B02D0786886
:101AA000FAF768FB3B6A03F40033002B0BD0FB69A9
:101AB00003F01003002B06D07B681B6810225A60CD
:101AC000786800F0F3F83B6A03F48033002B0BD006
:101AD000FB6903F00803002B06D07B681B68082213
:101AE0005A60786800F0EBF83B6A03F40043002B7F
:101AF0007BD0FB6903F00403002B72D03B6A03F434
:101B00008073002B08D0FB6803F00103002B03D087
:101B10007B6A43F001037B623B6A03F40073002B92
:101B200008D0FB6803F00203002B03D07B6A43F06C
:101B300002037B623B6A03F48063002B08D0FB68DE
:101B400003F00403002B03D07B6A43F004037B62A1
:101B50003B6A03F40063002B43D0FB6803F070037F
:101B6000002B3ED0FB6803F07003602B2BD0602B62
:101B70002ED8502B22D0502B2AD8402B19D0402BB6
:101B800026D8302B10D0302B22D8102B02D0202B6F
:101B900005D01DE07B6A43F008037B6219E07B6A95
:101BA00043F010037B6214E07B6A43F020037B6206
:101BB0000FE07B6A43F040037B620AE07B6A43F0FC
:101BC00080037B6205E07B6A43F480737B6200E004
:101BD00000BF7B681B689A697B681B6822F07002F3
:101BE0009A617B681B6804225A607B6A002B08D0CC
:101BF0007B685A6A7B6A1A437B685A62786800F08D
:101C000067F800BF2837BD4680BD80B483B000AF01
:101C1000786000BF0C37BD4680BC704780B483B08D
:101C200000AF786000BF0C37BD4680BC704780B401
:101C300083B000AF786000BF0C37BD4680BC7047F2
:101C400080B483B000AF786000BF0C37BD4680BC65
:101C5000704780B483B000AF786000BF0C37BD46DA
:101C600080BC704780B483B000AF786000BF0C3791
:101C7000BD4680BC704780B483B000AF786000BFC1
:101C80000C37BD4680BC704780B483B000AF78602D
:101C900000BF0C37BD4680BC704780B483B000AF36
:101CA000786000BF0C37BD4680BC704780B483B0FD
:101CB00000AF786000BF0C37BD4680BC704780B471
:101CC00083B000AF786000BF0C37BD4680BC704762
:101CD00080B483B000AF786000BF0C37BD4680BCD5
:101CE0007047000080B485B000AF78607B6803F077
:101CF0000703FB600C4BDB68BB60BA684FF6FF0361
:101D00001340BB60FB681A02BB68134343F0BF6318
:101D100043F40033BB60044ABB68D36000BF143790
:101D2000BD4680BC704700BF00ED00E080B400AF4E
:101D3000044BDB681B0A03F007031846BD4680BC52
:101D4000704700BF00ED00E080B483B000AF0346F1
:101D5000FB7197F90730002B0BDBFB7903F01F02B7
:101D6000064997F907305B09012000FA02F241F8B1
:101D7000232000BF0C37BD4680BC704700E100E067
:101D800080B483B000AF03463960FB7197F9073028
:101D9000002B0ADB3B68DAB20C4997F907301201D5
:101DA000D2B20B4483F800230AE03B68DAB2084958
:101DB000FB7903F00F03043B1201D2B20B441A76F5
:101DC00000BF0C37BD4680BC704700BF00E100E09B
:101DD00000ED00E080B489B000AFF860B9607A60CF
:101DE000FB6803F00703FB61FB69C3F10703042BE6
:101DF00028BF0423BB61FB690433062B02D9FB69AE
:101E0000033B00E000237B614FF0FF32BB6902FA25
:101E100003F3DA43BB681A407B699A404FF0FF3105
:101E20007B6901FA03F3D9437B680B4013431846DF
:101E30002437BD4680BC704780B582B000AF786063
:101E40007B68013BB3F1807F01D301230FE00A4A95
:101E50007B68013B53600F214FF0FF30FFF790FF8D
:101E6000054B00229A60044B07221A600023184693
:101E70000837BD4680BD00BF10E000E080B582B0ED
:101E800000AF78607868FFF72DFF00BF0837BD46C8
:101E900080BD80B586B000AF0346B9607A60FB7341
:101EA00000237B61FFF742FF78617A68B96878693F
:101EB000FFF790FF024697F90F3011461846FFF7DB
:101EC0005FFF00BF1837BD4680BD80B582B000AF50
:101ED0000346FB7197F907301846FFF735FF00BF3F
:101EE0000837BD4680BD80B582B000AF78607868A5
:101EF000FFF7A2FF034618460837BD4680BD80B5F0
:101F000082B000AF78607B68002B01D101230EE026
:101F10007B685B79DBB2002B05D17B6800221A71EC
:101F20007868F8F7E5FA7B6801225A7100231846B1
:101F30000837BD4680BD000080B485B000AF786032
:101F40000023FB607B68002B01D1012359E07B68F3
:101F50001B681A462D4B9A420FD87B681B681A469D
:101F60002B4B13442B4AA2FB03231B099A007B68CB
:101F70001A647B68284ADA630EE07B681B681A469D
:101F8000264B1344234AA2FB03231B099A007B68B8
:101F90001A647B68224ADA637B68022283F8212074
:101FA0007B681B681B68FB60FB6823F47F5323F08E
:101FB0003003FB607B685A687B689B681A437B68C8
:101FC000DB681A437B681B691A437B685B691A43A9
:101FD0007B689B691A437B68DB691343FA68134388
:101FE000FB607B681B68FA681A607B6800229A6352
:101FF0007B68012283F821207B68002283F820205F
:10200000002318461437BD4680BC704707040240C1
:10201000F8FFFDBFCDCCCCCC00000240F8FBFDBFEB
:102020000004024080B586B000AFF860B9607A6005
:102030003B600023FB75FB6893F82030012B01D136
:1020400002234BE0FB68012283F82020FB6893F811
:102050002130DBB2012B3AD1FB68022283F8212028
:10206000FB6800229A63FB681B681A68FB681B68A0
:1020700022F001021A603B687A68B968F86800F0DB
:10208000BCFBFB68DB6A002B08D0FB681B681A6886
:10209000FB681B6842F00E021A600FE0FB681B68C9
:1020A0001A68FB681B6822F004021A60FB681B6850
:1020B0001A68FB681B6842F00A021A60FB681B681A
:1020C0001A68FB681B6842F001021A6005E0FB68B1
:1020D000002283F820200223FB75FB7D1846183769
:1020E000BD4680BD80B485B000AF78600023FB732F
:1020F0007B6893F82130DBB2022B08D07B68042286
:102100009A637B68002283F82020012320E07B680B
:102110001B681A687B681B6822F00E021A607B68D5
:102120001B681A687B681B6822F001021A607B68D2
:102130001A6C7B68DB6B012101FA02F25A607B6842
:10214000012283F821207B68002283F82020FB7B7A
:1021500018461437BD4680BC7047000080B584B077
:1021600000AF78600023FB737B6893F82130DBB20B
:10217000022B05D07B6804229A630123FB73D6E00F
:102180007B681B681A687B681B6822F00E021A6065
:102190007B681B681A687B681B6822F001021A6062
:1021A0007B681B681A46644B9A4258D97B681B6847
:1021B000624A93424FD07B681B68614A934248D081
:1021C0007B681B685F4A934240D07B681B685E4A0D
:1021D000934238D07B681B685C4A934230D07B685E
:1021E0001B685B4A934228D07B681B68524A934223
:1021F00020D07B681B68574A934219D07B681B68C4
:10220000554A934212D07B681B68544A93420AD0C5
:102210007B681B68524A934202D14FF480531BE003
:102220004FF4803318E04FF4807315E0102313E06F
:10223000012311E04FF080730EE04FF480130BE0A8
:102240004FF4803308E04FF4805305E04FF480737F
:1022500002E0102300E00123424A536057E07B680C
:102260001B68364A93424FD07B681B68344A9342BE
:1022700048D07B681B68334A934240D07B681B6818
:10228000314A934238D07B681B68304A934230D041
:102290007B681B682E4A934228D07B681B68264ABD
:1022A000934220D07B681B682A4A934219D07B68EE
:1022B0001B68294A934212D07B681B68274A9342C5
:1022C0000AD07B681B68264A934202D14FF48053A0
:1022D0001BE04FF4803318E04FF4807315E01023B7
:1022E00013E0012311E04FF080730EE04FF48013F0
:1022F0000BE04FF4803308E04FF4805305E04FF4D7
:10230000807302E0102300E00123174A53607B68CA
:10231000012283F821207B68002283F820207B683B
:102320005B6B002B03D07B685B6B78689847FB7B0B
:1023300018461037BD4680BD8000024008000240AC
:102340001C0002403000024044000240580002409D
:102350006C000240080402401C04024030040240A9
:1023600044040240000402400000024080B584B0F2
:1023700000AF78607B68DB6B1B68FB607B681B6869
:102380001B68BB607B681B6C04229A40FB6813408F
:10239000002B00F0F180BB6803F00403002B00F079
:1023A000EB807B681B681B6803F02003002B07D1C0
:1023B0007B681B681A687B681B6822F004021A603D
:1023C0007B681B681A465F4B9A4258D97B681B682A
:1023D0005D4A93424FD07B681B685C4A934248D069
:1023E0007B681B685A4A934240D07B681B68594AF5
:1023F000934238D07B681B68574A934230D07B6841
:102400001B68564A934228D07B681B684D4A93420A
:1024100020D07B681B68524A934219D07B681B68A6
:10242000504A934212D07B681B684F4A93420AD0AD
:102430007B681B684D4A934202D14FF480431BE0F6
:102440004FF4802318E04FF4806315E0402313E03D
:10245000042311E04FF080630EE04FF480030BE0A3
:102460004FF4802308E04FF4804305E04FF480638D
:1024700002E0402300E004233D4A536057E07B68BC
:102480001B68314A93424FD07B681B682F4A9342A6
:1024900048D07B681B682E4A934240D07B681B68FB
:1024A0002C4A934238D07B681B682B4A934230D029
:1024B0007B681B68294A934228D07B681B68214AA5
:1024C000934220D07B681B68254A934219D07B68D1
:1024D0001B68244A934212D07B681B68224A9342AD
:1024E0000AD07B681B68214A934202D14FF4804393
:1024F0001BE04FF4802318E04FF4806315E0402385
:1025000013E0042311E04FF080630EE04FF48003EA
:102510000BE04FF4802308E04FF4804305E04FF4D4
:10252000806302E0402300E00423124A53607B688A
:10253000DB6A002B00F036817B68DB6A786898479D
:1025400030E100BF80000240080002401C00024051
:102550003000024044000240580002406C0002403B
:10256000080402401C0402403004024044040240BB
:1025700000040240000002407B681B6C02229A406B
:10258000FB681340002B00F0DD80BB6803F0020302
:10259000002B00F0D7807B681B681B6803F02003CA
:1025A000002B0BD17B681B681A687B681B6822F0C4
:1025B0000A021A607B68012283F821207B681B686D
:1025C0001A467B4B9A4258D97B681B68794A9342DA
:1025D0004FD07B681B68784A934248D07B681B6861
:1025E000764A934240D07B681B68754A934238D044
:1025F0007B681B68734A934230D07B681B68724AC1
:10260000934228D07B681B68694A934220D07B683C
:102610001B686E4A934219D07B681B686C4A9342D0
:1026200012D07B681B686B4A93420AD07B681B6898
:10263000694A934202D14FF400531BE04FF4003338
:1026400018E04FF4007315E0202313E0022311E09B
:102650004FF000730EE04FF400130BE04FF4003323
:1026600008E04FF4005305E04FF4007302E020232C
:1026700000E00223594A536057E07B681B684D4ACB
:1026800093424FD07B681B684B4A934248D07B688B
:102690001B684A4A934240D07B681B68484A934271
:1026A00038D07B681B68474A934230D07B681B68F0
:1026B000454A934228D07B681B683D4A934220D00C
:1026C0007B681B68414A934219D07B681B68404A6B
:1026D000934212D07B681B683E4A93420AD07B68C3
:1026E0001B683D4A934202D14FF400531BE04FF464
:1026F000003318E04FF4007315E0202313E00223A9
:1027000011E04FF000730EE04FF400130BE04FF4B4
:10271000003308E04FF4005305E04FF4007302E08B
:10272000202300E002232E4A53607B68002283F8B6
:1027300020207B689B6A002B34D07B689B6A78687A
:1027400098472FE07B681B6C08229A40FB68134077
:10275000002B28D0BB6803F00803002B23D07B6834
:102760001B681A687B681B6822F00E021A607B687F
:102770001A6C7B68DB6B012101FA02F25A607B68FC
:1027800001229A637B68012283F821207B68002262
:1027900083F820207B681B6B002B04D07B681B6BAD
:1027A0007868984700BF00BF1037BD4680BD00BFA6
:1027B00080000240080002401C000240300002403D
:1027C00044000240580002406C00024008040240ED
:1027D0001C04024030040240440402400004024051
:1027E0000000024080B483B000AF78607B689B6BD0
:1027F00018460C37BD4680BC704780B485B000AF2A
:10280000F860B9607A603B60FB681A6CFB68DB6B50
:10281000012101FA02F25A60FB681B683A685A60AB
:10282000FB685B68102B08D1FB681B687A689A60AC
:10283000FB681B68BA68DA6007E0FB681B68BA6867
:102840009A60FB681B687A68DA6000BF1437BD467F
:1028500080BC704780B48BB000AF786039600023D3
:102860007B6200233B6269E101227B6A02FA03F387
:10287000FB613B681B68FA691340BB61BA69FB697D
:102880009A4240F058813B685B689A4A93425ED016
:10289000984A934275D8984A934258D0964A9342A0
:1028A0006FD8964A934252D0944A934269D8944A38
:1028B00093424CD0924A934263D8924A934246D074
:1028C000904A93425DD8122B2AD8122B59D801A2D4
:1028D00052F823F04F290108292901083B29010852
:1028E0007D2901088329010883290108832901081A
:1028F0008329010883290108832901088329010804
:1029000083290108832901088329010883290108F3
:102910008329010883290108312901084529010873
:10292000794A934213D02CE03B68DB683B6229E094
:102930003B68DB6804333B6224E03B68DB680833B8
:102940003B621FE03B68DB680C333B621AE03B688C
:102950009B68002B02D104233B6213E03B689B6819
:10296000012B05D108233B627B68FA691A6109E0F3
:1029700008233B627B68FA695A6103E000233B62EB
:1029800000E000BFBB69FF2B01D87B6801E07B68DA
:1029900004337B61BB69FF2B02D87B6A9B0002E09A
:1029A0007B6A083B9B003B617B691A680F213B698E
:1029B00001FA03F3DB431A40396A3B6901FA03F376
:1029C0001A437B691A603B685B6803F08053002BF5
:1029D00000F0B1804D4B9B694C4A43F00103936179
:1029E0004A4B9B6903F00103BB60BB68484A7B6AA2
:1029F0009B08023352F82330FB607B6A03F0030329
:102A00009B000F2202FA03F3DB43FA681340FB60DA
:102A10007B68404A934213D07B683F4A93420DD073
:102A20007B683E4A934207D07B683D4A934201D17E
:102A3000032306E0042304E0022302E0012300E074
:102A400000237A6A02F0030292009340FA6813436B
:102A5000FB602F497B6A9B080233FA6841F8232008
:102A60003B685B6803F48013002B06D02D4B9A68FB
:102A70002C49BB6913438B6006E02A4B9A68BB69FB
:102A8000DB43284913408B603B685B6803F4001309
:102A9000002B06D0234BDA682249BB691343CB6075
:102AA00006E0204BDA68BB69DB431E491340CB606C
:102AB0003B685B6803F40033002B06D0194B5A685F
:102AC0001849BB6913434B6006E0164B5A68BB6953
:102AD000DB43144913404B603B685B6803F480336D
:102AE000002B21D00F4B1A680E49BB6913430B60B2
:102AF00021E000BF00003210000031100000221061
:102B000000002110000012100000111000100240FF
:102B10000000014000080140000C0140001001408D
:102B200000140140000401400B4B1A68BB69DB43F1
:102B3000094913400B607B6A01337B623B681A686A
:102B40007B6A22FA03F3002B7FF48EAE00BF00BF36
:102B50002C37BD4680BC70470004014080B485B06E
:102B600000AF78600B467B807B689A687B88134057
:102B7000002B02D00123FB7301E00023FB73FB7BDE
:102B800018461437BD4680BC704780B483B000AF90
:102B900078600B467B8013467B707B78002B03D0DC
:102BA0007A887B681A6103E07B881A047B681A6163
:102BB00000BF0C37BD4680BC7047000080B400AF3A
:102BC000034B01221A6000BFBD4680BC704700BFA6
:102BD00020000E4280B582B000AFFDF73FFC786068
:102BE000604B1B685F4A43F00103136008E0FDF788
:102BF00035FC02467B68D31A022B01D90323ACE0D3
:102C0000584B1B6803F00203002BF0D0554B1B6898
:102C100023F0F803534A43F080031360FDF71EFCD2
:102C20007860504B00225A600AE0FDF717FC02461C
:102C30007B68D31A41F28832934201D903238CE096
:102C4000484B5B6803F00C03002BEED1464B474A20
:102C50001A60474B1B681846FDF7BEFB0346002B66
:102C600001D0012379E0FDF7F9FB78603D4B1B684B
:102C70003C4A23F08073136008E0FDF7EFFB024647
:102C80007B68D31A022B01D9032366E0354B1B68FE
:102C900003F00073002BF0D1324B00225A60FDF795
:102CA000DDFB78602F4B1B682E4A23F41023136042
:102CB00008E0FDF7D3FB02467B68D31A642B01D9E9
:102CC00003234AE0274B1B6803F40033002BF0D1A9
:102CD000244B1B68234A23F480231360FDF7BEFBBB
:102CE0007860204B1B681F4A23F08063136008E064
:102CF000FDF7B4FB02467B68D31A642B01D903238A
:102D00002BE0184B1B6803F00063002BF0D1FDF79C
:102D1000A5FB7860134B1B68124A23F080531360A5
:102D200008E0FDF79BFB02467B68D31A642B01D9B0
:102D3000032312E00B4B1B6803F00053002BF0D170
:102D4000084B0022DA62074B5B6A064A43F0807345
:102D50005362044B00229A60002318460837BD4690
:102D600080BD00BF001002405000002000127A0019
:102D70005400002080B586B000AF78607B68002BDF
:102D800001D1012304E37B681B6803F00103002BDE
:102D900000F08780924B5B6803F00C03042B0CD08F
:102DA0008F4B5B6803F00C03082B12D18C4B5B68D4
:102DB00003F48033B3F5803F0BD1894B1B6803F4D8
:102DC0000033002B6CD07B689B68002B68D10123FB
:102DD000DEE27B689B68B3F5803F06D1804B1B68C1
:102DE0007F4A43F4803313602EE07B689B68002B9E
:102DF0000CD17B4B1B687A4A23F480331360784BE9
:102E00001B68774A23F4802313601DE07B689B686E
:102E1000B3F5A02F0CD1724B1B68714A43F4802389
:102E200013606F4B1B686E4A43F4803313600BE0F2
:102E30006B4B1B686A4A23F480331360684B1B6832
:102E4000674A23F4802313607B689B68002B13D0B0
:102E5000FDF704FB386108E0FDF700FB02463B6923
:102E6000D31A642B01D9032392E25D4B1B6803F450
:102E70000033002BF0D014E0FDF7F0FA386108E0E1
:102E8000FDF7ECFA02463B69D31A642B01D9032300
:102E90007EE2534B1B6803F40033002BF0D100E0BB
:102EA00000BF7B681B6803F00203002B63D04C4B10
:102EB0005B6803F00C03002B0BD0494B5B6803F0FD
:102EC0000C03082B1CD1464B5B6803F48033002BAA
:102ED00016D1434B1B6803F00203002B05D07B681F
:102EE0005B69012B01D0012352E23D4B1B6823F0AB
:102EF000F8027B689B69DB00394913430B603AE0B9
:102F00007B685B69002B20D0364B01221A60FDF7ED
:102F1000A5FA386108E0FDF7A1FA02463B69D31A29
:102F2000022B01D9032333E22D4B1B6803F002036C
:102F3000002BF0D02A4B1B6823F0F8027B689B69BA
:102F4000DB00274913430B6015E0264B00221A6073
:102F5000FDF784FA386108E0FDF780FA02463B6924
:102F6000D31A022B01D9032312E21D4B1B6803F075
:102F70000203002BF0D17B681B6803F00803002BD1
:102F80003AD07B68DB69002B19D0174B01221A60FD
:102F9000FDF764FA386108E0FDF760FA02463B6924
:102FA000D31A022B01D90323F2E10D4B5B6A03F024
:102FB0000203002BF0D0012000F0CAFB1CE00A4BFA
:102FC00000221A60FDF74AFA38610FE0FDF746FA71
:102FD00002463B69D31A022B08D90323D8E100BF6C
:102FE0000010024000004242800442429B4B5B6A58
:102FF00003F00203002BE9D17B681B6803F0040394
:10300000002B00F0A6800023FB75944BDB6903F0D6
:103010008053002B0DD1914BDB69904A43F08053D4
:10302000D3618E4BDB6903F08053BB60BB68012327
:10303000FB758B4B1B6803F48073002B18D1884BF6
:103040001B68874A43F480731360FDF707FA386101
:1030500008E0FDF703FA02463B69D31A642B01D955
:10306000032395E17E4B1B6803F48073002BF0D0A3
:103070007B681B69012B06D1784B1B6A774A43F0AA
:10308000010313622DE07B681B69002B0CD1734B8D
:103090001B6A724A23F001031362704B1B6A6F4A6A
:1030A00023F0040313621CE07B681B69052B0CD121
:1030B0006A4B1B6A694A43F004031362674B1B6A3D
:1030C000664A43F0010313620BE0644B1B6A634AD8
:1030D00023F001031362614B1B6A604A23F004036F
:1030E00013627B681B69002B15D0FDF7B7F93861B7
:1030F0000AE0FDF7B3F902463B69D31A41F2883280
:10310000934201D9032343E1544B1B6A03F00203AA
:10311000002BEED014E0FDF7A1F938610AE0FDF7CD
:103120009DF902463B69D31A41F28832934201D994
:1031300003232DE1494B1B6A03F00203002BEED160
:10314000FB7D012B05D1454BDB69444A23F08053BD
:10315000D3617B68DB6A002B00F08C803F4B5B689F
:1031600003F48033B3F5803F0ED13C4B5B6803F032
:103170000C03082B08D1394BDB6A03F48033B3F519
:10318000803F01D1012303E17B68DB6A022B4ED132
:10319000324B1B6803F08053002B09D02F4BDB6AA6
:1031A00003F0F0027B685B6B9A4201D00123EFE0F1
:1031B0002C4B00221A60FDF751F9386108E0FDF749
:1031C0004DF902463B69D31A642B01D90323DFE092
:1031D000224B1B6803F00063002BF0D11F4BDB6A0E
:1031E00023F0F0027B685B6B1C491343CB621B4BE3
:1031F000DB6A23F470627B681B6B18491343CB6254
:10320000184B01221A60FDF729F9386108E0FDF733
:1032100025F902463B69D31A642B01D90323B7E091
:103220000E4B1B6803F00063002BF0D022E00B4B29
:10323000DB6A0A4A23F48033D3620A4B00221A6005
:10324000FDF70CF938610FE0FDF708F902463B691C
:10325000D31A642B08D903239AE000BF0010024060
:1032600000700040680042424B4B1B6803F0006353
:10327000002BE9D17B681B6A002B00F08880464B4D
:103280005B6803F00C03082B68D07B681B6A022B79
:103290004DD1424B00221A60FDF7E0F8386108E09A
:1032A000FDF7DCF802463B69D31A022B01D9032350
:1032B0006EE0394B1B6803F00073002BF0D17B6884
:1032C0005B6AB3F5803F0FD1334BDA6A7B685B688A
:1032D00031491343CB62304BDB6A23F00F027B682A
:1032E000DB682D491343CB622B4B5B6823F47412CC
:1032F0007B68596A7B689B6A0B43274913434B6081
:10330000264B01221A60FDF7A9F8386108E0FDF7A5
:10331000A5F802463B69D31A022B01D9032337E0F3
:103320001D4B1B6803F00073002BF0D02FE01B4BEC
:1033300000221A60FDF792F8386108E0FDF78EF878
:1033400002463B69D31A022B01D9032320E0124B1A
:103350001B6803F00073002BF0D118E07B681B6A38
:10336000012B01D1012313E00B4B5B68FB60FB6871
:1033700003F480327B685B6A9A4206D1FB6803F4EF
:1033800070127B689B6A9A4201D0012300E00023FF
:1033900018461837BD4680BD00100240600042420A
:1033A00080B584B000AF786039607B68002B01D1B4
:1033B0000123D0E06A4B1B6803F007033A689A4286
:1033C00010D9674B1B6823F0070265493B6813431C
:1033D0000B60634B1B6803F007033A689A4201D005
:1033E0000123B8E07B681B6803F00203002B20D0A8
:1033F0007B681B6803F00403002B05D0594B5B6806
:10340000584A43F4E06353607B681B6803F0080389
:10341000002B05D0534B5B68524A43F46053536012
:10342000504B5B6823F0F0027B689B684D49134367
:103430004B607B681B6803F00103002B40D07B6866
:103440005B68012B07D1474B1B6803F40033002B4B
:1034500015D101237FE07B685B68022B07D1414BCC
:103460001B6803F00073002B09D1012373E03D4B6F
:103470001B6803F00203002B01D101236BE0394BE1
:103480005B6823F003027B685B68364913434B603B
:10349000FCF7E4FFF8600AE0FCF7E0FF0246FB6897
:1034A000D31A41F28832934201D9032353E02D4BC2
:1034B0005B6803F00C027B685B689B009A42EBD16F
:1034C000274B1B6803F007033A689A4210D2244B3B
:1034D0001B6823F0070222493B6813430B60204B13
:1034E0001B6803F007033A689A4201D0012332E0D7
:1034F0007B681B6803F00403002B08D0194B5B6842
:1035000023F4E0627B68DB68164913434B607B68F9
:103510001B6803F00803002B09D0124B5B6823F4EF
:1035200060527B681B69DB000E4913434B6000F05F
:1035300021F802460B4B5B681B0903F00F030A4995
:10354000CB5C22FA03F3094A1360094B1B68184647
:10355000FCF742FF002318461037BD4680BD00BF70
:1035600000200240001002400CA101085000002081
:10357000540000202DE9B04F8EB000AF0023FB6255
:103580000023BB6200237B6300237B6200233B6339
:1035900000233B620023FB614E4B5B68FB62FB6ACE
:1035A00003F00C03042B02D0082B03D089E04A4B14
:1035B0003B6389E0FB6A9B0C03F00F02474B9B5C6B
:1035C0007B62FB6A03F48033002B72D0414BDB6AD1
:1035D00003F00F02424B9B5CBB623E4BDB6A03F481
:1035E0008033002B53D03B4BDB6A1B0903F00F03E6
:1035F00001333B62374BDB6A1B0A03F00F030233D4
:10360000FB61FB6900229A4693467B6A00223B617C
:103610007A613B6903FB0BF27B690AFB03F31344FA
:103620003A69AAFB02010B4419462B4B03FB01F23A
:10363000002300FB03F31344274AA0FB02452B445D
:103640001D463B6A0022BB60FA60BB6A00223B60F9
:103650007A60D7E902010B46D7E900AB524602FB7C
:1036600003F25B4684460CFB03F3134402465146C7
:10367000A2FB01894B44994642464B4620462946C7
:10368000F5F7B8FD02460B4613467B6307E07B6AFD
:10369000114A03FB02F2BB6AB2FBF3F37B630F4BED
:1036A0005B7B1A467B6A934208D17B6B5B087B632A
:1036B00004E07B6A0B4A02FB03F37B637B6B3B6397
:1036C00002E0094B3B6300BF3B6B18463837BD46F1
:1036D000BDE8B08F0010024040787D0124A10108B0
:1036E00034A1010800093D0000127A0080B400AF47
:1036F000024B1B681846BD4680BC70475000002036
:1037000080B500AFFFF7F2FF0246054B5B681B0A6E
:1037100003F007030349CB5C22FA03F3184680BD8C
:10372000001002401CA1010880B500AFFFF7DEFFCA
:103730000246054B5B68DB0A03F007030349CB5CD9
:1037400022FA03F3184680BD001002401CA10108B4
:1037500080B485B000AF78600A4B1B680A4AA2FBB0
:1037600003235B0A7A6802FB03F3FB6000BFFB687C
:103770005A1EFA60002BF9D100BF00BF1437BD46B6
:1037800080BC704750000020D34D621080B588B0D7
:1037900000AF786000237B6100233B610023FB6165
:1037A0007B681B6803F00103002B7DD00023FB76B0
:1037B0008B4BDB6903F08053002B0DD1884BDB6909
:1037C000874A43F08053D361854BDB6903F0805314
:1037D000FB60FB680123FB76824B1B6803F480735C
:1037E000002B18D17F4B1B687E4A43F48073136013
:1037F000FCF734FE786108E0FCF730FE02467B6996
:10380000D31A642B01D90323E5E0764B1B6803F43C
:103810008073002BF0D0724B1B6A03F440733B6142
:103820003B69002B2ED07B685B6803F440733A69D8
:103830009A4227D06A4B1B6A23F440733B616A4B60
:1038400001221A60684B00221A60654A3B691362C4
:103850003B6903F00103002B14D0FCF7FFFD7861F6
:103860000AE0FCF7FBFD02467B69D31A41F288327D
:10387000934201D90323AEE0594B1B6A03F00203C4
:10388000002BEED0564B1B6A23F440727B685B68BA
:10389000534913430B62FB7E012B05D1504BDB696F
:1038A0004F4A23F08053D3617B681B6803F0020307
:1038B000002B08D04A4B5B6823F440427B689B682E
:1038C000474913434B607B681B6803F00403002BDC
:1038D00008D0434BDB6A23F400327B68DB68404945
:1038E0001343CB627B681B6803F00803002B08D0EE
:1038F0003B4BDB6A23F480227B681B693849134306
:10390000CB62374BDB6A03F40033002B05D1344B19
:10391000DB6A03F48023002B01D00123FB61FB69E8
:10392000012B48D12E4B1B6803F08053002B38D15C
:103930002B4B1B6803F08063002B09D0284BDB6AFC
:1039400003F0F0027B689B699A4201D0012342E0B8
:10395000234BDB6A23F0F0027B689B692049134309
:10396000CB621F4BDB6A23F470427B685B691C49A6
:103970001343CB621D4B01221A60FCF76FFD786187
:1039800008E0FCF76BFD02467B69D31A642B01D972
:10399000032320E0124B1B6803F00053002BF0D0F0
:1039A00009E00F4BDB6A03F470427B685B699A4263
:1039B00001D001230FE07B681B6803F01003002B8C
:1039C00008D0074B5B6823F480027B68DB690449FD
:1039D00013434B60002318462037BD4680BD00BF0F
:1039E0000010024000700040400442427000424219
:1039F00080B58AB000AF78600023FB6100237B6252
:103A00000023BB6100237B6100233B610023FB603B
:103A10000023BB6000233B627B68013B0F2B00F25D
:103A20001D8101A252F823F0DD3B0108413C010851
:103A30005D3C01083B3B01085D3C01085D3C010821
:103A40005D3C01088D3B01085D3C01085D3C0108BF
:103A50005D3C01085D3C01085D3C01085D3C0108DE
:103A60005D3C0108693A0108834B5B68BB60824B8F
:103A70001B6803F08073002B00F0F280BB689B0C86
:103A800003F00F037D4AD35CBB61BB6803F4803352
:103A9000002B3BD0784BDB6A03F00F03784AD35CF2
:103AA000FB61754BDB6A03F48033002B1CD0724B37
:103AB000DB6A1B0903F00F030133FB606E4BDB6A0B
:103AC0001B0A03F00F0302337B616E4AFB68B2FBF3
:103AD000F3F37A6903FB02F2FB69B2FBF3F2BB6911
:103AE00002FB03F37B6207E0664AFB69B2FBF3F279
:103AF000BB6902FB03F37B62604B5B7B1A46BB69CD
:103B0000934208D17B6A5B087B6204E0BB695E4A32
:103B100002FB03F37B62584B5B6803F48003B3F54D
:103B2000800F02D17B6A3B629AE07B6A5B00574A56
:103B3000A2FB03235B083B6292E04F4BDB6A03F47A
:103B40000033002B03D1FFF715FD38628AE04A4BA2
:103B50001B6803F08053002B00F08480464BDB6A27
:103B60001B0903F00F030133FB60434BDB6A1B0BA4
:103B700003F00F0302333B61424AFB68B2FBF3F3ED
:103B80003A6902FB03F35B003B626BE03A4BDB6A92
:103B900003F48023002B03D1FFF7ECFC386263E0D1
:103BA000354B1B6803F08053002B5DD0324BDB6A32
:103BB0001B0903F00F030133FB602F4BDB6A1B0B68
:103BC00003F00F0302333B612E4AFB68B2FBF3F3B1
:103BD0003A6902FB03F35B003B6245E0264B1B6A3C
:103BE000BB60BB6803F44073B3F5807F08D1BB684A
:103BF00003F00203002B03D04FF400433B621EE0AE
:103C0000BB6803F44073B3F5007F09D11A4B5B6ABC
:103C100003F00203002B03D049F640433B620EE061
:103C2000BB6803F44073B3F5407F1FD1124B1B6890
:103C300003F40033002B19D0154B3B6216E015E05E
:103C4000FFF772FD02460C4B5B689B0B03F003030E
:103C500001335B00B2FBF3F33B6208E000BF06E018
:103C600000BF04E000BF02E000BF00E000BF3B6A0D
:103C700018462837BD4680BD0010024044A1010807
:103C800054A1010840787D0100093D00ABAAAAAA11
:103C9000F0FA020080B584B000AF78600023FB60CA
:103CA0007B68002B01D101237AE07B685B7CDBB26F
:103CB000002B05D17B6800221A747868F9F760FF41
:103CC0007B6802225A74786800F070F80346002B73
:103CD00004D07B6804225A74012361E0786800F004
:103CE00092F80346002B04D07B6804225A74012307
:103CF00056E07B681B685A687B681B6822F00702E5
:103D00005A607B689B68002B05D0274B1B6B264AAB
:103D100023F001031363244BDB6A23F460727B6896
:103D20009B6821491343CB627B685B68B3F1FF3F1B
:103D300003D07B685B68FB600EE00120FFF758FE54
:103D4000F860FB68002B04D17B6804225A740123BD
:103D500026E0FB68013BFB60FB681A0C7B681B6874
:103D600002F00F029A607B681B68FA6892B2DA6010
:103D7000786800F070F80346002B04D07B680422BA
:103D80005A7401230CE07B680022DA737B680122FD
:103D90005A737B6801229A737B6801225A7400234C
:103DA00018461037BD4680BD006C004080B584B019
:103DB00000AF78600023FB607B68002B01D10123FA
:103DC0001DE07B681B685A687B681B6822F008024C
:103DD0005A60FCF743FBF86009E0FCF73FFB024642
:103DE000FB68D31AB3F57A7F01D9032307E07B6818
:103DF0001B685B6803F00803002BEED00023184615
:103E00001037BD4680BD80B584B000AF7860002318
:103E1000FB60FCF723FBF86009E0FCF71FFB0246A0
:103E2000FB68D31AB3F57A7F01D903230FE07B68CF
:103E30001B685B6803F02003002BEED07B681B68D7
:103E40005A687B681B6842F010025A6000231846CB
:103E50001037BD4680BD80B584B000AF78600023C8
:103E6000FB607B681B685A687B681B6822F0100245
:103E70005A60FCF7F3FAF86009E0FCF7EFFA024643
:103E8000FB68D31AB3F57A7F01D9032307E07B6877
:103E90001B685B6803F02003002BEED0002318465C
:103EA0001037BD4680BD80B582B000AF78607B68BA
:103EB000002B01D1012341E07B6893F83D30DBB258
:103EC000002B06D17B68002283F83C207868FBF742
:103ED00001FF7B68022283F83D207B681A687B68BB
:103EE00004331946104600F033FD7B68012283F845
:103EF00046207B68012283F83E207B68012283F8FC
:103F00003F207B68012283F840207B68012283F8F0
:103F100041207B68012283F842207B68012283F8DC
:103F200043207B68012283F844207B68012283F8C8
:103F300045207B68012283F83D200023184608377E
:103F4000BD4680BD80B582B000AF78607B68002B35
:103F500001D1012341E07B6893F83D30DBB2002BB7
:103F600006D17B68002283F83C20786800F039F89D
:103F70007B68022283F83D207B681A687B680433E3
:103F80001946104600F0E4FC7B68012283F84620C5
:103F90007B68012283F83E207B68012283F83F2062
:103FA0007B68012283F840207B68012283F841204E
:103FB0007B68012283F842207B68012283F843203A
:103FC0007B68012283F844207B68012283F8452026
:103FD0007B68012283F83D20002318460837BD4640
:103FE00080BD80B483B000AF786000BF0C37BD46A1
:103FF00080BC704780B584B000AF786039603B68A2
:10400000002B09D17B6893F83E30DBB2012B14BF43
:1040100001230023DBB222E03B68042B09D17B683B
:1040200093F83F30DBB2012B14BF01230023DBB236
:1040300015E03B68082B09D17B6893F84030DBB270
:10404000012B14BF01230023DBB208E07B6893F847
:104050004130DBB2012B14BF01230023DBB2002B64
:1040600001D0012363E03B68002B04D17B6802226E
:1040700083F83E2013E03B68042B04D17B680222C6
:1040800083F83F200BE03B68082B04D17B680222B9
:1040900083F8402003E07B68022283F841207B689C
:1040A0001B6801223968184600F0E8FE7B681B682F
:1040B000214A934207D17B681B685A6C7B681B6856
:1040C00042F400425A647B681B681B4A934213D037
:1040D0007B681B68B3F1804F0ED07B681B68174A62
:1040E000934209D07B681B68154A934204D07B68D1
:1040F0001B68144A934211D17B681B689B6803F0CC
:104100000703FB60FB68062B10D07B681B681A68EE
:104110007B681B6842F001021A6007E07B681B683D
:104120001A687B681B6842F001021A600023184677
:104130001037BD4680BD00BF002C01400004004088
:1041400000080040000C004080B582B000AF7860ED
:104150007B68002B01D1012341E07B6893F83D305F
:10416000DBB2002B06D17B68002283F83C20786804
:1041700000F039F87B68022283F83D207B681A68DA
:104180007B6804331946104600F0E2FB7B6801228D
:1041900083F846207B68012283F83E207B68012259
:1041A00083F83F207B68012283F840207B6801224E
:1041B00083F841207B68012283F842207B6801223A
:1041C00083F843207B68012283F844207B68012226
:1041D00083F845207B68012283F83D2000231846A0
:1041E0000837BD4680BD80B483B000AF786000BFA3
:1041F0000C37BD4680BC704780B584B000AF786096
:1042000039603B68002B09D17B6893F83E30DBB204
:10421000012B14BF01230023DBB222E03B68042BF7
:1042200009D17B6893F83F30DBB2012B14BF012327
:104230000023DBB215E03B68082B09D17B6893F8BB
:104240004030DBB2012B14BF01230023DBB208E0B6
:104250007B6893F84130DBB2012B14BF01230023AC
:10426000DBB2002B01D0012363E03B68002B04D1BB
:104270007B68022283F83E2013E03B68042B04D1C4
:104280007B68022283F83F200BE03B68082B04D1B7
:104290007B68022283F8402003E07B68022283F8D7
:1042A00041207B681B6801223968184600F0E6FD52
:1042B0007B681B68214A934207D17B681B685A6C54
:1042C0007B681B6842F400425A647B681B681B4A87
:1042D000934213D07B681B68B3F1804F0ED07B688C
:1042E0001B68174A934209D07B681B68154A9342A2
:1042F00004D07B681B68144A934211D17B681B6809
:104300009B6803F00703FB60FB68062B10D07B68FB
:104310001B681A687B681B6842F001021A6007E09C
:104320007B681B681A687B681B6842F001021A6090
:10433000002318461037BD4680BD00BF002C014049
:104340000004004000080040000C004080B584B02C
:1043500000AF78607B681B68DB68FB607B681B686C
:104360001B69BB60BB6803F00203002B20D0FB6815
:1043700003F00203002B1BD07B681B686FF0020266
:104380001A617B6801221A777B681B689B6903F0BE
:104390000303002B03D0786800F0BFFA05E07868CB
:1043A00000F0B2FA786800F0C1FA7B6800221A7750
:1043B000BB6803F00403002B20D0FB6803F0040368
:1043C000002B1BD07B681B686FF004021A617B68AE
:1043D00002221A777B681B689B6903F44073002BE9
:1043E00003D0786800F099FA05E0786800F08CFA5C
:1043F000786800F09BFA7B6800221A77BB6803F0AC
:104400000803002B20D0FB6803F00803002B1BD00F
:104410007B681B686FF008021A617B6804221A77B8
:104420007B681B68DB6903F00303002B03D078680B
:1044300000F073FA05E0786800F066FA786800F03A
:1044400075FA7B6800221A77BB6803F01003002B13
:1044500020D0FB6803F01003002B1BD07B681B6887
:104460006FF010021A617B6808221A777B681B685C
:10447000DB6903F44073002B03D0786800F04DFA39
:1044800005E0786800F040FA786800F04FFA7B6841
:1044900000221A77BB6803F00103002B0CD0FB68E5
:1044A00003F00103002B07D07B681B686FF001024B
:1044B0001A61786800F01FFABB6803F08003002BD4
:1044C0000CD0FB6803F08003002B07D07B681B68CF
:1044D0006FF080021A61786800F063FDBB6803F03A
:1044E0004003002B0CD0FB6803F04003002B07D0E7
:1044F0007B681B686FF040021A61786800F01FFA51
:10450000BB6803F02003002B0CD0FB6803F02003F2
:10451000002B07D07B681B686FF020021A61786857
:1045200000F036FD00BF1037BD4680BD80B586B0B7
:1045300000AFF860B9607A600023FB75FB6893F800
:104540003C30012B01D1022348E0FB68012283F8B3
:104550003C207B680C2B39D801A252F823F000BF15
:1045600095450108CD450108CD450108CD45010817
:10457000A3450108CD450108CD450108CD450108F9
:10458000B1450108CD450108CD450108CD450108DB
:10459000BF450108FB681B68B968184600F050FA6F
:1045A00017E0FB681B68B968184600F0AFFA10E026
:1045B000FB681B68B968184600F012FB09E0FB684D
:1045C0001B68B968184600F075FB02E00123FB7513
:1045D00000BFFB68002283F83C20FB7D184618379B
:1045E000BD4680BD80B586B000AFF860B9607A6026
:1045F0000023FB75FB6893F83C30012B01D10223AB
:10460000AEE0FB68012283F83C207B680C2B00F2B3
:104610009F8001A252F823F04D460108514701083E
:1046200051470108514701088D46010851470108CB
:104630005147010851470108CF4601085147010879
:1046400051470108514701080F470108FB681B68E3
:10465000B968184600F0F4F9FB681B689A69FB68B2
:104660001B6842F008029A61FB681B689A69FB6844
:104670001B6822F004029A61FB681B689969BB6899
:104680001A69FB681B680A439A6164E0FB681B684F
:10469000B968184600F03AFAFB681B689A69FB682B
:1046A0001B6842F400629A61FB681B689A69FB68A8
:1046B0001B6822F480629A61FB681B689969BB6879
:1046C0001B691A02FB681B680A439A6143E0FB6896
:1046D0001B68B968184600F083FAFB681B68DA6942
:1046E000FB681B6842F00802DA61FB681B68DA6944
:1046F000FB681B6822F00402DA61FB681B68D96959
:10470000BB681A69FB681B680A43DA6123E0FB682F
:104710001B68B968184600F0CDFAFB681B68DA69B7
:10472000FB681B6842F40062DA61FB681B68DA69A7
:10473000FB681B6822F48062DA61FB681B68D96938
:10474000BB681B691A02FB681B680A43DA6102E056
:104750000123FB7500BFFB68002283F83C20FB7D32
:1047600018461837BD4680BD80B584B000AF78606C
:1047700039600023FB737B6893F83C30012B01D137
:104780000223B4E07B68012283F83C207B6802228C
:1047900083F83D207B681B689B68BB60BB6823F087
:1047A0007703BB60BB6823F47F43BB607B681B68F7
:1047B000BA689A603B681B68B3F5005F3ED0B3F5FA
:1047C000005F00F28780B3F5805F00F08680B3F56C
:1047D000805F7FD8702B1AD0702B7BD8602B50D085
:1047E000602B77D8502B3CD0502B73D8402B58D00F
:1047F000402B6FD8302B64D0302B6BD8202B60D05F
:10480000202B67D8002B5CD0102B5AD062E07B683D
:1048100018683B6899683B685A683B68DB6800F039
:104820000EFB7B681B689B68BB60BB6843F077032B
:10483000BB607B681B68BA689A604FE07B68186849
:104840003B6899683B685A683B68DB6800F0F7FA98
:104850007B681B689A687B681B6842F480429A6098
:104860003CE07B6818683B6859683B68DB681A461F
:1048700000F06EFA7B681B685021184600F0C5FAFC
:104880002CE07B6818683B6859683B68DB681A460F
:1048900000F08CFA7B681B686021184600F0B5FABE
:1048A0001CE07B6818683B6859683B68DB681A46FF
:1048B00000F04EFA7B681B684021184600F0A5FA0C
:1048C0000CE07B681A683B681B681946104600F0CC
:1048D0009CFA03E00123FB7300E000BF7B68012228
:1048E00083F83D207B68002283F83C20FB7B184640
:1048F0001037BD4680BD80B483B000AF786000BF84
:104900000C37BD4680BC704780B483B000AF786080
:1049100000BF0C37BD4680BC704780B483B000AF89
:10492000786000BF0C37BD4680BC704780B483B050
:1049300000AF786000BF0C37BD4680BC704780B4C4
:1049400083B000AF786000BF0C37BD4680BC7047B5
:1049500080B485B000AF786039607B681B68FB600D
:104960007B68334A93420FD07B68B3F1804F0BD002
:104970007B68304A934207D07B682F4A934203D02A
:104980007B682E4A934208D1FB6823F07003FB60DA
:104990003B685B68FA681343FB607B68244A934278
:1049A0000FD07B68B3F1804F0BD07B68214A9342D4
:1049B00007D07B68204A934203D07B681F4A93420A
:1049C00008D1FB6823F44073FB603B68DB68FA683E
:1049D0001343FB60FB6823F080023B685B69134371
:1049E000FB607B68FA681A603B689A687B68DA62E9
:1049F0003B681A687B689A627B680D4A934203D1D0
:104A00003B681A697B681A637B6801225A617B687C
:104A10001B6903F00103002B05D07B681B6923F0A1
:104A200001027B681A6100BF1437BD4680BC704725
:104A3000002C01400004004000080040000C004031
:104A400080B487B000AF786039607B681B6A7B6197
:104A50007B681B6A23F001027B681A627B685B68D3
:104A60003B617B689B69FB60FB6823F07003FB6024
:104A7000FB6823F00303FB603B681B68FA68134381
:104A8000FB607B6923F002037B613B689B687A696A
:104A900013437B617B681C4A93420CD17B6923F0F2
:104AA00008037B613B68DB687A6913437B617B6940
:104AB00023F004037B617B68134A934211D13B6965
:104AC00023F480733B613B6923F400733B613B68D3
:104AD0005B693A6913433B613B689B693A691343DD
:104AE0003B617B683A695A607B68FA689A613B6807
:104AF0005A687B685A637B687A691A6200BF1C3700
:104B0000BD4680BC704700BF002C014080B487B018
:104B100000AF786039607B681B6A7B617B681B6AC9
:104B200023F010027B681A627B685B683B617B68DC
:104B30009B69FB60FB6823F4E043FB60FB6823F4A4
:104B40004073FB603B681B681B02FA681343FB6001
:104B50007B6923F020037B613B689B681B017A69BA
:104B600013437B617B681D4A93420DD17B6923F01F
:104B700080037B613B68DB681B017A6913437B61BF
:104B80007B6923F040037B617B68144A934213D115
:104B90003B6923F480633B613B6923F400633B6121
:104BA0003B685B699B003A6913433B613B689B69C7
:104BB0009B003A6913433B617B683A695A607B68A2
:104BC000FA689A613B685A687B689A637B687A697D
:104BD0001A6200BF1C37BD4680BC7047002C0140E4
:104BE00080B487B000AF786039607B681B6A7B61F6
:104BF0007B681B6A23F480727B681A627B685B683F
:104C00003B617B68DB69FB60FB6823F07003FB6042
:104C1000FB6823F00303FB603B681B68FA681343DF
:104C2000FB607B6923F400737B613B689B681B021C
:104C30007A6913437B617B681D4A93420DD17B697E
:104C400023F400637B613B68DB681B027A691343D2
:104C50007B617B6923F480637B617B68144A9342A8
:104C600013D13B6923F480533B613B6923F4005328
:104C70003B613B685B691B013A6913433B613B68DD
:104C80009B691B013A6913433B617B683A695A602F
:104C90007B68FA68DA613B685A687B68DA637B682C
:104CA0007A691A6200BF1C37BD4680BC704700BFDE
:104CB000002C014080B487B000AF786039607B6819
:104CC0001B6A3B617B681B6A23F480527B681A6213
:104CD0007B685B687B617B68DB69FB60FB6823F456
:104CE000E043FB60FB6823F44073FB603B681B6898
:104CF0001B02FA681343FB603B6923F400533B61DA
:104D00003B689B681B033A6913433B617B680F4A0E
:104D1000934209D17B6923F480437B613B685B69E3
:104D20009B017A6913437B617B687A695A607B686F
:104D3000FA68DA613B685A687B681A647B683A698A
:104D40001A6200BF1C37BD4680BC7047002C014072
:104D500080B487B000AFF860B9607A60FB681B6A06
:104D60007B61FB681B6A23F00102FB681A62FB6827
:104D70009B693B613B6923F0F0033B617B681B014E
:104D80003A6913433B617B6923F00A037B617A69CB
:104D9000BB6813437B61FB683A699A61FB687A6977
:104DA0001A6200BF1C37BD4680BC704780B487B014
:104DB00000AFF860B9607A60FB681B6A7B61FB68D2
:104DC0001B6A23F01002FB681A62FB689B693B6157
:104DD0003B6923F470433B617B681B033A691343CF
:104DE0003B617B6923F0A0037B61BB681B017A698F
:104DF00013437B61FB683A699A61FB687A691A62BE
:104E000000BF1C37BD4680BC704780B485B000AF82
:104E1000786039607B689B68FB60FB6823F07003F7
:104E2000FB603A68FB68134343F00703FB607B6851
:104E3000FA689A6000BF1437BD4680BC704780B4E2
:104E400087B000AFF860B9607A603B60FB689B6830
:104E50007B617B6923F47F437B613B681A027B683B
:104E60001A43BB6813437A6913437B61FB687A6911
:104E70009A6000BF1C37BD4680BC704780B487B0C5
:104E800000AFF860B9607A60BB6803F01F030122CD
:104E900002FA03F37B61FB681A6A7B69DB431A4001
:104EA000FB681A62FB681A6ABB6803F01F03796823
:104EB00001FA03F31A43FB681A6200BF1C37BD46B0
:104EC00080BC704780B485B000AF786039607B6883
:104ED00093F83C30012B01D102234BE07B68012287
:104EE00083F83C207B68022283F83D207B681B68A6
:104EF0005B68FB607B681B689B68BB60FB6823F09A
:104F00007003FB603B681B68FA681343FB607B68B7
:104F10001B68FA685A607B681B68194A934213D071
:104F20007B681B68B3F1804F0ED07B681B68154A05
:104F3000934209D07B681B68134A934204D07B6874
:104F40001B68124A93420CD1BB6823F08003BB60FC
:104F50003B685B68BA681343BB607B681B68BA68D0
:104F60009A607B68012283F83D207B68002283F8E9
:104F70003C20002318461437BD4680BC704700BF54
:104F8000002C01400004004000080040000C0040DC
:104F900080B483B000AF786000BF0C37BD4680BCE2
:104FA000704780B483B000AF786000BF0C37BD4657
:104FB00080BC704780B582B000AF78607B68002B02
:104FC00001D1012342E07B6893F84130DBB2002B32
:104FD00006D17B68002283F840207868FAF7C2FF88
:104FE0007B68242283F841207B681B68DA687B6831
:104FF0001B6822F40052DA60786801F003F97B68DC
:105000001B681A697B681B6822F490421A617B68EE
:105010001B685A697B681B6822F02A025A617B6808
:105020001B68DA687B681B6842F40052DA607B68B0
:1050300000225A647B68202283F841207B6820226A
:1050400083F842207B6800225A6300231846083701
:10505000BD4680BD80B58CB000AFF860B960134626
:10506000FB80FB6893F84130DBB2202B56D1BB6844
:10507000002B02D0FB88002B01D101234FE0BA683E
:10508000FB681A62FB68FA889A84FB68FA88DA84FB
:10509000FB6800225A64FB68212283F84120FB68E8
:1050A0009B6B214A9A62FB689B6B204ADA62FB6821
:1050B0009B6B1F4A1A63FB689B6B00225A6307F1C4
:1050C0000803FB62FB68986BFB6A1968FB681B6846
:1050D00004331A46FB88FCF7A5FFFB681B686FF0DA
:1050E00040021A60FB681B681433BB61BB6953E85C
:1050F000003F7B617B6943F08003BB62FB681B68F8
:105100001433BA6A7A623B62396A7A6A41E80023E8
:10511000FB61FB69002BE5D1002300E00223184668
:105120003037BD4680BD00BF295A0108C35A010867
:10513000475C010880B58CB000AFF860B9601346D9
:10514000FB80FB6893F84230DBB2202B4AD1BB686E
:10515000002B02D0FB88002B01D1012343E0FB6828
:1051600001221A63FB6800225A63FB881A46B96859
:10517000F86800F0B2FD034687F82F3097F82F301B
:10518000002B2CD1FB681B6B012B25D100233B612D
:10519000FB681B681B683B61FB681B685B683B61C5
:1051A0003B69FB681B680C33BB61BB6953E8003F7C
:1051B0007B617B6943F01003BB62FB681B680C33A7
:1051C000BA6A7A623B62396A7A6A41E80023FB6113
:1051D000FB69002BE5D102E0012387F82F3097F817
:1051E0002F3000E0022318463037BD4680BD80B521
:1051F0008CB000AFF860B9601346FB80FB6893F891
:105200004230DBB2202B46D1BB68002B02D0FB889A
:10521000002B01D101233FE0FB6801221A63FB68E8
:1052200000225A63FB881A46B968F86800F08EFDC0
:10523000034687F82F30FB681B6B012B25D1002319
:105240003B61FB681B681B683B61FB681B685B6814
:105250003B613B69FB681B680C33BB61BB6953E86E
:10526000003F7B617B6943F01003BB62FB681B68F6
:105270000C33BA6A7A623B62396A7A6A41E800237F
:10528000FB61FB69002BE5D102E0012387F82F3099
:1052900097F82F3000E0022318463037BD4680BD16
:1052A00080B58EB000AF78607B681B680C333B62C2
:1052B0003B6A53E8003FFB61FB6923F0C0037B635B
:1052C0007B681B680C337A6BFA62BB62B96AFA6A54
:1052D00041E800237B627B6A002BE5D17B681B6879
:1052E0005B6903F08003002B36D07B681B681433A6
:1052F000FB60FB6853E8003FBB60BB6823F08003A2
:105300003B637B681B6814333A6BBA617B617969D4
:10531000BA6941E800233B613B69002BE5D17B681A
:105320009B6B002B18D07B689B6B00225A637B68B9
:105330009B6B1846FCF7D6FE0346002B0CD07B680F
:105340009B6B1846FDF74EFA0346202B04D17B6871
:1053500010225A64032307E07B680022DA847B680A
:10536000202283F84120002318463837BD4680BDEF
:1053700080B59AB000AF78607B681B680C33BB6463
:10538000BB6C53E8003F7B647B6C23F490737B66BB
:105390007B681B680C337A6E7A653B65396D7A6D74
:1053A00041E80023FB64FB6C002BE5D17B681B68A4
:1053B00014337B637B6B53E8003F3B633B6B23F011
:1053C00001033B667B681B6814333A6E3A64FB63E7
:1053D000F96B3A6C41E80023BB63BB6B002BE5D152
:1053E0007B681B6B012B19D17B681B680C333B62FC
:1053F0003B6A53E8003FFB61FB6923F01003FB6548
:105400007B681B680C33FA6DFA62BB62B96AFA6A90
:1054100041E800237B627B6A002BE5D17B681B6837
:105420005B6903F04003002B36D07B681B681433A4
:10543000FB60FB6853E8003FBB60BB6823F04003A0
:10544000BB657B681B681433BA6DBA617B6179698F
:10545000BA6941E800233B613B69002BE5D17B68D9
:10546000DB6B002B18D07B68DB6B00225A637B68F8
:10547000DB6B1846FCF736FE0346002B0CD07B682E
:10548000DB6B1846FDF7AEF90346202B04D17B6891
:1054900010225A6403230AE07B680022DA857B68C5
:1054A000202283F842207B6800221A6300231846DA
:1054B0006837BD4680BD000080B5BAB000AF7860E7
:1054C0007B681B681B68C7F8E4307B681B68DB6877
:1054D000C7F8E0307B681B685B69C7F8DC300023E5
:1054E000C7F8D8300023C7F8D430D7F8E43003F039
:1054F0000F03C7F8D830D7F8D830002B0FD1D7F822
:10550000E43003F02003002B09D0D7F8E03003F09B
:105510002003002B03D0786800F0B6FD5BE2D7F8DB
:10552000D830002B00F0DE80D7F8DC3003F0010328
:10553000002B06D1D7F8E03003F49073002B00F075
:10554000D180D7F8E43003F00103002B0BD0D7F85B
:10555000E03003F48073002B05D07B685B6C43F074
:1055600001027B685A64D7F8E43003F00403002B8F
:105570000BD0D7F8DC3003F00103002B05D07B689B
:105580005B6C43F002027B685A64D7F8E43003F0A6
:105590000203002B0BD0D7F8DC3003F00103002B03
:1055A00005D07B685B6C43F004027B685A64D7F8D3
:1055B000E43003F00803002B11D0D7F8E03003F0FB
:1055C0002003002B05D1D7F8DC3003F00103002BBA
:1055D00005D07B685B6C43F008027B685A647B688B
:1055E0005B6C002B00F0F281D7F8E43003F020036D
:1055F000002B08D0D7F8E03003F02003002B02D0B6
:10560000786800F041FD7B681B685B6903F040032C
:10561000002B14BF01230023DBB2C7F8D4307B6812
:105620005B6C03F00803002B03D1D7F8D430002BB8
:105630004FD0786800F04BFC7B681B685B6903F017
:105640004003002B41D07B681B681433C7F89C30A3
:10565000D7F89C3053E8003FC7F89830D7F8983017
:1056600023F04003C7F8D0307B681B681433D7F8A9
:10567000D020C7F8A820C7F8A430D7F8A410D7F8CE
:10568000A82041E80023C7F8A030D7F8A030002BAD
:10569000D9D17B68DB6B002B13D07B68DB6B7E4A38
:1056A0005A637B68DB6B1846FCF758FD0346002BFA
:1056B00016D07B68DB6B5B6B7A68D26B10469847C1
:1056C0000EE07868F8F738FB0AE07868F8F734FB02
:1056D00006E07868F8F730FB7B6800225A6475E1D1
:1056E00000BF73E17B681B6B012B40F04F81D7F843
:1056F000E43003F01003002B00F04881D7F8E030CD
:1057000003F01003002B00F041810023BB607B6895
:105710001B681B68BB607B681B685B68BB60BB6801
:105720007B681B685B6903F04003002B00F0B680C8
:105730007B68DB6B1B685B68A7F8BE30B7F8BE30D0
:10574000002B00F045817B689B8DB7F8BE209A4204
:1057500080F03E817B68B7F8BE20DA857B68DB6B22
:105760009B69202B00F088807B681B680C33C7F88E
:105770008830D7F8883053E8003FC7F88430D7F82E
:10578000843023F48073C7F8B8307B681B680C330F
:10579000D7F8B820C7F89420C7F89030D7F8901001
:1057A000D7F8942041E80023C7F88C30D7F88C3024
:1057B000002BD9D17B681B6814337B677B6F53E860
:1057C000003F3B673B6F23F00103C7F8B4307B68B1
:1057D0001B681433D7F8B420C7F88020FB67F96F33
:1057E000D7F8802041E80023BB67BB6F002BE1D1D5
:1057F0007B681B6814333B663B6E53E8003FFB65D8
:10580000FB6D23F04003C7F8B0307B681B6814338E
:10581000D7F8B020FA66BB66B96EFA6E41E800238D
:105820007B667B6E002BE3D17B68202283F84220CD
:105830007B6800221A637B681B680C33FB64FB6C7B
:1058400053E8003FBB64BB6C23F01003C7F8AC30D7
:105850007B681B680C33D7F8AC20BA657B65796D23
:10586000BA6D41E800233B653B6D002BE3D17B68BB
:10587000DB6B1846FCF736FC7B6802225A637B68B8
:105880009A8D7B68DB8D9BB2D31A9BB219467868E0
:10589000F9F7C2F99CE000BF935F01087B689A8D1D
:1058A0007B68DB8D9BB2D31AA7F8CE307B68DB8D8B
:1058B0009BB2002B00F08E80B7F8CE30002B00F0AA
:1058C00089807B681B680C33BB63BB6B53E8003F6C
:1058D0007B637B6B23F49073C7F8C8307B681B68CD
:1058E0000C33D7F8C8207A643B64396C7A6C41E891
:1058F0000023FB63FB6B002BE3D17B681B68143335
:105900007B627B6A53E8003F3B623B6A23F0010302
:10591000C7F8C4307B681B681433D7F8C4203A63D7
:10592000FB62F96A3A6B41E80023BB62BB6A002B59
:10593000E3D17B68202283F842207B6800221A632F
:105940007B681B680C333B613B6953E8003FFB609D
:10595000FB6823F01003C7F8C0307B681B680C336A
:10596000D7F8C020FA61BB61B969FA6941E8002340
:105970007B617B69002BE3D17B6802225A63B7F815
:10598000CE3019467868F9F747F923E0D7F8E430C4
:1059900003F08003002B09D0D7F8E03003F0800338
:1059A000002B03D0786800F008FB14E0D7F8E4304F
:1059B00003F04003002B0ED0D7F8E03003F0400393
:1059C000002B08D0786800F047FB04E000BF02E03D
:1059D00000BF00E000BFE837BD4680BD80B483B0A3
:1059E00000AF786000BF0C37BD4680BC704780B404
:1059F00083B000AF786000BF0C37BD4680BC7047F5
:105A000080B483B000AF786000BF0C37BD4680BC67
:105A1000704780B483B000AF78607B685B6C1846D9
:105A20000C37BD4680BC704780B590B000AF786041
:105A30007B685B6AFB637B681B681B6803F0200361
:105A4000002B37D1FB6B0022DA84FB6B1B6814330D
:105A50007B627B6A53E8003F3B623B6A23F0800332
:105A6000BB63FB6B1B681433BA6B3A63FB62F96A66
:105A70003A6B41E80023BB62BB6A002BE5D1FB6BAC
:105A80001B680C333B613B6953E8003FFB60FB68DC
:105A900043F040037B63FB6B1B680C337A6BFA614A
:105AA000BB61B969FA6941E800237B617B69002B1E
:105AB000E5D102E0F86BF9F729F900BF4037BD46A0
:105AC00080BD80B584B000AF78607B685B6AFB60A6
:105AD000F868FFF783FF00BF1037BD4680BD80B573
:105AE0009CB000AF78607B685B6AFB667B681B6874
:105AF0001B6803F02003002B72D1FB6E0022DA85B5
:105B0000FB6E1B680C33FB64FB6C53E8003FBB640B
:105B1000BB6C23F48073BB66FB6E1B680C33BA6EE0
:105B2000BA657B65796DBA6D41E800233B653B6DD5
:105B3000002BE5D1FB6E1B681433BB63BB6B53E8D2
:105B4000003F7B637B6B23F001037B66FB6E1B686E
:105B500014337A6E7A643B64396C7A6C41E80023C2
:105B6000FB63FB6B002BE5D1FB6E1B6814337B6280
:105B70007B6A53E8003F3B623B6A23F040033B668D
:105B8000FB6E1B6814333A6E3A63FB62F96A3A6B38
:105B900041E80023BB62BB6A002BE5D1FB6E2022EB
:105BA00083F84220FB6E1B6B012B19D1FB6E1B6827
:105BB0000C333B613B6953E8003FFB60FB6823F01B
:105BC0001003FB65FB6E1B680C33FA6DFA61BB6159
:105BD000B969FA6941E800237B617B69002BE5D153
:105BE000FB6E00225A63FB6E1B6B012B06D1FB6E12
:105BF0009B8D1946F86EF9F70FF802E0F86EFFF783
:105C0000F6FE00BF7037BD4680BD80B584B000AFE2
:105C100078607B685B6AFB60FB6801225A63FB6803
:105C20001B6B012B08D1FB689B8D5B089BB219464F
:105C3000F868F8F7F1FF02E0F868FFF7E1FE00BF4F
:105C40001037BD4680BD80B584B000AF78600023BA
:105C5000FB607B685B6ABB60BB681B685B6903F0C9
:105C60008003002B14BF01230023DBB2FB60BB6861
:105C700093F84130DBB2212B08D1FB68002B05D013
:105C8000BB680022DA84B86800F0FAF8BB681B68C9
:105C90005B6903F04003002B14BF01230023DBB238
:105CA000FB60BB6893F84230DBB2222B08D1FB6863
:105CB000002B05D0BB680022DA85B86800F007F930
:105CC000BB685B6C43F01002BB685A64B868F8F7B5
:105CD00033F800BF1037BD4680BD80B485B000AF3B
:105CE000F860B9601346FB80FB68BA689A62FB688B
:105CF000FA889A85FB68FA88DA85FB6800225A647C
:105D0000FB68222283F84220FB681B69002B07D026
:105D1000FB681B68DA68FB681B6842F48072DA6013
:105D2000FB681B685A69FB681B6842F001025A61F4
:105D3000FB681B68DA68FB681B6842F02002DA60C7
:105D4000002318461437BD4680BC704780B598B014
:105D500000AFF860B9601346FB80BA68FB689A62CE
:105D6000FB68FA889A85FB6800225A64FB68222245
:105D700083F84220FB68DB6B3E4A9A62FB68DB6B70
:105D80003D4ADA62FB68DB6B3C4A1A63FB68DB6BFB
:105D900000225A6307F10803FB65FB68D86BFB68B8
:105DA0001B6804331946FB6D1A68FB88FCF73AF947
:105DB00000233B61FB681B681B683B61FB681B6839
:105DC0005B683B613B69FB681B69002B19D0FB6872
:105DD0001B680C333B643B6C53E8003FFB63FB6B7D
:105DE00043F48073BB65FB681B680C33BA6DFA64BF
:105DF000BB64B96CFA6C41E800237B647B6C002BBC
:105E0000E5D1FB681B681433FB62FB6A53E8003F73
:105E1000BB62BB6A43F001037B65FB681B681433FC
:105E20007A6DBA637B63796BBA6B41E800233B639D
:105E30003B6B002BE5D1FB681B681433BB61BB696E
:105E400053E8003F7B617B6943F040033B65FB689F
:105E50001B6814333A6D7A623B62396A7A6A41E8A8
:105E60000023FB61FB69002BE5D100231846603756
:105E7000BD4680BDDF5A01080B5C0108475C010884
:105E800080B489B000AF78607B681B680C33FB601E
:105E9000FB6853E8003FBB60BB6823F0C003FB61B5
:105EA0007B681B680C33FA69BA617B617969BA69EE
:105EB00041E800233B613B69002BE5D17B68202250
:105EC00083F8412000BF2437BD4680BC704780B4B2
:105ED00095B000AF78607B681B680C337B637B6B8D
:105EE00053E8003F3B633B6B23F49073FB647B6898
:105EF0001B680C33FA6C3A64FB63F96B3A6C41E84B
:105F00000023BB63BB6B002BE5D17B681B6814339C
:105F10003B623B6A53E8003FFB61FB6923F00103EE
:105F2000BB647B681B681433BA6CFA62BB62B96AE3
:105F3000FA6A41E800237B627B6A002BE5D17B682B
:105F40001B6B012B19D17B681B680C33FB60FB6852
:105F500053E8003FBB60BB6823F010037B647B68A1
:105F60001B680C337A6CBA617B617969BA6941E864
:105F700000233B613B69002BE5D17B68202283F83D
:105F800042207B6800221A6300BF5437BD4680BCA4
:105F9000704780B584B000AF78607B685B6AFB6057
:105FA000FB680022DA85FB680022DA84F868F7F7DC
:105FB000C3FE00BF1037BD4680BD80B485B000AFC2
:105FC00078607B6893F84130DBB2212B3ED17B684F
:105FD0009B68B3F5805F14D17B681B69002B10D1DF
:105FE0007B681B6AFB60FB681B881A467B681B6822
:105FF000C2F308025A607B681B6A9A1C7B681A62AB
:1060000008E07B681B6A591C7A6811621A787B6801
:106010001B685A607B68DB8C9BB2013B9BB27A6841
:106020001946D184002B0FD17B681B68DA687B6826
:106030001B6822F08002DA607B681B68DA687B6884
:106040001B6842F04002DA60002300E00223184699
:106050001437BD4680BC704780B582B000AF786011
:106060007B681B68DA687B681B6822F04002DA6094
:106070007B68202283F841207868F8F747FE0023E8
:1060800018460837BD4680BD80B58CB000AF78603B
:106090007B6893F84230DBB2222B40F0AE807B6805
:1060A0009B68B3F5805F17D17B681B69002B13D108
:1060B0000023FB627B689B6ABB627B681B685B6832
:1060C0009BB2C3F308039AB2BB6A1A807B689B6ACF
:1060D0009A1C7B689A6226E07B689B6AFB620023BD
:1060E000BB627B689B68B3F5805F07D07B689B6869
:1060F000002B0AD17B681B69002B06D17B681B68CB
:106100005B68DAB2FB6A1A7008E07B681B685B6840
:10611000DBB203F07F03DAB2FB6A1A707B689B6A1A
:106120005A1C7B689A627B68DB8D9BB2013B9BB2F9
:106130007A681946D185002B5DD17B681B68DA68C7
:106140007B681B6822F02002DA607B681B68DA68D3
:106150007B681B6822F48072DA607B681B685A696E
:106160007B681B6822F001025A617B68202283F859
:1061700042207B6800225A637B681B6B012B35D160
:106180007B6800221A637B681B680C337B617B6928
:1061900053E8003F3B613B6923F010037B627B685F
:1061A0001B680C337A6A3A62FB61F9693A6A41E822
:1061B0000023BB61BB69002BE5D17B681B681B68B2
:1061C00003F01003102B0AD10023FB607B681B68CF
:1061D0001B68FB607B681B685B68FB60FB687B6817
:1061E0009B8D19467868F8F717FD02E07868FFF78D
:1061F000FEFB002302E0002300E0022318463037B4
:10620000BD4680BD80B584B000AF78607B681B68F8
:106210001B6923F440517B68DA687B681B680A437A
:106220001A617B689A687B681B691A437B685B69A3
:106230001343BB607B681B68DB6823F4B05323F017
:106240000C037A681268B9680B43D3607B681B68DB
:106250005B6923F440717B689A697B681B680A4319
:106260005A617B681B682C4A934203D1FDF75CFAA4
:10627000F86002E0FDF744FAF860FA6813469B0004
:1062800013449A001A447B685B689B00B2FBF3F3EB
:10629000224AA2FB03235B091901FA6813469B00FB
:1062A00013449A001A447B685B689B00B2FBF3F2CC
:1062B0001A4BA3FB02035B09642000FB03F3D31A10
:1062C0001B013233154AA2FB03235B0903F0F003E1
:1062D0001944FA6813469B0013449A001A447B68D9
:1062E0005B689B00B2FBF3F20C4BA3FB02035B0960
:1062F000642000FB03F3D31A1B013233074AA2FBCD
:1063000003235B0903F00F027B681B680A449A6051
:1063100000BF1037BD4680BD003801401F85EB51DE
:10632000002B2DE9F0471D46BBBF03F100431D467E
:1063300000232D2388B01446B8BF1446129A109E2D
:106340001370149BDDF84CA023F02008B8F1460F21
:1063500005D0B8F1450F00D10136022300E0032338
:1063600007AA049206AACDE902A2CDE90036224688
:106370002B4600F0B5FEB8F1470F074619D1119B27
:10638000DB070ED500EB0609002200232046294634
:10639000F2F776FB08B1CDF81C903022079B4B45F5
:1063A0001ED33846079B159ADB1B136008B0BDE867
:1063B000F087B8F1460F00EB0609E5D10378302BE2
:1063C0000AD10022002320462946F2F759FB18B9CA
:1063D000C6F10106CAF80060DAF800309944D3E744
:1063E000591C07911A70D9E7F7B50029B6BF2D23BC
:1063F0002B23494209290270437029DD0DF107035F
:106400001D460A27B1FBF7F61A4607FB161430346F
:1064100002F8014C0C46632C314603F1FF33F1DCEA
:106420003031941E03F8011C2346411CAB420AD3B1
:106430000DF109039B1AAC4288BF002302330344C9
:10644000181A03B0F0BD13F8016B01F8016FEDE706
:10645000302330318370C170031DF1E72DE9F04F17
:1064600091B00C46DDF8688016461F46054600F0E0
:10647000FBFC036818460893F1F7D6FE00230E9341
:10648000D8F800300990073323F0070303F108021E
:1064900094F818A0D4F800B0C8F80020D3E9008917
:1064A00029F000430B93CDF828804FF0FF32DDE94F
:1064B0000A01C4E912899C4BF2F714FB70BBDDE9B9
:1064C0000A014FF0FF32984BF2F7EEFA30BB002290
:1064D000002340464946F2F7DDFA10B12D2384F837
:1064E0004330924A924BBAF1470F8CBF9046984680
:1064F00003234FF0000923612BF00403236033468C
:106500002146284600970FAA00F0D4F9013040F048
:1065100090804FF0FF3011B0BDE8F08F42464B46FF
:1065200040464946F2F7DEFA48B14B46002BB8BF69
:106530002D23804AB8BF84F843307F4BD3E763688C
:106540000AF0DF015A1C3FD10623636000224BF49E
:106550008063236006920EAACDE904A20DAA0392DD
:106560000DF13302CDE901326368424600932846BB
:106570004B460A91FFF7D4FE0A99804647290D99A8
:1065800028D1C81C02DB6368994240DDAAF1020AE7
:106590005FFA8AFA5246013904F150000D91FFF773
:1065A00023FF0E9A81461318012A236102DC226818
:1065B000D20701D5013323619DF83330002B9ED0E3
:1065C0002D2384F843309AE74729BFD1002BBDD152
:1065D0000123BAE7BAF1650FDCD9BAF1660F18D119
:1065E000002963680BDD216113B92268D00702D549
:1065F00001330B4423614FF00009A165DCE713B9B7
:106600002268D20701D50233F4E70123F2E74FF005
:10661000670A0E9B994205DB23682161D807EAD5FA
:106620004B1CE7E70029CCBF0122C1F10202134451
:10663000E0E723685A0507D42369424631462846D5
:10664000B84701302BD164E7BAF1650F40F2DC8026
:10665000D4E9120100220023F2F712FA002833D005
:10666000012331462846354AB84701303FF451AF3F
:10667000DDE90D38434502DB2368D8070FD5DDE996
:10668000082331462846B84701303FF442AF4FF067
:10669000000908F1FF3804F11A0AC84509DC23682B
:1066A0009B0700F10281E0680F9B9842B8BF184633
:1066B00031E70123524631462846B84701303FF4BE
:1066C00028AF09F10109E8E70D9B002B38DC012315
:1066D00031462846194AB84701303FF41AAFDDE980
:1066E0000D3959EA030302D12368D907D7D5DDE96B
:1066F000082331462846B84701303FF40AAF4FF02F
:10670000000A04F11A0B0D9B5B42534501DC4B461A
:1067100093E701235A4631462846B84701303FF4F3
:10672000F8AE0AF1010AEEE7FFFFEF7F68A101086A
:1067300064A1010870A101086CA1010874A10108FD
:10674000A36DDDF838A05345A8BF5346002B9946EA
:1067500036DC4FF0000B29EAE97904F11A02A36D47
:106760000A93A3EB09035B4531DC0D9B9A453ADCA8
:106770002368DA0737D40D9BAAEB03090A9BAAEB1F
:1067800003039945A8BF9946B9F1000F33DC4FF0D8
:10679000000829EAE97904F11A0B0D9BAAEB03031F
:1067A000A3EB090343457FF77AAF01235A463146ED
:1067B0002846B84701303FF4ACAE08F10108ECE7D9
:1067C000424631462846B8470130C2D1A1E60123EE
:1067D000314628460A92B84701303FF49AAE0A9AE9
:1067E0000BF1010BBBE73146DDE908232846B8472A
:1067F0000130C0D18DE60A9A4B46314628464244C4
:10680000B8470130C3D184E6DDF838A0BAF1010FF2
:1068100001DCDB0736D50123424631462846B8471E
:1068200001303FF476AEDDE9082331462846B8470B
:1068300001303FF46EAED4E91201002200230AF1C8
:10684000FF3AF2F71DF9C0B9534608F1010231468B
:106850002846B84701300CD15BE601235A46314641
:106860002846B84701303FF454AE08F10108D0453E
:10687000F3DB4B4604F15002E0E64FF0000804F170
:106880001A0BF4E701234246E1E701234A46314669
:106890002846B84701303FF43CAE08F10108E368F0
:1068A0000F995B1A4345F0DCFDE64FF0000804F158
:1068B0001909F4E72DE9F047164698468A680B69EE
:1068C00007469342B8BF1346336091F843200C4605
:1068D000DDF820900AB1013333602368990642BF86
:1068E000336802333360256815F0060506D104F1DC
:1068F000190AE36832689B1AAB422BDC94F84330E8
:106900002268003B18BF0123920630D44146384626
:1069100004F14302C847013023D02368226903F001
:106920000603042B14BF002533684FF0000608BF90
:10693000E56804F11A0408BFED1A54F8123C08BFC8
:1069400025EAE5759342C4BF9B1AED18B5421AD1EA
:10695000002008E00123524641463846C84701302E
:1069600003D14FF0FF30BDE8F0870135C1E730209B
:10697000E11881F843005A1C94F845102244023370
:1069800082F84310C2E70123224641463846C847F1
:106990000130E6D00136D9E72DE9FF470F7E914659
:1069A000782F80460C469A460C9E01F1430207D888
:1069B000622F0AD8002F00F0D180582F00F0B88045
:1069C00004F1420684F842703AE0A7F16303152B04
:1069D000F6D801A151F823F0316A0108456A01088F
:1069E000C1690108C1690108C1690108C1690108DB
:1069F000456A0108C1690108C1690108C169010846
:106A0000C1690108436B01086F6A0108FD6A01084A
:106A1000C1690108C1690108656B0108C169010804
:106A20006F6A0108C1690108C1690108056B0108A5
:106A300033681A1D1B68326004F1420684F8423044
:106A400001239CE033682068191D3160060601D5DA
:106A50001D6803E04506FBD5B3F90050002D03DAAD
:106A60002D236D4284F843300A23584811E02168F1
:106A70003368080653F8045B02D4490648BFADB238
:106A80006F2F336014BF0A2308235048002184F875
:106A900043106668002EA66005DB21682E4321F0B6
:106AA000040121604BD01646B5FBF3F103FB1157EF
:106AB000C75D06F8017D2F46BB420D46F4D9082B71
:106AC0000BD12368DF0708D5236961689942DEBFCF
:106AD000302306F8013C06F1FF36921B22614B463B
:106AE00021464046CDF800A003AAFFF7E3FE01309F
:106AF0004AD14FF0FF3004B0BDE8F087236843F07F
:106B0000200323607827324884F845702368316871
:106B10001F0651F8045B02D45F0648BFADB2316076
:106B2000D90744BF43F0200323601DB11023ADE714
:106B30002648E9E7236823F020032360F6E716469A
:106B4000BDE733682568181D616930602E061B6833
:106B500001D5196002E06806FBD5198000231646AE
:106B60002361BCE7336800211A1D32601E68626829
:106B7000304600F0F0F908B1801B60606368236163
:106B8000002384F84330AAE7324649464046236949
:106B9000D0470130ADD023689B0713D4E068039B36
:106BA0009842B8BF1846A6E70123324649464046F8
:106BB000D04701309DD00135E36803995B1AAB42A1
:106BC000F2DCEBE7002504F11906F5E776A10108F0
:106BD00087A10108002310B50446C0E90033C0E9CD
:106BE0000433836081814366C28183611946082230
:106BF0005C3000F031F90D4B246263620C4BA362F0
:106C00000C4BE3620C4B23630C4B9C4206D003F10C
:106C10006802944202D0D0339C4205D104F158005E
:106C2000BDE8104000F094B910BD00BF596D0108D7
:106C30007B6D0108B36D0108D76D01086015002058
:106C4000024A0349034800F069B800BF5C00002015
:106C5000298901086C00002041680C4B10B599424D
:106C6000044601D001F060FEA168094B994202D0B0
:106C7000204601F059FEE168064B994204D02046B7
:106C8000BDE8104001F050BE10BD00BF60150020EF
:106C9000C81500203016002010B50B4B0B4C0C4AC9
:106CA00020461A6004210022FFF794FF04F16800D7
:106CB00001220921FFF78EFF04F1D0000222BDE876
:106CC00010401221FFF786BF9816002060150020A3
:106CD000416C0108014800F03CB900BFA11600203A
:106CE000014800F037B900BFA116002010B50446D6
:106CF000FFF7F0FF236A1BB1BDE81040FFF7F0BFBC
:106D0000044B2362044B1B68002BF5D1FFF7C4FF33
:106D1000F2E700BF596C0108981600202DE9F843EE
:106D20000746884614460026D4E90195B9F10109C1
:106D300005D52468002CF7D13046BDE8F883AB892F
:106D4000012B07D9B5F90E30013303D02946384657
:106D5000C04706436835E9E710B50C46B1F90E1097
:106D600000F0A8F80028ABBF636DA3891B1823F4BB
:106D70008053ACBF6365A38110BD2DE9F0411F4670
:106D80008B890546DB050C46164605D502230022F5
:106D9000B1F90E1000F07CF8A389324623F4805339
:106DA000A38128463B46B4F90E10BDE8F04100F03F
:106DB00093B810B50C46B1F90E1000F069F8431CF9
:106DC000A38915BF606523F4805343F48053A381E6
:106DD00018BFA38110BDB1F90E1000F049B830B54D
:106DE0001446002C05461A469BB005DA8B23036037
:106DF0004FF0FF301BB030BD4FF40273ADF80C30D4
:106E00004FF0000319930CBF234604F1FF330293A4
:106E100005934FF6FF7300910491ADF80E3069466B
:106E20001E9B01F005FC431CBCBF8B232B60002C78
:106E3000E0D00022009B1A70DCE7000007B5009349
:106E400013460A46014603480068FFF7C8FF03B02F
:106E50005DF804FB6800002003460244934200D121
:106E6000704703F8011BF9E700487047A8010020AC
:106E700038B50023054D044608462B60F8F7A3FDFE
:106E8000431C02D12B6803B1236038BD9C1600203F
:106E900038B50446084611460022054D2A601A46B8
:106EA000F8F7B5FD431C02D12B6803B1236038BD50
:106EB0009C16002038B50446084611460022054DB0
:106EC0002A601A46F8F762FD431C02D12B6803B111
:106ED000236038BD9C16002038B50446084611468C
:106EE0000022054D2A601A46F3F720FB431C02D10D
:106EF0002B6803B1236038BD9C160020014B186835
:106F0000704700BF6800002070B500260C4D0D4C86
:106F1000641BA410A64209D102F076F800260A4D9F
:106F20000A4C641BA410A64205D170BD55F8043B61
:106F300098470136EEE755F8043B98470136F2E7EB
:106F4000E4A40108E4A40108E4A40108E8A40108F9
:106F5000704770477047034610B5C9B20244934268
:106F6000184601D1002003E0047801338C42F6D1A9
:106F700010BD0A44914200F1FF3300D1704710B5B3
:106F800011F8014B914203F8014FF9D110BD0000F7
:106F90001FB514461A46094B05461B68D8684CB104
:106FA000074BCDE9013400912B46064901F0E4FC82
:106FB00001F01EFD044B1C46F3E700BF68000020F3
:106FC00098A10108A5A10108D3A101082DE9F74F57
:106FD00003690C690746A3427EDB013CA30000F174
:106FE000140501F11408009305EB8403019358F88C
:106FF000243055F8242001339A42B2FBF3F608EB13
:1070000084092ED34FF0000AC446AE46D3465CF83E
:10701000043B98B206FB00A01B0C020C06FB0323EA
:10702000DEF8002080B292B2121A5A44DEF8000054
:107030004FEA134A9BB2C3EB224303EB104392B2D5
:1070400042EA0342E1454FEA234B4EF8042BDED2DD
:10705000009BEB582BB9019B043B9D421A462FD352
:107060003C61384601F080F9002825DB29460020E4
:1070700058F8042BD1F800C01FFA82FE1FFA8CF3D7
:10708000A3EB0E030344120CC2EB234202EB1C429F
:107090009BB243EA0243C1454FEA224041F8043B18
:1070A000E6D255F8242005EB840322B9043B9D4227
:1070B0001A460BD33C610136304603B0BDE8F08F71
:1070C0001268043B002ACBD1013CC6E71268043B9E
:1070D000002AEFD1013CEAE70020EEE700000000C3
:1070E0002DE9F04F14461D46C76997B08146CDE99A
:1070F0000645239E7FB9102000F00EFE0246C9F817
:107100001C0020B9EF21AC4BAC48FFF741FFC0E9B0
:1071100001770760C760D9F81C30196859B15A68FF
:10712000012393404A608B60484600F0EBFE00224A
:10713000D9F81C301A602B1EAFBF0023012223F0A8
:1071400000430793A8BF3360DDF81C809C4BB8BF99
:10715000326033EA080312D142F20F73229A1360AD
:10716000C8F31303234300F05E85249BDFF854A289
:10717000002B00F060850AF1030300F05ABDDDE941
:107180000623CDE90C23DDE90C0100220023F1F7F1
:1071900077FC074658B10123229A1360249B13B150
:1071A000894B249A1360DFF824A200F044BD14AB8D
:1071B000019315AB00934846DDE90C2301F084F9F7
:1071C000C8F30A560390002E78D0DDE90C010D9B20
:1071D000A6F2FF36C3F3130343F07F5343F4401387
:1071E0001297194600227A4BF1F72AF86CA3D3E9DB
:1071F0000023F1F7DDF96CA3D3E90023F1F722F8BE
:10720000044630460D46F1F769F969A3D3E9002336
:10721000F1F7CEF902460B4620462946F1F712F85F
:1072200004460D46F1F774FC002207460023204671
:107230002946F1F72FFC40B13846F1F74FF92246C5
:107240002B46F1F71DFC00B9013F162F54D8DDE99C
:107250000C01604B03EBC703D3E90023F1F71AFCE1
:1072600000284BD00023013F0F93149B9B1B5A1EF9
:1072700049BFC3F10103002304930023099254BFC3
:1072800004930993002F3BDB099B0E973B44099322
:1072900000230A93209B092B65D8052BC4BF043B10
:1072A0002093209BC8BF0024A3F10203D8BF012470
:1072B000032B64D8DFE803F05355382CDDE9146361
:1072C0001E4406F23243202BC1BFC3F1400308FA2B
:1072D00003F806F2124324FA03F3D6BFC3F12003E6
:1072E00048EA030004FA03F0F1F7E8F80122A1F1FB
:1072F000F873013E129274E70123B5E70F90B4E7EB
:10730000049BDB1B04937B420A9300230E93C1E78B
:1073100001230B93219B07EB030B0BF10103012BC3
:107320000893B8BF012306E001230B93219B002B98
:1073300028DD9B46089300210422D9F81C0002F1A5
:1073400014059D4226D94160484600F09BFD8246C7
:10735000002843D1024640F2AF111F4BD4E6002370
:10736000E3E70023D5E7012400230B9420934FF09B
:10737000FF3B00221223CDF820B02192DBE701234E
:107380000B93F4E74FF0010B5B46CDF820B0CDF83E
:1073900084B0D0E701315200D1E700BFAFF30080E5
:1073A00061436F63A787D23FB3C8608B288AC63F0B
:1073B000FB799F501344D33FE1A10108F8A10108D4
:1073C0000000F07FDDA1010875A1010874A101088A
:1073D0000000F83F10A3010850A20108D9F81C30A2
:1073E0001860089B0E2B00F2A180002C00F09E80FC
:1073F000002F33DD9C4B07F00F0203EBC203F805AF
:10740000D3E90034CDE910344FEA271416D5DDE96D
:107410000C01964B0326D3E90823F1F7F3F9CDE9E4
:10742000060104F00F04914D54B9DDE91023DDE9A4
:107430000601F1F7E7F9CDE9060128E00226F2E7B7
:10744000E10708D5DDE91001D5E90023F1F7B0F82F
:10745000CDE91001013664100835E5E700F0AF8092
:10746000DDE90C017C42804B04F00F0203EBC20308
:10747000D3E90023F1F79CF802260023CDE90601A9
:107480007A4D2411002C40F08F80002BD3D1DDE900
:1074900006450F9B002B00F09480002220462946D1
:1074A000734BF1F7F7FA002800F08B80089B002B54
:1074B00000F08780BBF1000F34DD20460022294612
:1074C0006C4BF1F775F85C46CDE9060107F1FF3822
:1074D00001363046F1F702F8DDE90623F1F768F8E6
:1074E0000022654BF0F7AEFE0546A1F15076002C68
:1074F0006AD1DDE906010022604BF0F7A1FE0246E9
:107500000B46CDE906232A463346F1F7E1FA002877
:1075100040F09882DDE906012A4606F10043F1F7C2
:10752000B9FA38BBDDE90C34CDE90634159B002BE4
:10753000C0F257810E2F00F354814B4B03EBC7036E
:10754000D3E90034CDE90434219B002B80F2E5809F
:10755000089B002B00F3E1800CD1DDE9040100223F
:10756000464BF1F725F8DDE90623F1F7A7FA0028E5
:1075700000F0668200242546219B56466FEA0308E8
:1075800000272146484600F0BDFC002D00F0BD80DC
:107590002FB1AF4203D03946484600F0B3FC29462C
:1075A000484600F0AFFCB0E0E20705D5D5E900237E
:1075B000F0F7FEFF012301366410083562E702266A
:1075C00065E7B846089C84E7274B0B9903EBC40397
:1075D00053E902235444002954D000202849F1F7EC
:1075E00011F933462A46F0F72BFE5646CDE9100135
:1075F000DDE90601F1F78CFA0546F0F76FFF024668
:107600000B46DDE90601F0F71BFE02460B4630355E
:10761000CDE90623DDE9102306F8015BF1F73AFA1C
:10762000002872D1DDE9062300201149F0F708FE99
:10763000DDE91023F1F72EFA002840F0B480A642CD
:107640003FF470AFDDE9100100220A4BF0F7B0FF04
:107650000022CDE91001DDE90601064BF0F7A8FF95
:10766000CDE90601C4E700BF10A30108E8A20108A4
:107670000000F03F0000244000001C4000001440C7
:107680000000E03F31462846F0F792FF5646CDE92C
:1076900010011394DDE90601F1F73AFA0546F0F717
:1076A0001DFF02460B46DDE90601F0F7C9FD024663
:1076B0000B46303506F8015BA642CDE906234FF0B4
:1076C000000224D1DDE91001AE4BF0F7BBFD02460C
:1076D0000B46DDE90601F1F7FBF9002863D1DDE98E
:1076E00010230020A749F0F7ABFD02460B46DDE969
:1076F0000601F1F7CFF900283FF414AF139E731E73
:10770000139316F8013C302BF8D047463BE09E4BD4
:10771000F0F74EFFCDE90601BCE75646DDE9064528
:10772000DDE9042320462946F1F76CF8F1F7F0F97A
:107730008046F0F7D3FEDDE90423F0F739FF024677
:107740000B4620462946F0F77BFD08F13004089DE2
:1077500006F8014BA6EB0A04A54202460B4633D1BC
:10776000F0F770FDDDE9042304460D46F1F7B0F9AA
:10777000C0B9DDE9042320462946F1F781F910B1AB
:1077800018F0010F0ED14846039900F0BBFB00230F
:107790003370229B01371F60249B002B00F04B822B
:1077A0001E6048E2B84633461E4613F8012D392ABA
:1077B00006D19A45F8D1302208F101088AF8002054
:1077C0001A7801321A70A0E700226F4BF0F7F0FE32
:1077D0000022002304460D46F1F752F900289FD0FD
:1077E000D1E70B9A002A00F0EA80209A012A00F3E0
:1077F000CD80129A002A00F0C18003F233430A9C24
:10780000049E049A01211A440492099A48461A4493
:10781000099200F02BFC054666B1099B002B09DD9F
:10782000B342A8BF3346049AF61AD21A0492099AB0
:10783000D31A09930A9B0BB30B9B002B00F0C68055
:10784000002C00F0C08029462246484600F0C6FCC5
:10785000039A01460546484600F01EFC03998046FF
:10786000484600F04FFB0A9B1B1B0A9300F0B180B7
:1078700041460A9A484600F0B1FC0390012148466F
:1078800000F0F4FB0E9B0446002B00F0D8811A4652
:107890000146484600F0A2FC209B0446012B00F361
:1078A0009F80069B002B40F09780079BC3F3130338
:1078B000002B40F09380079B23F000431B0D1B051A
:1078C00033B1049B01330493099B013309930123D2
:1078D0000A930E9B002B00F0B881236904EB83030D
:1078E000186900F077FBC0F12000099B184410F0E4
:1078F0001F0000F08280C0F12003042B73DD049B85
:10790000C0F11C0003440493099B064403440993FB
:10791000049B002B05DD1A464846039900F0B8FC8D
:107920000390099B002B05DD21461A46484600F0CE
:10793000AFFC04460F9B002B61D02146039800F05A
:1079400013FD00285BDA00230A224846039900F061
:10795000FBFA0B9B07F1FF380390002B00F07781B7
:10796000294600230A22484600F0EEFABBF1000F38
:1079700005466FDC209B022B49DC6BE0149BC3F1B6
:1079800036033CE70000E03F00002440089B5C1EFB
:107990000A9BA34209DB1C1B089B002BBFF630AFE0
:1079A000049B089A9E1A00232BE70A9B0E9AE31A5F
:1079B0001A440A94049E0024089B0E9221E70A9C14
:1079C000049E0B9D28E7DDF80C8051E70A9A039985
:1079D00050E7CDF80C8051E7002379E7069B77E765
:1079E00000230A9379E793D0049A1C331A44049233
:1079F000099A1E441A4409928AE70346F4E7089B51
:107A0000B846002B20DC9B46209B022B1EDDBBF1E1
:107A1000000F7FF4B1AD21465B460522484600F0D9
:107A200093FA01460446039800F09EFC00287FF775
:107A3000A3AD5646312308F1010806F8013B9FE546
:107A4000B846089C2546F4E7DDF820B00B9B002BD8
:107A500000F00181002E05DD29463246484600F03F
:107A600017FC05460A9B002B5CD04846696800F06D
:107A700009FA064628B9024640F2EF21804BFFF78B
:107A800043BB2A6905F10C01023292000C30FFF76A
:107A900070FA01223146484600F0FAFB2F460546AF
:107AA0000AF1010304930AEB0B030A93069B03F00C
:107AB00001030993049B2146039803F1FF3BFFF761
:107AC00085FA034639463033069003980B9300F04D
:107AD0004BFC2A4608902146484600F061FCC268EB
:107AE00006460B9B02BB0146039800F03DFC024694
:107AF0000B9B31464846CDE90B3200F003FA209B40
:107B00000C9A049E42EA0301099B19430B9B0DD179
:107B1000392B27D0089A002A01DD069B31338BF8D8
:107B200000302EE52846B9E70122E2E7089900294E
:107B300004DB209801430998014320D1002AEEDD9F
:107B4000012203994846049300F0A2FB21460390CA
:107B500000F00AFC0028049B02DCE0D1DA07DED545
:107B6000392BDAD139238BF8003033461E4616F80C
:107B7000012C013B392A4ED001321A7001E5002A4E
:107B800003DD392BEED00133C9E7049A0A9902F8D4
:107B9000013C8A4228D000230A220399484600F07B
:107BA000D3F9AF4203904FF000034FF00A02394679
:107BB000484607D100F0C8F907460546049B013343
:107BC000049377E700F0C0F92946074600230A220C
:107BD000484600F0B9F90546F0E7BBF1000FCCBF0D
:107BE0005E46012600275644012203994846049325
:107BF00000F04EFB2146039000F0B6FB0028B4DCF9
:107C000002D1049BDB07B0D433461E4613F8012D86
:107C1000302AFAD0B5E49A45A8D1312308F10108F9
:107C20008AF80030ADE4249BDFF858A01BB10AF1BC
:107C30000803249A1360504617B0BDE8F08F209BCC
:107C4000012B7FF72EAE0E9B0A9301204DE6BBF170
:107C5000000F7FF7D9AE564621460398FFF7B6F9D5
:107C600000F1300306F8013BA6EB0A029345B4DDB0
:107C700000230A224846039900F066F90390EBE7D7
:107C800050A20108D4A1010838B50546002940D00A
:107C900051F8043C0C1F002BB8BFE41800F0E6F8C4
:107CA0001C4A136833B9636014602846BDE8384045
:107CB00000F0E2B8A34208D9206821188B4201BF26
:107CC00019685B6809182160EDE71A465B680BB11B
:107CD000A342FAD911685018A0420BD12068014480
:107CE000501883421160E0D118685B680844106046
:107CF0005360DAE702D90C232B60D6E720682118FD
:107D00008B4201BF19685B68091821606360546089
:107D1000CBE738BDA8160020024B0146186800F0DA
:107D200025B800BF6800002070B50F4E0C463168C2
:107D3000054611B900F04CFE30602146284600F09F
:107D400047FE431C03D14FF0FF34204670BDC41CD6
:107D500024F00304A042F8D0211A284600F038FE8F
:107D60000130F2D1EFE700BFA41600202DE9F8435F
:107D7000CD1C25F0030508350C2D38BF0C25002D32
:107D8000064601DBA94204D90C2333600020BDE87C
:107D9000F883DFF8D48000F069F8D8F800301C468A
:107DA00044BB29463046FFF7BFFF431C044658D169
:107DB000D8F800402746002F43D1002C4BD0236831
:107DC0003946304604EB030900F002FE814542D1FA
:107DD000216830466D1A2946FFF7A6FF01303AD0D8
:107DE00023682B442360D8F800305A6862BBC8F877
:107DF00000700FE02268521B20D40B2A17D961199A
:107E0000A342256018BF5960636808BFC8F8001016
:107E100062514B60304600F02FF804F10B00231D37
:107E200020F00700C21A1CBF1B1AA350AFE76268FC
:107E3000A3420CBFC8F800205A60EBE723466468F1
:107E4000AEE73C467F68B6E71A465B68A342FBD1C3
:107E500000235360DEE70C233046336000F00CF85B
:107E600094E70560D6E700BFA81600200148FFF799
:107E700070B800BFA01600200148FFF76BB800BF24
:107E8000A016002070B5C66904460D4676B91020CC
:107E9000FFF742FF0246E06120B96B21174B1848FB
:107EA000FFF776F8C0E901660660C660E669F36828
:107EB00083B1E369DB6853F82500B8B9012101FA01
:107EC00005F6721D2046920000F099FD60B1C0E9F0
:107ED00001560EE021220421204600F090FDE369C6
:107EE000F060DB68002BE4D1002070BD026843F82D
:107EF00025200023C0E90333F7E700BFE1A1010813
:107F000061A2010870B5C66905460C4676B9102015
:107F1000FFF702FF0246E86120B98F21084B0948AC
:107F2000FFF736F8C0E901660660C6603CB1EB6950
:107F30006268DB6853F82210216043F8224070BD6C
:107F4000E1A1010861A201082DE9F04107460C46B4
:107F50001E4600200D6901F1140CDCF800300130E0
:107F600099B202FB01611E0C0B0C02FB063389B2B5
:107F700001EB034185424FEA13464CF8041BECDC4D
:107F80000EB3A368AB4219DC616838460131FFF7D4
:107F900079FF804628B90246BA210C4B0C48FEF7FF
:107FA000F7FF226904F10C01023292000C30FEF757
:107FB000E0FF21463846FFF7A5FF444604EB850362
:107FC00001355E6125612046BDE8F08150A20108BF
:107FD00061A201080346B0F5803F3ABF03041020B8
:107FE0000020B3F1807F3CBF1B020830B3F1805FFB
:107FF0003CBF1B010430B3F1804F3CBF9B000230FB
:10800000002B05DB13F0804F00F1010008BF20209A
:1080100070470368024613F007000BD0D90721D43C
:10802000980749BF5B089B08012013605CBF0220D2
:108030001360704799B209B910201B0CD9B209B965
:1080400008301B0A190704BF1B090430990704BF35
:108050009B080230D90703D45B0800F1010003D06C
:1080600013607047002070472020704710B50C4601
:108070000121FFF707FF024628B940F24511044BE2
:108080000448FEF785FF01234461036110BD00BF72
:1080900050A2010861A201082DE9F04F17460A69B4
:1080A0003B6989469A42A2BF3B460F4699463D69C5
:1080B000D9F810A0BB68796805EB0A06B34285B011
:1080C000B8BF0131FFF7DEFE30B902464FF4B1719F
:1080D000404B4148FEF75CFF00F1140423460022A8
:1080E00004EB860E734520D307F1140809F114013F
:1080F00008EB850501EB8A030293EB1B153B23F08C
:10810000030304331537BD4238BF04230193029B98
:1081100003918B420CD8002E03DD5EF8043D002B4A
:1081200055D0066105B0BDE8F08F43F8042BD9E7C0
:10813000B1F800A0BAF1000F1FD0C446A146002735
:108140005CF8042BD9F800301FFA82FB9BB20AFBC3
:108150000B333B44D9F80070120C3F0C0AFB02723F
:1081600002EB13429BB243EA024365454FEA1247D2
:1081700049F8043BE4D8019BE750039B0431B3F872
:108180000290B9F1000F20D04746A4464FF0000AF4
:108190002368B7F800B0BCF802209BB209FB0B22A1
:1081A000524443EA02434CF8043B57F8043B4FEA7D
:1081B000134ABCF80030BD4209FB0A3303EB1243FB
:1081C0004FEA134AE5D8019AA35004349FE7013ED1
:1081D000A1E700BF50A2010861A201082DE9F84300
:1081E000154612F0030207460E4607D0254C013A09
:1081F000002354F82220FFF7A7FE0646AD103DD01D
:10820000FC697CB91020FFF787FD0246F86128B9A8
:1082100040F2B3111C4B1D48FEF7BAFEC0E9014401
:108220000460C460D7F81C80D8F808404CB940F20C
:1082300071213846FFF71AFF00230446C8F80800EA
:1082400003604FF00009EB070AD531462246384655
:10825000FFF722FF804631463846FFF753FE464679
:108260006D100BD0206838B9224621463846FFF7FA
:1082700013FF2060C0F800900446E4E73046BDE8F4
:10828000F88300BFD8A20108E1A1010861A201089A
:108290002DE9F0470C46074691462369496803EBF0
:1082A0006218A3684FEA621A08F10106B3420BDBB9
:1082B0003846FFF7E7FD054648B902464FF4EF712F
:1082C000274B2848FEF764FE01315B00EEE70023F0
:1082D00000F1140100F110021846534533DB206908
:1082E0002AEAEA7A04F1140319F01F0901EB8A0162
:1082F00003EB800C2BD08A460022C9F1200E1868AF
:1083000000FA09F010434AF8040B53F8042B9C457B
:1083100022FA0EF2F3D8ACEB0403153B23F003036F
:10832000043304F11500604588BF0423CA500AB124
:1083300008F10206013E384621462E61FFF7E2FDB4
:108340002846BDE8F08742F8040F0133C5E7043939
:1083500053F8042B9C4541F8042FF9D8EAE700BFF5
:1083600050A2010861A2010803460A69006930B5FC
:10837000801A0ED11433143103EB820401EB820115
:1083800054F8045D51F8042D954203D005D24FF006
:10839000FF3030BDA342F3D3FBE70120F9E7000033
:1083A0002DE9F74F89460646114648461446FFF721
:1083B000DBFF051E12D129463046FFF763FD02465A
:1083C00028B940F237213E4B3E48FEF7E1FD01233C
:1083D000C0E90435104603B0BDE8F08FBCBF4B4682
:1083E000A1463046D9F80410BABF1C460125002525
:1083F000FFF748FD024618B940F24521304BE3E74C
:1084000000F1140BD9F8107009F11003C5604FF09A
:10841000000C09F11405D946266904F1140E05EB88
:1084200087080EEB86060193019B5EF8040B53F858
:1084300004AF81B201931FFA8AF35B1A000C634404
:10844000C0EB1A4000EB23409BB243EA0043764561
:108450004FEA204C49F8043BE6D8331B153B23F088
:10846000030315340433A64238BF04231D445B4480
:108470001E462C4644450ED308F10301491B21F04A
:108480000301033DA84538BF00210B4453F8041DE8
:1084900099B117619EE7E64654F8041B1FFA81FC68
:1084A000F444080C714400EB2C4089B241EA0041CD
:1084B0004FEA204C46F8041BDCE7013FE6E700BF2B
:1084C00050A2010861A201082DE9734301219046E1
:1084D0009946089EFFF7D6FC044630B9024640F2A2
:1084E0000F31234B2348FEF753FDC9F30A55C9F357
:1084F00013030DB143F480130193B8F1000324D0AA
:1085000068460093FFF785FDDDE90012D8B1C0F1A0
:10851000200302FA03F30B43C24063610192019B03
:10852000002B0CBF01220222A3612261ADB1A5F292
:10853000334505443560C0F13500099B186020467D
:1085400002B0BDE870836161E9E701A8FFF761FD52
:10855000019B012263612030E7E7A0F2324004EB87
:10856000820330601869FFF735FDC0EB4210E4E785
:1085700050A2010861A201082DE9F0471F468E684C
:108580008246BE420C4690460B682DD8B1F90C20AD
:1085900012F4906F26D06569096905EB4505A3EBD8
:1085A000010905EBD5757B1C4B446D109D4238BF0E
:1085B0001D46530527D52946FFF7D8FB064660B36D
:1085C0004A462169FEF7D5FCA38923F4906343F062
:1085D0008003A38126614E4426603E466561A5EB7B
:1085E0000905A560BE4200D93E4632464146206894
:1085F00000F0D4F90020A3689B1BA36023683344D8
:108600002360BDE8F0872A4600F01FFA06460028DE
:10861000E0D150462169FFF737FB0C23CAF8003040
:10862000A3894FF0FF3043F04003A381E9E7000046
:108630002DE9F04F98468B8907461B060D461446D8
:108640009DB010D50B6973B94021FFF78FFB2860EF
:10865000286130B90C233B604FF0FF301DB0BDE8FE
:10866000F08F40236B610023099320238DF829307C
:1086700030234FF00109CDF80C80DFF898818DF898
:108680002A3023469A4613F8012B0AB1252AF9D13C
:10869000BAEB040B0BD05B46224629463846FFF75F
:1086A0006BFF013000F0A780099A5A4409929AF8AA
:1086B0000030002B00F09F8000234FF0FF32CDE907
:1086C00005230AF1010A049307938DF853301A9396
:1086D0005446052214F8011B4E48FEF73CFC049A50
:1086E000D8B9D00644BF20238DF85330110744BFBA
:1086F0002B238DF853309AF800302A2B15D054468E
:1087000000204FF00A0C079A214611F8013B303B3C
:10871000092B4BD9B0B1079214E0A0EB080309FA7A
:1087200003F31343A2460493D2E7039B191D1B686E
:108730000391002BBBBF5B4242F0020207930793F9
:10874000B8BF049223782E2B0AD163782A2B32D11A
:10875000039B02341A1D1B68039243EAE3730593DB
:10876000DFF8B4A0032250462178FEF7F4FB38B1BD
:108770004022049BA0EB0A0082401343013404937F
:1087800014F8011B062225488DF82810FEF7E3FB9C
:10879000002836D0224B1BBB039B073323F0070373
:1087A00008330393099B334409936AE70C4601207D
:1087B0000CFB0232A8E700234FF00A0C19460134E3
:1087C0000593204610F8012B303A092A03D9002BD3
:1087D000C6D00591C4E7044601230CFB0121F0E754
:1087E00003AB00932A4638460E4B04A9FDF736FE2C
:1087F000421C0646D6D1AB895B063FF52DAF0998E2
:108800002CE703AB00932A463846064B04A9FEF733
:10881000C3F8EDE7BAA20108C0A20108C4A201088A
:108820005D64010879850108B1F90C20F8B51607D7
:1088300005460C4654D44B68002B02DC0B6C002B15
:1088400048DDE66A002E45D0002312F480522F68DE
:10885000216A2B6030D0626DA389590705D5636802
:10886000D21A636B0BB1236CD21A00232846E66A36
:10887000216AB047431CA38906D129681D292BD83A
:10888000284ACA40D60727D5002262602269D90447
:10889000226004D5421C01D12B6803B96065616B6D
:1088A0002F60B9B104F14403994202D02846FFF782
:1088B000EBF9002363630DE001232846B04702462D
:1088C000501CC9D12B68002BC6D01D2B01D0162BF4
:1088D0001DD12F60002021E043F040031BB21AE0BD
:1088E0000F69002FF6D0930718BF00230E6808BF4A
:1088F0004B69F61B0F608B60002EEBDD33463A466A
:108900002846216AD4F828C0E047002807DCB4F9DB
:108910000C3043F040034FF0FF30A381F8BD074413
:10892000361AE9E70100402038B50B6905460C46C8
:1089300013B90025284638BD18B1036A0BB9FEF7F4
:10894000D5F9B4F90C30002BF3D0626ED00704D403
:10895000990502D4A06DFEF7FCFA28462146FFF7E0
:1089600063FF636E0546DA07E4D4A3899B05E1D46F
:10897000A06DFEF7EFFADDE70EB403B5014603ABD9
:10898000054853F8042B0068019300F0C1F802B0C9
:108990005DF804EB03B0704768000020884210B512
:1089A00001EB020402D98442234607D8431EA142A8
:1089B00008D011F8012B03F8012FF8E70146024413
:1089C0008A4200D110BD13F8014D02F8014DF7E7BE
:1089D00038B50023054D044608462B60F7F724F808
:1089E000431C02D12B6803B1236038BD9C160020C4
:1089F000062008B500F060FA0120F6F7BCFF70B55C
:108A0000A1FB025434B92946FFF7B0F9064628B94C
:108A1000304670BD0C2200260260F9E72A46214646
:108A2000FEF71AFAF4E782B001B901A942B14BB1DD
:108A300013780B601278101E18BF012002B0704727
:108A40001046FBE76FF00100F8E72DE9F04107461B
:108A500014460D4621B91146BDE8F041FFF786B92D
:108A60002AB9FFF711F925462846BDE8F08100F044
:108A70003FFA8442064602D8B4EB500FF4D82146A0
:108A80003846FFF773F9804608B94546ECE7B4422B
:108A90002246294628BF3246FEF76BFA2946384659
:108AA000FFF7F2F8F1E70346084641B1FF2A04D97F
:108AB0008A224FF0FF301A60704701200A70704719
:108AC000936810B4013B002B936007DA9469A342CA
:108AD00001DB0A2902D110BC00F032B91368581C1E
:108AE00010601970084610BC7047F8B506460F466E
:108AF0001446D518AC4201D1002007E03A46304672
:108B000014F8011BFFF7DCFF431CF3D1F8BD000094
:108B10002DE9F04F0D461446984606469DB018B113
:108B2000036A0BB9FEF7E2F86B6ED90705D4AB897F
:108B30009A0502D4A86DFEF70CFAAB891B0701D584
:108B40002B699BB92946304600F038F970B16B6E3D
:108B5000DC0704D54FF0FF301DB0BDE8F08FAB89C6
:108B60009805F7D4A86DFEF7F5F9F3E7002309930C
:108B700020238DF8293030234FF00109CDF80C80E7
:108B8000DFF8A8818DF82A3023469A4613F8012B86
:108B90000AB1252AF9D1BAEB040B0BD05B46224669
:108BA00029463046FFF7A1FF013000F0A780099A5F
:108BB0005A4409929AF80030002B00F09F8000235D
:108BC0004FF0FF32CDE905230AF1010A0493079320
:108BD0008DF853301A935446052214F8011B53485C
:108BE000FEF7B9F9049AD8B9D10644BF20238DF80D
:108BF0005330130744BF2B238DF853309AF80030BD
:108C00002A2B15D0544600204FF00A0C079A214613
:108C100011F8013B303B092B4BD9B0B1079214E05E
:108C2000A0EB080309FA03F31343A2460493D2E727
:108C3000039B191D1B680391002BBBBF5B4242F0D5
:108C4000020207930793B8BF049223782E2B0AD110
:108C500063782A2B32D1039B02341A1D1B680392BE
:108C600043EAE3730593DFF8C8A003225046217856
:108C7000FEF771F938B14022049BA0EB0A00824054
:108C800013430134049314F8011B062229488DF87C
:108C90002810FEF760F900283FD0274B1BBB039B31
:108CA000073323F0070308330393099B3B440993DD
:108CB0006AE70C4601200CFB0232A8E700234FF0C4
:108CC0000A0C194601340593204610F8012B303A5E
:108CD000092A03D9002BC6D00591C4E70446012315
:108CE0000CFB0121F0E703AB00932A463046134BFF
:108CF00004A9FDF7B3FB0746781CD6D16B6ED907E4
:108D000005D4AB899A0502D4A86DFEF723F9AB8987
:108D10005B063FF51FAF09981EE703AB00932A4699
:108D20003046064B04A9FDF737FEE4E7BAA2010876
:108D3000C0A20108C4A201085D640108EB8A010811
:108D4000F8B50E461446054618B1036A0BB9FDF78F
:108D5000CDFFA369A360A3891A0701D5236943B98D
:108D60002146284600F02AF818B14FF0FF37384660
:108D7000F8BD23682269F6B2981A636937468342C0
:108D800005DC21462846FFF7CFFD0028EDD1A3687A
:108D9000013BA36023685A1C22601E706269431C59
:108DA0009A4204D0A389DB07E1D50A2EDFD1214600
:108DB0002846FFF7B9FD0028D9D0D6E738B5294BAA
:108DC000054618680C4618B1036A0BB9FDF78EFF0B
:108DD000B4F90C30190722D4DA0607D409222A6024
:108DE00043F040034FF0FF30A38133E0580712D522
:108DF000616B41B104F14403994202D02846FEF769
:108E000043FF00236363A38923F02403A38100238A
:108E1000636023692360A38943F00803A381236966
:108E20004BB9A38903F42073B3F5007F03D0214627
:108E3000284600F08AF8B4F90C3013F001020AD089
:108E40000022A26062695242A261226942B913F013
:108E50008000C5D138BD990758BF6269A260F4E7A8
:108E60000020F7E7680000201F2938B505460C46AA
:108E700004D9162303604FF0FF3038BDC26B12B126
:108E800052F821304BB9284600F030F8224601460E
:108E90002846BDE8384000F017B8012B0AD0591C0D
:108EA00003D1162303600120E7E70021204642F8A2
:108EB000241098470020E0E7024B01461868FFF7AE
:108EC000D3BF00BF6800002038B50023064D04461C
:108ED000084611462B60F6F73EFD431C02D12B6875
:108EE00003B1236038BD00BF9C160020F6F72CBDEF
:108EF00051F8043C181F002BBCBF0B58C01870471A
:108F000070B50C46B1F90E10154600291E4696B0F4
:108F10000CDAA389002113F0800F14BF40234FF413
:108F20008063002031602B6016B070BD6A4600F08F
:108F300049F80028EDDB019901F47041A1F50053D7
:108F4000594259414FF48063EBE78B89F7B59D0790
:108F500006460C4607D504F147032360236101232D
:108F6000636103B0F0BD6A4601ABFFF7C9FF009F24
:108F7000054639463046FEF7F9FE48B9B4F90C30DB
:108F80009A05EED423F0030343F00203A381E2E742
:108F9000A389C4E9040743F08003A381019B2060F7
:108FA0005BB13046B4F90E1000F01EF828B1A38969
:108FB00023F0030343F00103A381A3891D43A5818B
:108FC000CFE7000038B50023064D04460846114699
:108FD0002B60F6F703FD431C02D12B6803B123601D
:108FE00038BD00BF9C16002038B50023054D04464F
:108FF00008462B60F6F701FD431C02D12B6803B134
:10900000236038BD9C160020F8B500BFF8BC08BC32
:109010009E467047F8B500BFF8BC08BC9E46704736
:10902000434F4E4E30204572726F723A2025640ACB
:1090300000000000436F6E6E6563746F723A2055D6
:109040006E6B6E6F776E0A00436F6E6E6563746F42
:10905000723A20556E706C75676765640A0000008F
:10906000436F6E6E6563746F723A20446973616218
:109070006C65640A00000000436F6E6E6563746F78
:10908000723A20507265706172696E670A00000062
:10909000436F6E6E6563746F723A204175746852E7
:1090A000657175697265640A00000000436F6E6E39
:1090B0006563746F723A2057616974696E67466FB1
:1090C00072456E657267790A00000000436F6E6E2C
:1090D0006563746F723A204368617267696E6750A6
:1090E000617573656445560A00000000436F6E6E3B
:1090F0006563746F723A204368617267696E675086
:109100006175736564455653450A0000436F6E6E82
:109110006563746F723A204368617267696E670AAB
:1091200000000000436F6E6E6563746F723A2041F9
:1091300075746854696D656F75740A00436F6E6E5F
:109140006563746F723A2046696E69736865640A74
:1091500000000000436F6E6E6563746F723A2046C4
:10916000696E6973686564455653450A00000000DE
:10917000436F6E6E6563746F723A2046696E6973F1
:1091800068656445560A0000436F6E6E6563746FD0
:10919000723A205265706C756767696E670A0000E5
:1091A0004350207374617465206368616E67656401
:1091B0003A202564202D3E2025640A004350206477
:1091C000757479206368616E6765643A202575203F
:1091D0002D3E2025750A00004649524520414C414C
:1091E000524D206163746976617465640A00000001
:1091F0004661737420646973636861726765207483
:109200007269676765722025752D3E257520493D79
:1092100025750A004661737420646973636861721E
:10922000676520636F6D706C6574652C20563D25F5
:10923000750A000046617374206469736368617223
:1092400067652061626F727465642C20563D2575D8
:109250000A000000434353206D6F64756C652073F2
:10926000746172740A00000053657269616C206E4B
:10927000756D6265723A2025640A0000426F617262
:1092800064207265766973696F6E3A2025640A00FE
:10929000436F6E6E6563746F722063757272656E74
:1092A00074206C696D69743A2025752E25752041EE
:1092B0000A00000046572076657273696F6E3A2087
:1092C00025642E25642E25640A000000554E524563
:1092D00041445900494E4954000000005245414460
:1092E00059000000574149545F4F4E00434F4E54C0
:1092F0005F4F4E00434F4E4E4543544544000000DF
:1093000046445F4F4646000046445F57414954007B
:1093100046445F534554000046445F4F4E000000F2
:1093200046445F4F4E5F5741495400004355525FDA
:1093300044524F5000000000434F4E545F4F46468A
:1093400000000000574149545F4F464600000000AE
:109350004F46465F50415553450000003F00000016
:1093600050535520646961672073743D25732072E2
:1093700065713D2575562F25752E25754120776120
:109380006E743D2575562F25752E25754120636118
:109390006E3D2575562F25752E257541206D65610D
:1093A000733D2575562F25642E25754120656E4F1A
:1093B00075743D2575206F75743D2575207264792F
:1093C0003D2575206F6E3D257520636F6E743D25BC
:1093D000752061633D25752068763D257520707385
:1093E000645F626C6B3D2575206572723D2575204A
:1093F00073303D3078253032782073313D30782518
:109400003032782073323D307825303278206361F5
:109410006E5F6167653D256C756D730A0000000025
:109420002073630020756E6576656E0020696E742A
:109430005F636F6D6D00000020696E5F6275730081
:10944000206C6F636B000000206469736368000028
:1094500020656570726F6D002064635F6F666600E3
:10946000206661756C7400002070726F74000000DB
:109470002066616E00000000206F7400206F6F7620
:1094800000000000206F6F63000000002063616E29
:109490005F696E740000000020706C696D00000050
:1094A00020616464725F64757000000020756E65F1
:1094B00076656E5F686900002070685F6C6F73731B
:1094C0000000000020756E62616C0000207576005F
:1094D000206F7600207066635F6F66660000000094
:1094E00050535520666C616773257325732573256A
:1094F00073257325732573257325732573257325AC
:10950000732573257325732573257325732573259B
:10951000732573257325730A0000000050535520EE
:10952000737461747573206368616E67652073304E
:109530003D3078253032782D3E3078253032782015
:1095400073313D3078253032782D3E3078253032F9
:10955000782073323D3078253032782D3E307825B2
:109560003032780A0000000050535520737564644F
:10957000656E6C792064697361626C6564207768DC
:10958000696C65206368617267696E6720726561E6
:10959000736F6E3D63616E5F6C6F737420563D2513
:1095A0007520493D256420636F6E743D25752073D9
:1095B000303D3078253032782073313D3078253099
:1095C00032782073323D3078253032782063616EF6
:1095D0005F6167653D256C756D730A0050535520BA
:1095E00073756464656E6C792064697361626C651F
:1095F00064207768696C65206368617267696E676B
:1096000020726561736F6E3D6F75747075745F6CF9
:109610006F737420563D257520493D256420636F86
:109620006E743D25752073303D30782530327820BA
:1096300073313D3078253032782073323D307825D3
:109640003032782063616E5F6167653D256C756DB2
:10965000730A00004856206C696D69742072657346
:109660006574206F7574707574206F66660A0000EB
:109670004856206C696D6974207265736574206E3C
:109680006F205053550A00004856206C696D69746C
:10969000204F4E20563D256420493D256420636EB1
:1096A000743D25640A0000004856206C696D697499
:1096B000206C6F636B656420636E743D25640A00E3
:1096C0004856206C696D6974204F464620563D25EA
:1096D0006420493D256420636E743D25640A0000C2
:1096E0005053552073742025732D3E257320656ECD
:1096F0004F75743D2575207264793D2575206F6E18
:109700003D257520636F6E743D2575206572723D31
:1097100025750A005053552043414E2074696D65EC
:109720006F7574206167653D256C756D73202D3EE6
:10973000206F66666C696E650A0000005053552004
:109740006F6E2074696D656F75740A004443206301
:109750006F6E746163746F7220636C6F73656420E5
:1097600028434F4E545F4F4E2D3E434F4E4E454380
:109770005445442C2066623D25752C20743D256C93
:10978000756D73290A000000436F6E746163746F16
:1097900072206572726F722C2073746F7070696EB4
:1097A000672E2E2E0A0000004661737420646973D0
:1097B0006368617267652061626F7274202D3E205C
:1097C00073746F700A0000004661737420646973DB
:1097D000636861726765206F66662061636B2C2029
:1097E000563D2575202D3E207365742025750A0091
:1097F0004661737420646973636861726765206F82
:1098000066662074696D656F75742C20563D2575EC
:109810000A000000466173742064697363686172B2
:109820006765206F6E2074696D656F75742C2056A6
:109830003D25752028746172676574202575290A95
:1098400000000000444320636F6E746163746F72A4
:10985000206F70656E20636D6420284355525F440D
:10986000524F502D3E434F4E545F4F46462C204999
:109870003D25752C207761697465643D256C756D97
:1098800073290A00444320636F6E746163746F72BE
:10989000206F70656E6564202866623D302C2074F0
:1098A0003D256C756D73290A000000004443206358
:1098B0006F6E746163746F72206F70656E2074696F
:1098C0006D656F7574202872656C61793D25752012
:1098D00066623D25752C20743D256C756D73290AD3
:1098E00000000000505355206F66662074696D6556
:1098F0006F75740A00000000504520004E4520009E
:10990000464520004F52452000000000444D4120B4
:10991000000000005541525425752048414C2065F7
:1099200072726F72206465636F64653A204E4F4EA9
:10993000450A00005541525425752048414C206588
:1099400072726F72206465636F64653A20257325B7
:10995000732573257325732573207261773D3078E5
:109960002530386C780A0000554152543320525843
:109970002061726D206661696C65642028257329F9
:109980003A2048414C5F5374617475733D256420DF
:109990006572725F61667465723D30782530386C2F
:1099A000780A000055415254332052582061726D9C
:1099B000206661696C65642064657461696C73001C
:1099C00055415254332052582064726F703A2077B8
:1099D000726F6E6720687561727420696E205278AC
:1099E0004576656E7443616C6C6261636B202873AD
:1099F000697A653D2575290A0000000055415254D9
:109A0000332052582064726F703A20527845766540
:109A10006E742073697A653D30202869646C652C0A
:109A2000206E6F207061796C6F6164290A000000FC
:109A300052784576656E7443616C6C6261636B004D
:109A400055415254332052582064726F703A20733B
:109A5000697A653D2575203E2072785F627566667D
:109A6000657220257520286F766572666C6F772C7D
:109A7000206E6F7420706172736564290A000000A3
:109A80005541525425752048414C206572726F72C1
:109A90002028495352293A207261773D3078253089
:109AA000386C7820E28094205258206D61792062D1
:109AB0006520636F7272757074656420756E746969
:109AC0006C2072652D61726D0A0000004572726F24
:109AD0007243616C6C6261636B00000055415254CB
:109AE0003320545820444D4120726573656E6420C4
:109AF0006661696C656400004553544F5020747270
:109B0000696767657265640A0000000053746F70CE
:109B100070696E67206368617267696E672E2E2EAA
:109B20000A00000046696E697368656445562C201A
:109B300073746F7070696E672E2E2E0A000000001D
:109B4000457665726573742074696D656F75740A06
:109B500000000000457665726573742074696D6558
:109B60006F75742C2073746F7070696E67206368F2
:109B7000617267696E672E2E2E0A0000436861725B
:109B800067696E67206572726F722025642C20737E
:109B900074617465202D3E2064697361626C656434
:109BA0000A0000004368617267696E672070657221
:109BB0006D69747465642C207374617274206368B9
:109BC000617267696E670A0043617220756E706C1E
:109BD00075676765640A00005265706C7567676930
:109BE0006E672E2E2E0A00005265706C75676769CD
:109BF0006E672066696E69736865642C206275748F
